Archive member included to satisfy reference by file (symbol)

/opt/st/stm32cubeide_1.9.0/plugins/com.st.stm32cube.ide.mcu.externaltools.gnu-tools-for-stm32.10.3-2021.10.linux64_1.0.0.202111181127/tools/bin/../lib/gcc/arm-none-eabi/10.3.1/../../../../arm-none-eabi/lib/thumb/v6-m/nofp/libc_nano.a(lib_a-atoi.o)
                              ./App/LoRaWAN/src/main.o (atoi)
/opt/st/stm32cubeide_1.9.0/plugins/com.st.stm32cube.ide.mcu.externaltools.gnu-tools-for-stm32.10.3-2021.10.linux64_1.0.0.202111181127/tools/bin/../lib/gcc/arm-none-eabi/10.3.1/../../../../arm-none-eabi/lib/thumb/v6-m/nofp/libc_nano.a(lib_a-exit.o)
                              /opt/st/stm32cubeide_1.9.0/plugins/com.st.stm32cube.ide.mcu.externaltools.gnu-tools-for-stm32.10.3-2021.10.linux64_1.0.0.202111181127/tools/bin/../lib/gcc/arm-none-eabi/10.3.1/../../../../arm-none-eabi/lib/thumb/v6-m/nofp/crt0.o (exit)
/opt/st/stm32cubeide_1.9.0/plugins/com.st.stm32cube.ide.mcu.externaltools.gnu-tools-for-stm32.10.3-2021.10.linux64_1.0.0.202111181127/tools/bin/../lib/gcc/arm-none-eabi/10.3.1/../../../../arm-none-eabi/lib/thumb/v6-m/nofp/libc_nano.a(lib_a-impure.o)
                              /opt/st/stm32cubeide_1.9.0/plugins/com.st.stm32cube.ide.mcu.externaltools.gnu-tools-for-stm32.10.3-2021.10.linux64_1.0.0.202111181127/tools/bin/../lib/gcc/arm-none-eabi/10.3.1/../../../../arm-none-eabi/lib/thumb/v6-m/nofp/libc_nano.a(lib_a-exit.o) (_global_impure_ptr)
/opt/st/stm32cubeide_1.9.0/plugins/com.st.stm32cube.ide.mcu.externaltools.gnu-tools-for-stm32.10.3-2021.10.linux64_1.0.0.202111181127/tools/bin/../lib/gcc/arm-none-eabi/10.3.1/../../../../arm-none-eabi/lib/thumb/v6-m/nofp/libc_nano.a(lib_a-init.o)
                              /opt/st/stm32cubeide_1.9.0/plugins/com.st.stm32cube.ide.mcu.externaltools.gnu-tools-for-stm32.10.3-2021.10.linux64_1.0.0.202111181127/tools/bin/../lib/gcc/arm-none-eabi/10.3.1/../../../../arm-none-eabi/lib/thumb/v6-m/nofp/crt0.o (__libc_init_array)
/opt/st/stm32cubeide_1.9.0/plugins/com.st.stm32cube.ide.mcu.externaltools.gnu-tools-for-stm32.10.3-2021.10.linux64_1.0.0.202111181127/tools/bin/../lib/gcc/arm-none-eabi/10.3.1/../../../../arm-none-eabi/lib/thumb/v6-m/nofp/libc_nano.a(lib_a-memset.o)
                              /opt/st/stm32cubeide_1.9.0/plugins/com.st.stm32cube.ide.mcu.externaltools.gnu-tools-for-stm32.10.3-2021.10.linux64_1.0.0.202111181127/tools/bin/../lib/gcc/arm-none-eabi/10.3.1/../../../../arm-none-eabi/lib/thumb/v6-m/nofp/crt0.o (memset)
/opt/st/stm32cubeide_1.9.0/plugins/com.st.stm32cube.ide.mcu.externaltools.gnu-tools-for-stm32.10.3-2021.10.linux64_1.0.0.202111181127/tools/bin/../lib/gcc/arm-none-eabi/10.3.1/../../../../arm-none-eabi/lib/thumb/v6-m/nofp/libc_nano.a(lib_a-mktime.o)
                              ./App/LoRaWAN/src/main.o (mktime)
/opt/st/stm32cubeide_1.9.0/plugins/com.st.stm32cube.ide.mcu.externaltools.gnu-tools-for-stm32.10.3-2021.10.linux64_1.0.0.202111181127/tools/bin/../lib/gcc/arm-none-eabi/10.3.1/../../../../arm-none-eabi/lib/thumb/v6-m/nofp/libc_nano.a(lib_a-nano-vfprintf_float.o)
                              (_printf_float)
/opt/st/stm32cubeide_1.9.0/plugins/com.st.stm32cube.ide.mcu.externaltools.gnu-tools-for-stm32.10.3-2021.10.linux64_1.0.0.202111181127/tools/bin/../lib/gcc/arm-none-eabi/10.3.1/../../../../arm-none-eabi/lib/thumb/v6-m/nofp/libc_nano.a(lib_a-nano-vfprintf_i.o)
                              /opt/st/stm32cubeide_1.9.0/plugins/com.st.stm32cube.ide.mcu.externaltools.gnu-tools-for-stm32.10.3-2021.10.linux64_1.0.0.202111181127/tools/bin/../lib/gcc/arm-none-eabi/10.3.1/../../../../arm-none-eabi/lib/thumb/v6-m/nofp/libc_nano.a(lib_a-nano-vfprintf_float.o) (_printf_common)
/opt/st/stm32cubeide_1.9.0/plugins/com.st.stm32cube.ide.mcu.externaltools.gnu-tools-for-stm32.10.3-2021.10.linux64_1.0.0.202111181127/tools/bin/../lib/gcc/arm-none-eabi/10.3.1/../../../../arm-none-eabi/lib/thumb/v6-m/nofp/libc_nano.a(lib_a-nano-vfscanf_float.o)
                              (_scanf_float)
/opt/st/stm32cubeide_1.9.0/plugins/com.st.stm32cube.ide.mcu.externaltools.gnu-tools-for-stm32.10.3-2021.10.linux64_1.0.0.202111181127/tools/bin/../lib/gcc/arm-none-eabi/10.3.1/../../../../arm-none-eabi/lib/thumb/v6-m/nofp/libc_nano.a(lib_a-sf_nan.o)
                              /opt/st/stm32cubeide_1.9.0/plugins/com.st.stm32cube.ide.mcu.externaltools.gnu-tools-for-stm32.10.3-2021.10.linux64_1.0.0.202111181127/tools/bin/../lib/gcc/arm-none-eabi/10.3.1/../../../../arm-none-eabi/lib/thumb/v6-m/nofp/libc_nano.a(lib_a-nano-vfscanf_float.o) (nanf)
/opt/st/stm32cubeide_1.9.0/plugins/com.st.stm32cube.ide.mcu.externaltools.gnu-tools-for-stm32.10.3-2021.10.linux64_1.0.0.202111181127/tools/bin/../lib/gcc/arm-none-eabi/10.3.1/../../../../arm-none-eabi/lib/thumb/v6-m/nofp/libc_nano.a(lib_a-sprintf.o)
                              /opt/st/stm32cubeide_1.9.0/plugins/com.st.stm32cube.ide.mcu.externaltools.gnu-tools-for-stm32.10.3-2021.10.linux64_1.0.0.202111181127/tools/bin/../lib/gcc/arm-none-eabi/10.3.1/../../../../arm-none-eabi/lib/thumb/v6-m/nofp/libc_nano.a(lib_a-nano-vfscanf_float.o) (sprintf)
/opt/st/stm32cubeide_1.9.0/plugins/com.st.stm32cube.ide.mcu.externaltools.gnu-tools-for-stm32.10.3-2021.10.linux64_1.0.0.202111181127/tools/bin/../lib/gcc/arm-none-eabi/10.3.1/../../../../arm-none-eabi/lib/thumb/v6-m/nofp/libc_nano.a(lib_a-strlen.o)
                              /opt/st/stm32cubeide_1.9.0/plugins/com.st.stm32cube.ide.mcu.externaltools.gnu-tools-for-stm32.10.3-2021.10.linux64_1.0.0.202111181127/tools/bin/../lib/gcc/arm-none-eabi/10.3.1/../../../../arm-none-eabi/lib/thumb/v6-m/nofp/libc_nano.a(lib_a-nano-vfprintf_float.o) (strlen)
/opt/st/stm32cubeide_1.9.0/plugins/com.st.stm32cube.ide.mcu.externaltools.gnu-tools-for-stm32.10.3-2021.10.linux64_1.0.0.202111181127/tools/bin/../lib/gcc/arm-none-eabi/10.3.1/../../../../arm-none-eabi/lib/thumb/v6-m/nofp/libc_nano.a(lib_a-strrchr.o)
                              ./Drivers/Middlewares/LoRaWAN/Utilities/trace.o (strrchr)
/opt/st/stm32cubeide_1.9.0/plugins/com.st.stm32cube.ide.mcu.externaltools.gnu-tools-for-stm32.10.3-2021.10.linux64_1.0.0.202111181127/tools/bin/../lib/gcc/arm-none-eabi/10.3.1/../../../../arm-none-eabi/lib/thumb/v6-m/nofp/libc_nano.a(lib_a-strtod.o)
                              /opt/st/stm32cubeide_1.9.0/plugins/com.st.stm32cube.ide.mcu.externaltools.gnu-tools-for-stm32.10.3-2021.10.linux64_1.0.0.202111181127/tools/bin/../lib/gcc/arm-none-eabi/10.3.1/../../../../arm-none-eabi/lib/thumb/v6-m/nofp/libc_nano.a(lib_a-nano-vfscanf_float.o) (_strtod_r)
/opt/st/stm32cubeide_1.9.0/plugins/com.st.stm32cube.ide.mcu.externaltools.gnu-tools-for-stm32.10.3-2021.10.linux64_1.0.0.202111181127/tools/bin/../lib/gcc/arm-none-eabi/10.3.1/../../../../arm-none-eabi/lib/thumb/v6-m/nofp/libc_nano.a(lib_a-strtol.o)
                              /opt/st/stm32cubeide_1.9.0/plugins/com.st.stm32cube.ide.mcu.externaltools.gnu-tools-for-stm32.10.3-2021.10.linux64_1.0.0.202111181127/tools/bin/../lib/gcc/arm-none-eabi/10.3.1/../../../../arm-none-eabi/lib/thumb/v6-m/nofp/libc_nano.a(lib_a-atoi.o) (_strtol_r)
/opt/st/stm32cubeide_1.9.0/plugins/com.st.stm32cube.ide.mcu.externaltools.gnu-tools-for-stm32.10.3-2021.10.linux64_1.0.0.202111181127/tools/bin/../lib/gcc/arm-none-eabi/10.3.1/../../../../arm-none-eabi/lib/thumb/v6-m/nofp/libc_nano.a(lib_a-tzcalc_limits.o)
                              /opt/st/stm32cubeide_1.9.0/plugins/com.st.stm32cube.ide.mcu.externaltools.gnu-tools-for-stm32.10.3-2021.10.linux64_1.0.0.202111181127/tools/bin/../lib/gcc/arm-none-eabi/10.3.1/../../../../arm-none-eabi/lib/thumb/v6-m/nofp/libc_nano.a(lib_a-mktime.o) (__tzcalc_limits)
/opt/st/stm32cubeide_1.9.0/plugins/com.st.stm32cube.ide.mcu.externaltools.gnu-tools-for-stm32.10.3-2021.10.linux64_1.0.0.202111181127/tools/bin/../lib/gcc/arm-none-eabi/10.3.1/../../../../arm-none-eabi/lib/thumb/v6-m/nofp/libc_nano.a(lib_a-tzlock.o)
                              /opt/st/stm32cubeide_1.9.0/plugins/com.st.stm32cube.ide.mcu.externaltools.gnu-tools-for-stm32.10.3-2021.10.linux64_1.0.0.202111181127/tools/bin/../lib/gcc/arm-none-eabi/10.3.1/../../../../arm-none-eabi/lib/thumb/v6-m/nofp/libc_nano.a(lib_a-mktime.o) (__tz_lock)
/opt/st/stm32cubeide_1.9.0/plugins/com.st.stm32cube.ide.mcu.externaltools.gnu-tools-for-stm32.10.3-2021.10.linux64_1.0.0.202111181127/tools/bin/../lib/gcc/arm-none-eabi/10.3.1/../../../../arm-none-eabi/lib/thumb/v6-m/nofp/libc_nano.a(lib_a-tzset.o)
                              /opt/st/stm32cubeide_1.9.0/plugins/com.st.stm32cube.ide.mcu.externaltools.gnu-tools-for-stm32.10.3-2021.10.linux64_1.0.0.202111181127/tools/bin/../lib/gcc/arm-none-eabi/10.3.1/../../../../arm-none-eabi/lib/thumb/v6-m/nofp/libc_nano.a(lib_a-mktime.o) (_tzset_unlocked)
/opt/st/stm32cubeide_1.9.0/plugins/com.st.stm32cube.ide.mcu.externaltools.gnu-tools-for-stm32.10.3-2021.10.linux64_1.0.0.202111181127/tools/bin/../lib/gcc/arm-none-eabi/10.3.1/../../../../arm-none-eabi/lib/thumb/v6-m/nofp/libc_nano.a(lib_a-tzset_r.o)
                              /opt/st/stm32cubeide_1.9.0/plugins/com.st.stm32cube.ide.mcu.externaltools.gnu-tools-for-stm32.10.3-2021.10.linux64_1.0.0.202111181127/tools/bin/../lib/gcc/arm-none-eabi/10.3.1/../../../../arm-none-eabi/lib/thumb/v6-m/nofp/libc_nano.a(lib_a-tzset.o) (_tzset_unlocked_r)
/opt/st/stm32cubeide_1.9.0/plugins/com.st.stm32cube.ide.mcu.externaltools.gnu-tools-for-stm32.10.3-2021.10.linux64_1.0.0.202111181127/tools/bin/../lib/gcc/arm-none-eabi/10.3.1/../../../../arm-none-eabi/lib/thumb/v6-m/nofp/libc_nano.a(lib_a-tzvars.o)
                              /opt/st/stm32cubeide_1.9.0/plugins/com.st.stm32cube.ide.mcu.externaltools.gnu-tools-for-stm32.10.3-2021.10.linux64_1.0.0.202111181127/tools/bin/../lib/gcc/arm-none-eabi/10.3.1/../../../../arm-none-eabi/lib/thumb/v6-m/nofp/libc_nano.a(lib_a-tzset_r.o) (_timezone)
/opt/st/stm32cubeide_1.9.0/plugins/com.st.stm32cube.ide.mcu.externaltools.gnu-tools-for-stm32.10.3-2021.10.linux64_1.0.0.202111181127/tools/bin/../lib/gcc/arm-none-eabi/10.3.1/../../../../arm-none-eabi/lib/thumb/v6-m/nofp/libc_nano.a(lib_a-vsnprintf.o)
                              ./Drivers/Middlewares/LoRaWAN/Utilities/trace.o (vsnprintf)
/opt/st/stm32cubeide_1.9.0/plugins/com.st.stm32cube.ide.mcu.externaltools.gnu-tools-for-stm32.10.3-2021.10.linux64_1.0.0.202111181127/tools/bin/../lib/gcc/arm-none-eabi/10.3.1/../../../../arm-none-eabi/lib/thumb/v6-m/nofp/libc_nano.a(lib_a-ctype_.o)
                              /opt/st/stm32cubeide_1.9.0/plugins/com.st.stm32cube.ide.mcu.externaltools.gnu-tools-for-stm32.10.3-2021.10.linux64_1.0.0.202111181127/tools/bin/../lib/gcc/arm-none-eabi/10.3.1/../../../../arm-none-eabi/lib/thumb/v6-m/nofp/libc_nano.a(lib_a-strtol.o) (_ctype_)
/opt/st/stm32cubeide_1.9.0/plugins/com.st.stm32cube.ide.mcu.externaltools.gnu-tools-for-stm32.10.3-2021.10.linux64_1.0.0.202111181127/tools/bin/../lib/gcc/arm-none-eabi/10.3.1/../../../../arm-none-eabi/lib/thumb/v6-m/nofp/libc_nano.a(lib_a-div.o)
                              /opt/st/stm32cubeide_1.9.0/plugins/com.st.stm32cube.ide.mcu.externaltools.gnu-tools-for-stm32.10.3-2021.10.linux64_1.0.0.202111181127/tools/bin/../lib/gcc/arm-none-eabi/10.3.1/../../../../arm-none-eabi/lib/thumb/v6-m/nofp/libc_nano.a(lib_a-mktime.o) (div)
/opt/st/stm32cubeide_1.9.0/plugins/com.st.stm32cube.ide.mcu.externaltools.gnu-tools-for-stm32.10.3-2021.10.linux64_1.0.0.202111181127/tools/bin/../lib/gcc/arm-none-eabi/10.3.1/../../../../arm-none-eabi/lib/thumb/v6-m/nofp/libc_nano.a(lib_a-dtoa.o)
                              /opt/st/stm32cubeide_1.9.0/plugins/com.st.stm32cube.ide.mcu.externaltools.gnu-tools-for-stm32.10.3-2021.10.linux64_1.0.0.202111181127/tools/bin/../lib/gcc/arm-none-eabi/10.3.1/../../../../arm-none-eabi/lib/thumb/v6-m/nofp/libc_nano.a(lib_a-nano-vfprintf_float.o) (_dtoa_r)
/opt/st/stm32cubeide_1.9.0/plugins/com.st.stm32cube.ide.mcu.externaltools.gnu-tools-for-stm32.10.3-2021.10.linux64_1.0.0.202111181127/tools/bin/../lib/gcc/arm-none-eabi/10.3.1/../../../../arm-none-eabi/lib/thumb/v6-m/nofp/libc_nano.a(lib_a-errno.o)
                              /opt/st/stm32cubeide_1.9.0/plugins/com.st.stm32cube.ide.mcu.externaltools.gnu-tools-for-stm32.10.3-2021.10.linux64_1.0.0.202111181127/tools/bin/../lib/gcc/arm-none-eabi/10.3.1/../../../../arm-none-eabi/lib/thumb/v6-m/nofp/libc_nano.a(lib_a-strtol.o) (__errno)
/opt/st/stm32cubeide_1.9.0/plugins/com.st.stm32cube.ide.mcu.externaltools.gnu-tools-for-stm32.10.3-2021.10.linux64_1.0.0.202111181127/tools/bin/../lib/gcc/arm-none-eabi/10.3.1/../../../../arm-none-eabi/lib/thumb/v6-m/nofp/libc_nano.a(lib_a-gdtoa-gethex.o)
                              /opt/st/stm32cubeide_1.9.0/plugins/com.st.stm32cube.ide.mcu.externaltools.gnu-tools-for-stm32.10.3-2021.10.linux64_1.0.0.202111181127/tools/bin/../lib/gcc/arm-none-eabi/10.3.1/../../../../arm-none-eabi/lib/thumb/v6-m/nofp/libc_nano.a(lib_a-strtod.o) (__gethex)
/opt/st/stm32cubeide_1.9.0/plugins/com.st.stm32cube.ide.mcu.externaltools.gnu-tools-for-stm32.10.3-2021.10.linux64_1.0.0.202111181127/tools/bin/../lib/gcc/arm-none-eabi/10.3.1/../../../../arm-none-eabi/lib/thumb/v6-m/nofp/libc_nano.a(lib_a-gdtoa-hexnan.o)
                              /opt/st/stm32cubeide_1.9.0/plugins/com.st.stm32cube.ide.mcu.externaltools.gnu-tools-for-stm32.10.3-2021.10.linux64_1.0.0.202111181127/tools/bin/../lib/gcc/arm-none-eabi/10.3.1/../../../../arm-none-eabi/lib/thumb/v6-m/nofp/libc_nano.a(lib_a-strtod.o) (__match)
/opt/st/stm32cubeide_1.9.0/plugins/com.st.stm32cube.ide.mcu.externaltools.gnu-tools-for-stm32.10.3-2021.10.linux64_1.0.0.202111181127/tools/bin/../lib/gcc/arm-none-eabi/10.3.1/../../../../arm-none-eabi/lib/thumb/v6-m/nofp/libc_nano.a(lib_a-getenv_r.o)
                              /opt/st/stm32cubeide_1.9.0/plugins/com.st.stm32cube.ide.mcu.externaltools.gnu-tools-for-stm32.10.3-2021.10.linux64_1.0.0.202111181127/tools/bin/../lib/gcc/arm-none-eabi/10.3.1/../../../../arm-none-eabi/lib/thumb/v6-m/nofp/libc_nano.a(lib_a-tzset_r.o) (_getenv_r)
/opt/st/stm32cubeide_1.9.0/plugins/com.st.stm32cube.ide.mcu.externaltools.gnu-tools-for-stm32.10.3-2021.10.linux64_1.0.0.202111181127/tools/bin/../lib/gcc/arm-none-eabi/10.3.1/../../../../arm-none-eabi/lib/thumb/v6-m/nofp/libc_nano.a(lib_a-gettzinfo.o)
                              /opt/st/stm32cubeide_1.9.0/plugins/com.st.stm32cube.ide.mcu.externaltools.gnu-tools-for-stm32.10.3-2021.10.linux64_1.0.0.202111181127/tools/bin/../lib/gcc/arm-none-eabi/10.3.1/../../../../arm-none-eabi/lib/thumb/v6-m/nofp/libc_nano.a(lib_a-mktime.o) (__gettzinfo)
/opt/st/stm32cubeide_1.9.0/plugins/com.st.stm32cube.ide.mcu.externaltools.gnu-tools-for-stm32.10.3-2021.10.linux64_1.0.0.202111181127/tools/bin/../lib/gcc/arm-none-eabi/10.3.1/../../../../arm-none-eabi/lib/thumb/v6-m/nofp/libc_nano.a(lib_a-lnumeric.o)
                              /opt/st/stm32cubeide_1.9.0/plugins/com.st.stm32cube.ide.mcu.externaltools.gnu-tools-for-stm32.10.3-2021.10.linux64_1.0.0.202111181127/tools/bin/../lib/gcc/arm-none-eabi/10.3.1/../../../../arm-none-eabi/lib/thumb/v6-m/nofp/libc_nano.a(lib_a-strtod.o) (_C_numeric_locale)
/opt/st/stm32cubeide_1.9.0/plugins/com.st.stm32cube.ide.mcu.externaltools.gnu-tools-for-stm32.10.3-2021.10.linux64_1.0.0.202111181127/tools/bin/../lib/gcc/arm-none-eabi/10.3.1/../../../../arm-none-eabi/lib/thumb/v6-m/nofp/libc_nano.a(lib_a-locale.o)
                              /opt/st/stm32cubeide_1.9.0/plugins/com.st.stm32cube.ide.mcu.externaltools.gnu-tools-for-stm32.10.3-2021.10.linux64_1.0.0.202111181127/tools/bin/../lib/gcc/arm-none-eabi/10.3.1/../../../../arm-none-eabi/lib/thumb/v6-m/nofp/libc_nano.a(lib_a-strtod.o) (__global_locale)
/opt/st/stm32cubeide_1.9.0/plugins/com.st.stm32cube.ide.mcu.externaltools.gnu-tools-for-stm32.10.3-2021.10.linux64_1.0.0.202111181127/tools/bin/../lib/gcc/arm-none-eabi/10.3.1/../../../../arm-none-eabi/lib/thumb/v6-m/nofp/libc_nano.a(lib_a-localeconv.o)
                              /opt/st/stm32cubeide_1.9.0/plugins/com.st.stm32cube.ide.mcu.externaltools.gnu-tools-for-stm32.10.3-2021.10.linux64_1.0.0.202111181127/tools/bin/../lib/gcc/arm-none-eabi/10.3.1/../../../../arm-none-eabi/lib/thumb/v6-m/nofp/libc_nano.a(lib_a-nano-vfprintf_float.o) (_localeconv_r)
/opt/st/stm32cubeide_1.9.0/plugins/com.st.stm32cube.ide.mcu.externaltools.gnu-tools-for-stm32.10.3-2021.10.linux64_1.0.0.202111181127/tools/bin/../lib/gcc/arm-none-eabi/10.3.1/../../../../arm-none-eabi/lib/thumb/v6-m/nofp/libc_nano.a(lib_a-lock.o)
                              /opt/st/stm32cubeide_1.9.0/plugins/com.st.stm32cube.ide.mcu.externaltools.gnu-tools-for-stm32.10.3-2021.10.linux64_1.0.0.202111181127/tools/bin/../lib/gcc/arm-none-eabi/10.3.1/../../../../arm-none-eabi/lib/thumb/v6-m/nofp/libc_nano.a(lib_a-tzlock.o) (__retarget_lock_acquire)
/opt/st/stm32cubeide_1.9.0/plugins/com.st.stm32cube.ide.mcu.externaltools.gnu-tools-for-stm32.10.3-2021.10.linux64_1.0.0.202111181127/tools/bin/../lib/gcc/arm-none-eabi/10.3.1/../../../../arm-none-eabi/lib/thumb/v6-m/nofp/libc_nano.a(lib_a-malloc.o)
                              /opt/st/stm32cubeide_1.9.0/plugins/com.st.stm32cube.ide.mcu.externaltools.gnu-tools-for-stm32.10.3-2021.10.linux64_1.0.0.202111181127/tools/bin/../lib/gcc/arm-none-eabi/10.3.1/../../../../arm-none-eabi/lib/thumb/v6-m/nofp/libc_nano.a(lib_a-dtoa.o) (malloc)
/opt/st/stm32cubeide_1.9.0/plugins/com.st.stm32cube.ide.mcu.externaltools.gnu-tools-for-stm32.10.3-2021.10.linux64_1.0.0.202111181127/tools/bin/../lib/gcc/arm-none-eabi/10.3.1/../../../../arm-none-eabi/lib/thumb/v6-m/nofp/libc_nano.a(lib_a-mbtowc_r.o)
                              /opt/st/stm32cubeide_1.9.0/plugins/com.st.stm32cube.ide.mcu.externaltools.gnu-tools-for-stm32.10.3-2021.10.linux64_1.0.0.202111181127/tools/bin/../lib/gcc/arm-none-eabi/10.3.1/../../../../arm-none-eabi/lib/thumb/v6-m/nofp/libc_nano.a(lib_a-locale.o) (__ascii_mbtowc)
/opt/st/stm32cubeide_1.9.0/plugins/com.st.stm32cube.ide.mcu.externaltools.gnu-tools-for-stm32.10.3-2021.10.linux64_1.0.0.202111181127/tools/bin/../lib/gcc/arm-none-eabi/10.3.1/../../../../arm-none-eabi/lib/thumb/v6-m/nofp/libc_nano.a(lib_a-memchr-stub.o)
                              /opt/st/stm32cubeide_1.9.0/plugins/com.st.stm32cube.ide.mcu.externaltools.gnu-tools-for-stm32.10.3-2021.10.linux64_1.0.0.202111181127/tools/bin/../lib/gcc/arm-none-eabi/10.3.1/../../../../arm-none-eabi/lib/thumb/v6-m/nofp/libc_nano.a(lib_a-nano-vfprintf_i.o) (memchr)
/opt/st/stm32cubeide_1.9.0/plugins/com.st.stm32cube.ide.mcu.externaltools.gnu-tools-for-stm32.10.3-2021.10.linux64_1.0.0.202111181127/tools/bin/../lib/gcc/arm-none-eabi/10.3.1/../../../../arm-none-eabi/lib/thumb/v6-m/nofp/libc_nano.a(lib_a-memcpy-stub.o)
                              /opt/st/stm32cubeide_1.9.0/plugins/com.st.stm32cube.ide.mcu.externaltools.gnu-tools-for-stm32.10.3-2021.10.linux64_1.0.0.202111181127/tools/bin/../lib/gcc/arm-none-eabi/10.3.1/../../../../arm-none-eabi/lib/thumb/v6-m/nofp/libc_nano.a(lib_a-strtod.o) (memcpy)
/opt/st/stm32cubeide_1.9.0/plugins/com.st.stm32cube.ide.mcu.externaltools.gnu-tools-for-stm32.10.3-2021.10.linux64_1.0.0.202111181127/tools/bin/../lib/gcc/arm-none-eabi/10.3.1/../../../../arm-none-eabi/lib/thumb/v6-m/nofp/libc_nano.a(lib_a-month_lengths.o)
                              /opt/st/stm32cubeide_1.9.0/plugins/com.st.stm32cube.ide.mcu.externaltools.gnu-tools-for-stm32.10.3-2021.10.linux64_1.0.0.202111181127/tools/bin/../lib/gcc/arm-none-eabi/10.3.1/../../../../arm-none-eabi/lib/thumb/v6-m/nofp/libc_nano.a(lib_a-tzcalc_limits.o) (__month_lengths)
/opt/st/stm32cubeide_1.9.0/plugins/com.st.stm32cube.ide.mcu.externaltools.gnu-tools-for-stm32.10.3-2021.10.linux64_1.0.0.202111181127/tools/bin/../lib/gcc/arm-none-eabi/10.3.1/../../../../arm-none-eabi/lib/thumb/v6-m/nofp/libc_nano.a(lib_a-mprec.o)
                              /opt/st/stm32cubeide_1.9.0/plugins/com.st.stm32cube.ide.mcu.externaltools.gnu-tools-for-stm32.10.3-2021.10.linux64_1.0.0.202111181127/tools/bin/../lib/gcc/arm-none-eabi/10.3.1/../../../../arm-none-eabi/lib/thumb/v6-m/nofp/libc_nano.a(lib_a-strtod.o) (_Balloc)
/opt/st/stm32cubeide_1.9.0/plugins/com.st.stm32cube.ide.mcu.externaltools.gnu-tools-for-stm32.10.3-2021.10.linux64_1.0.0.202111181127/tools/bin/../lib/gcc/arm-none-eabi/10.3.1/../../../../arm-none-eabi/lib/thumb/v6-m/nofp/libc_nano.a(lib_a-nano-callocr.o)
                              /opt/st/stm32cubeide_1.9.0/plugins/com.st.stm32cube.ide.mcu.externaltools.gnu-tools-for-stm32.10.3-2021.10.linux64_1.0.0.202111181127/tools/bin/../lib/gcc/arm-none-eabi/10.3.1/../../../../arm-none-eabi/lib/thumb/v6-m/nofp/libc_nano.a(lib_a-mprec.o) (_calloc_r)
/opt/st/stm32cubeide_1.9.0/plugins/com.st.stm32cube.ide.mcu.externaltools.gnu-tools-for-stm32.10.3-2021.10.linux64_1.0.0.202111181127/tools/bin/../lib/gcc/arm-none-eabi/10.3.1/../../../../arm-none-eabi/lib/thumb/v6-m/nofp/libc_nano.a(lib_a-nano-freer.o)
                              /opt/st/stm32cubeide_1.9.0/plugins/com.st.stm32cube.ide.mcu.externaltools.gnu-tools-for-stm32.10.3-2021.10.linux64_1.0.0.202111181127/tools/bin/../lib/gcc/arm-none-eabi/10.3.1/../../../../arm-none-eabi/lib/thumb/v6-m/nofp/libc_nano.a(lib_a-malloc.o) (_free_r)
/opt/st/stm32cubeide_1.9.0/plugins/com.st.stm32cube.ide.mcu.externaltools.gnu-tools-for-stm32.10.3-2021.10.linux64_1.0.0.202111181127/tools/bin/../lib/gcc/arm-none-eabi/10.3.1/../../../../arm-none-eabi/lib/thumb/v6-m/nofp/libc_nano.a(lib_a-nano-mallocr.o)
                              /opt/st/stm32cubeide_1.9.0/plugins/com.st.stm32cube.ide.mcu.externaltools.gnu-tools-for-stm32.10.3-2021.10.linux64_1.0.0.202111181127/tools/bin/../lib/gcc/arm-none-eabi/10.3.1/../../../../arm-none-eabi/lib/thumb/v6-m/nofp/libc_nano.a(lib_a-tzset_r.o) (_malloc_r)
/opt/st/stm32cubeide_1.9.0/plugins/com.st.stm32cube.ide.mcu.externaltools.gnu-tools-for-stm32.10.3-2021.10.linux64_1.0.0.202111181127/tools/bin/../lib/gcc/arm-none-eabi/10.3.1/../../../../arm-none-eabi/lib/thumb/v6-m/nofp/libc_nano.a(lib_a-nano-svfprintf.o)
                              /opt/st/stm32cubeide_1.9.0/plugins/com.st.stm32cube.ide.mcu.externaltools.gnu-tools-for-stm32.10.3-2021.10.linux64_1.0.0.202111181127/tools/bin/../lib/gcc/arm-none-eabi/10.3.1/../../../../arm-none-eabi/lib/thumb/v6-m/nofp/libc_nano.a(lib_a-sprintf.o) (_svfprintf_r)
/opt/st/stm32cubeide_1.9.0/plugins/com.st.stm32cube.ide.mcu.externaltools.gnu-tools-for-stm32.10.3-2021.10.linux64_1.0.0.202111181127/tools/bin/../lib/gcc/arm-none-eabi/10.3.1/../../../../arm-none-eabi/lib/thumb/v6-m/nofp/libc_nano.a(lib_a-s_nan.o)
                              /opt/st/stm32cubeide_1.9.0/plugins/com.st.stm32cube.ide.mcu.externaltools.gnu-tools-for-stm32.10.3-2021.10.linux64_1.0.0.202111181127/tools/bin/../lib/gcc/arm-none-eabi/10.3.1/../../../../arm-none-eabi/lib/thumb/v6-m/nofp/libc_nano.a(lib_a-strtod.o) (nan)
/opt/st/stm32cubeide_1.9.0/plugins/com.st.stm32cube.ide.mcu.externaltools.gnu-tools-for-stm32.10.3-2021.10.linux64_1.0.0.202111181127/tools/bin/../lib/gcc/arm-none-eabi/10.3.1/../../../../arm-none-eabi/lib/thumb/v6-m/nofp/libc_nano.a(lib_a-sbrkr.o)
                              /opt/st/stm32cubeide_1.9.0/plugins/com.st.stm32cube.ide.mcu.externaltools.gnu-tools-for-stm32.10.3-2021.10.linux64_1.0.0.202111181127/tools/bin/../lib/gcc/arm-none-eabi/10.3.1/../../../../arm-none-eabi/lib/thumb/v6-m/nofp/libc_nano.a(lib_a-nano-mallocr.o) (_sbrk_r)
/opt/st/stm32cubeide_1.9.0/plugins/com.st.stm32cube.ide.mcu.externaltools.gnu-tools-for-stm32.10.3-2021.10.linux64_1.0.0.202111181127/tools/bin/../lib/gcc/arm-none-eabi/10.3.1/../../../../arm-none-eabi/lib/thumb/v6-m/nofp/libc_nano.a(lib_a-sscanf.o)
                              /opt/st/stm32cubeide_1.9.0/plugins/com.st.stm32cube.ide.mcu.externaltools.gnu-tools-for-stm32.10.3-2021.10.linux64_1.0.0.202111181127/tools/bin/../lib/gcc/arm-none-eabi/10.3.1/../../../../arm-none-eabi/lib/thumb/v6-m/nofp/libc_nano.a(lib_a-tzset_r.o) (siscanf)
/opt/st/stm32cubeide_1.9.0/plugins/com.st.stm32cube.ide.mcu.externaltools.gnu-tools-for-stm32.10.3-2021.10.linux64_1.0.0.202111181127/tools/bin/../lib/gcc/arm-none-eabi/10.3.1/../../../../arm-none-eabi/lib/thumb/v6-m/nofp/libc_nano.a(lib_a-stdio.o)
                              /opt/st/stm32cubeide_1.9.0/plugins/com.st.stm32cube.ide.mcu.externaltools.gnu-tools-for-stm32.10.3-2021.10.linux64_1.0.0.202111181127/tools/bin/../lib/gcc/arm-none-eabi/10.3.1/../../../../arm-none-eabi/lib/thumb/v6-m/nofp/libc_nano.a(lib_a-sscanf.o) (__seofread)
/opt/st/stm32cubeide_1.9.0/plugins/com.st.stm32cube.ide.mcu.externaltools.gnu-tools-for-stm32.10.3-2021.10.linux64_1.0.0.202111181127/tools/bin/../lib/gcc/arm-none-eabi/10.3.1/../../../../arm-none-eabi/lib/thumb/v6-m/nofp/libc_nano.a(lib_a-strchr.o)
                              /opt/st/stm32cubeide_1.9.0/plugins/com.st.stm32cube.ide.mcu.externaltools.gnu-tools-for-stm32.10.3-2021.10.linux64_1.0.0.202111181127/tools/bin/../lib/gcc/arm-none-eabi/10.3.1/../../../../arm-none-eabi/lib/thumb/v6-m/nofp/libc_nano.a(lib_a-strrchr.o) (strchr)
/opt/st/stm32cubeide_1.9.0/plugins/com.st.stm32cube.ide.mcu.externaltools.gnu-tools-for-stm32.10.3-2021.10.linux64_1.0.0.202111181127/tools/bin/../lib/gcc/arm-none-eabi/10.3.1/../../../../arm-none-eabi/lib/thumb/v6-m/nofp/libc_nano.a(lib_a-strcmp.o)
                              /opt/st/stm32cubeide_1.9.0/plugins/com.st.stm32cube.ide.mcu.externaltools.gnu-tools-for-stm32.10.3-2021.10.linux64_1.0.0.202111181127/tools/bin/../lib/gcc/arm-none-eabi/10.3.1/../../../../arm-none-eabi/lib/thumb/v6-m/nofp/libc_nano.a(lib_a-tzset_r.o) (strcmp)
/opt/st/stm32cubeide_1.9.0/plugins/com.st.stm32cube.ide.mcu.externaltools.gnu-tools-for-stm32.10.3-2021.10.linux64_1.0.0.202111181127/tools/bin/../lib/gcc/arm-none-eabi/10.3.1/../../../../arm-none-eabi/lib/thumb/v6-m/nofp/libc_nano.a(lib_a-strcpy.o)
                              /opt/st/stm32cubeide_1.9.0/plugins/com.st.stm32cube.ide.mcu.externaltools.gnu-tools-for-stm32.10.3-2021.10.linux64_1.0.0.202111181127/tools/bin/../lib/gcc/arm-none-eabi/10.3.1/../../../../arm-none-eabi/lib/thumb/v6-m/nofp/libc_nano.a(lib_a-tzset_r.o) (strcpy)
/opt/st/stm32cubeide_1.9.0/plugins/com.st.stm32cube.ide.mcu.externaltools.gnu-tools-for-stm32.10.3-2021.10.linux64_1.0.0.202111181127/tools/bin/../lib/gcc/arm-none-eabi/10.3.1/../../../../arm-none-eabi/lib/thumb/v6-m/nofp/libc_nano.a(lib_a-strncmp.o)
                              /opt/st/stm32cubeide_1.9.0/plugins/com.st.stm32cube.ide.mcu.externaltools.gnu-tools-for-stm32.10.3-2021.10.linux64_1.0.0.202111181127/tools/bin/../lib/gcc/arm-none-eabi/10.3.1/../../../../arm-none-eabi/lib/thumb/v6-m/nofp/libc_nano.a(lib_a-strtod.o) (strncmp)
/opt/st/stm32cubeide_1.9.0/plugins/com.st.stm32cube.ide.mcu.externaltools.gnu-tools-for-stm32.10.3-2021.10.linux64_1.0.0.202111181127/tools/bin/../lib/gcc/arm-none-eabi/10.3.1/../../../../arm-none-eabi/lib/thumb/v6-m/nofp/libc_nano.a(lib_a-strtoul.o)
                              /opt/st/stm32cubeide_1.9.0/plugins/com.st.stm32cube.ide.mcu.externaltools.gnu-tools-for-stm32.10.3-2021.10.linux64_1.0.0.202111181127/tools/bin/../lib/gcc/arm-none-eabi/10.3.1/../../../../arm-none-eabi/lib/thumb/v6-m/nofp/libc_nano.a(lib_a-tzset_r.o) (strtoul)
/opt/st/stm32cubeide_1.9.0/plugins/com.st.stm32cube.ide.mcu.externaltools.gnu-tools-for-stm32.10.3-2021.10.linux64_1.0.0.202111181127/tools/bin/../lib/gcc/arm-none-eabi/10.3.1/../../../../arm-none-eabi/lib/thumb/v6-m/nofp/libc_nano.a(lib_a-wctomb_r.o)
                              /opt/st/stm32cubeide_1.9.0/plugins/com.st.stm32cube.ide.mcu.externaltools.gnu-tools-for-stm32.10.3-2021.10.linux64_1.0.0.202111181127/tools/bin/../lib/gcc/arm-none-eabi/10.3.1/../../../../arm-none-eabi/lib/thumb/v6-m/nofp/libc_nano.a(lib_a-locale.o) (__ascii_wctomb)
/opt/st/stm32cubeide_1.9.0/plugins/com.st.stm32cube.ide.mcu.externaltools.gnu-tools-for-stm32.10.3-2021.10.linux64_1.0.0.202111181127/tools/bin/../lib/gcc/arm-none-eabi/10.3.1/../../../../arm-none-eabi/lib/thumb/v6-m/nofp/libc_nano.a(lib_a-writer.o)
                              /opt/st/stm32cubeide_1.9.0/plugins/com.st.stm32cube.ide.mcu.externaltools.gnu-tools-for-stm32.10.3-2021.10.linux64_1.0.0.202111181127/tools/bin/../lib/gcc/arm-none-eabi/10.3.1/../../../../arm-none-eabi/lib/thumb/v6-m/nofp/libc_nano.a(lib_a-stdio.o) (_write_r)
/opt/st/stm32cubeide_1.9.0/plugins/com.st.stm32cube.ide.mcu.externaltools.gnu-tools-for-stm32.10.3-2021.10.linux64_1.0.0.202111181127/tools/bin/../lib/gcc/arm-none-eabi/10.3.1/../../../../arm-none-eabi/lib/thumb/v6-m/nofp/libc_nano.a(lib_a-assert.o)
                              /opt/st/stm32cubeide_1.9.0/plugins/com.st.stm32cube.ide.mcu.externaltools.gnu-tools-for-stm32.10.3-2021.10.linux64_1.0.0.202111181127/tools/bin/../lib/gcc/arm-none-eabi/10.3.1/../../../../arm-none-eabi/lib/thumb/v6-m/nofp/libc_nano.a(lib_a-dtoa.o) (__assert_func)
/opt/st/stm32cubeide_1.9.0/plugins/com.st.stm32cube.ide.mcu.externaltools.gnu-tools-for-stm32.10.3-2021.10.linux64_1.0.0.202111181127/tools/bin/../lib/gcc/arm-none-eabi/10.3.1/../../../../arm-none-eabi/lib/thumb/v6-m/nofp/libc_nano.a(lib_a-closer.o)
                              /opt/st/stm32cubeide_1.9.0/plugins/com.st.stm32cube.ide.mcu.externaltools.gnu-tools-for-stm32.10.3-2021.10.linux64_1.0.0.202111181127/tools/bin/../lib/gcc/arm-none-eabi/10.3.1/../../../../arm-none-eabi/lib/thumb/v6-m/nofp/libc_nano.a(lib_a-stdio.o) (_close_r)
/opt/st/stm32cubeide_1.9.0/plugins/com.st.stm32cube.ide.mcu.externaltools.gnu-tools-for-stm32.10.3-2021.10.linux64_1.0.0.202111181127/tools/bin/../lib/gcc/arm-none-eabi/10.3.1/../../../../arm-none-eabi/lib/thumb/v6-m/nofp/libc_nano.a(lib_a-environ.o)
                              /opt/st/stm32cubeide_1.9.0/plugins/com.st.stm32cube.ide.mcu.externaltools.gnu-tools-for-stm32.10.3-2021.10.linux64_1.0.0.202111181127/tools/bin/../lib/gcc/arm-none-eabi/10.3.1/../../../../arm-none-eabi/lib/thumb/v6-m/nofp/libc_nano.a(lib_a-getenv_r.o) (environ)
/opt/st/stm32cubeide_1.9.0/plugins/com.st.stm32cube.ide.mcu.externaltools.gnu-tools-for-stm32.10.3-2021.10.linux64_1.0.0.202111181127/tools/bin/../lib/gcc/arm-none-eabi/10.3.1/../../../../arm-none-eabi/lib/thumb/v6-m/nofp/libc_nano.a(lib_a-envlock.o)
                              /opt/st/stm32cubeide_1.9.0/plugins/com.st.stm32cube.ide.mcu.externaltools.gnu-tools-for-stm32.10.3-2021.10.linux64_1.0.0.202111181127/tools/bin/../lib/gcc/arm-none-eabi/10.3.1/../../../../arm-none-eabi/lib/thumb/v6-m/nofp/libc_nano.a(lib_a-getenv_r.o) (__env_lock)
/opt/st/stm32cubeide_1.9.0/plugins/com.st.stm32cube.ide.mcu.externaltools.gnu-tools-for-stm32.10.3-2021.10.linux64_1.0.0.202111181127/tools/bin/../lib/gcc/arm-none-eabi/10.3.1/../../../../arm-none-eabi/lib/thumb/v6-m/nofp/libc_nano.a(lib_a-fprintf.o)
                              /opt/st/stm32cubeide_1.9.0/plugins/com.st.stm32cube.ide.mcu.externaltools.gnu-tools-for-stm32.10.3-2021.10.linux64_1.0.0.202111181127/tools/bin/../lib/gcc/arm-none-eabi/10.3.1/../../../../arm-none-eabi/lib/thumb/v6-m/nofp/libc_nano.a(lib_a-assert.o) (fiprintf)
/opt/st/stm32cubeide_1.9.0/plugins/com.st.stm32cube.ide.mcu.externaltools.gnu-tools-for-stm32.10.3-2021.10.linux64_1.0.0.202111181127/tools/bin/../lib/gcc/arm-none-eabi/10.3.1/../../../../arm-none-eabi/lib/thumb/v6-m/nofp/libc_nano.a(lib_a-lseekr.o)
                              /opt/st/stm32cubeide_1.9.0/plugins/com.st.stm32cube.ide.mcu.externaltools.gnu-tools-for-stm32.10.3-2021.10.linux64_1.0.0.202111181127/tools/bin/../lib/gcc/arm-none-eabi/10.3.1/../../../../arm-none-eabi/lib/thumb/v6-m/nofp/libc_nano.a(lib_a-stdio.o) (_lseek_r)
/opt/st/stm32cubeide_1.9.0/plugins/com.st.stm32cube.ide.mcu.externaltools.gnu-tools-for-stm32.10.3-2021.10.linux64_1.0.0.202111181127/tools/bin/../lib/gcc/arm-none-eabi/10.3.1/../../../../arm-none-eabi/lib/thumb/v6-m/nofp/libc_nano.a(lib_a-memmove.o)
                              /opt/st/stm32cubeide_1.9.0/plugins/com.st.stm32cube.ide.mcu.externaltools.gnu-tools-for-stm32.10.3-2021.10.linux64_1.0.0.202111181127/tools/bin/../lib/gcc/arm-none-eabi/10.3.1/../../../../arm-none-eabi/lib/thumb/v6-m/nofp/libc_nano.a(lib_a-nano-svfprintf.o) (memmove)
/opt/st/stm32cubeide_1.9.0/plugins/com.st.stm32cube.ide.mcu.externaltools.gnu-tools-for-stm32.10.3-2021.10.linux64_1.0.0.202111181127/tools/bin/../lib/gcc/arm-none-eabi/10.3.1/../../../../arm-none-eabi/lib/thumb/v6-m/nofp/libc_nano.a(lib_a-mlock.o)
                              /opt/st/stm32cubeide_1.9.0/plugins/com.st.stm32cube.ide.mcu.externaltools.gnu-tools-for-stm32.10.3-2021.10.linux64_1.0.0.202111181127/tools/bin/../lib/gcc/arm-none-eabi/10.3.1/../../../../arm-none-eabi/lib/thumb/v6-m/nofp/libc_nano.a(lib_a-nano-freer.o) (__malloc_lock)
/opt/st/stm32cubeide_1.9.0/plugins/com.st.stm32cube.ide.mcu.externaltools.gnu-tools-for-stm32.10.3-2021.10.linux64_1.0.0.202111181127/tools/bin/../lib/gcc/arm-none-eabi/10.3.1/../../../../arm-none-eabi/lib/thumb/v6-m/nofp/libc_nano.a(lib_a-nano-reallocr.o)
                              /opt/st/stm32cubeide_1.9.0/plugins/com.st.stm32cube.ide.mcu.externaltools.gnu-tools-for-stm32.10.3-2021.10.linux64_1.0.0.202111181127/tools/bin/../lib/gcc/arm-none-eabi/10.3.1/../../../../arm-none-eabi/lib/thumb/v6-m/nofp/libc_nano.a(lib_a-nano-svfprintf.o) (_realloc_r)
/opt/st/stm32cubeide_1.9.0/plugins/com.st.stm32cube.ide.mcu.externaltools.gnu-tools-for-stm32.10.3-2021.10.linux64_1.0.0.202111181127/tools/bin/../lib/gcc/arm-none-eabi/10.3.1/../../../../arm-none-eabi/lib/thumb/v6-m/nofp/libc_nano.a(lib_a-nano-svfscanf.o)
                              /opt/st/stm32cubeide_1.9.0/plugins/com.st.stm32cube.ide.mcu.externaltools.gnu-tools-for-stm32.10.3-2021.10.linux64_1.0.0.202111181127/tools/bin/../lib/gcc/arm-none-eabi/10.3.1/../../../../arm-none-eabi/lib/thumb/v6-m/nofp/libc_nano.a(lib_a-sscanf.o) (__ssvfscanf_r)
/opt/st/stm32cubeide_1.9.0/plugins/com.st.stm32cube.ide.mcu.externaltools.gnu-tools-for-stm32.10.3-2021.10.linux64_1.0.0.202111181127/tools/bin/../lib/gcc/arm-none-eabi/10.3.1/../../../../arm-none-eabi/lib/thumb/v6-m/nofp/libc_nano.a(lib_a-nano-vfprintf.o)
                              /opt/st/stm32cubeide_1.9.0/plugins/com.st.stm32cube.ide.mcu.externaltools.gnu-tools-for-stm32.10.3-2021.10.linux64_1.0.0.202111181127/tools/bin/../lib/gcc/arm-none-eabi/10.3.1/../../../../arm-none-eabi/lib/thumb/v6-m/nofp/libc_nano.a(lib_a-fprintf.o) (_vfprintf_r)
/opt/st/stm32cubeide_1.9.0/plugins/com.st.stm32cube.ide.mcu.externaltools.gnu-tools-for-stm32.10.3-2021.10.linux64_1.0.0.202111181127/tools/bin/../lib/gcc/arm-none-eabi/10.3.1/../../../../arm-none-eabi/lib/thumb/v6-m/nofp/libc_nano.a(lib_a-nano-vfscanf_i.o)
                              /opt/st/stm32cubeide_1.9.0/plugins/com.st.stm32cube.ide.mcu.externaltools.gnu-tools-for-stm32.10.3-2021.10.linux64_1.0.0.202111181127/tools/bin/../lib/gcc/arm-none-eabi/10.3.1/../../../../arm-none-eabi/lib/thumb/v6-m/nofp/libc_nano.a(lib_a-nano-svfscanf.o) (_scanf_chars)
/opt/st/stm32cubeide_1.9.0/plugins/com.st.stm32cube.ide.mcu.externaltools.gnu-tools-for-stm32.10.3-2021.10.linux64_1.0.0.202111181127/tools/bin/../lib/gcc/arm-none-eabi/10.3.1/../../../../arm-none-eabi/lib/thumb/v6-m/nofp/libc_nano.a(lib_a-readr.o)
                              /opt/st/stm32cubeide_1.9.0/plugins/com.st.stm32cube.ide.mcu.externaltools.gnu-tools-for-stm32.10.3-2021.10.linux64_1.0.0.202111181127/tools/bin/../lib/gcc/arm-none-eabi/10.3.1/../../../../arm-none-eabi/lib/thumb/v6-m/nofp/libc_nano.a(lib_a-stdio.o) (_read_r)
/opt/st/stm32cubeide_1.9.0/plugins/com.st.stm32cube.ide.mcu.externaltools.gnu-tools-for-stm32.10.3-2021.10.linux64_1.0.0.202111181127/tools/bin/../lib/gcc/arm-none-eabi/10.3.1/../../../../arm-none-eabi/lib/thumb/v6-m/nofp/libc_nano.a(lib_a-reent.o)
                              /opt/st/stm32cubeide_1.9.0/plugins/com.st.stm32cube.ide.mcu.externaltools.gnu-tools-for-stm32.10.3-2021.10.linux64_1.0.0.202111181127/tools/bin/../lib/gcc/arm-none-eabi/10.3.1/../../../../arm-none-eabi/lib/thumb/v6-m/nofp/libc_nano.a(lib_a-sbrkr.o) (errno)
/opt/st/stm32cubeide_1.9.0/plugins/com.st.stm32cube.ide.mcu.externaltools.gnu-tools-for-stm32.10.3-2021.10.linux64_1.0.0.202111181127/tools/bin/../lib/gcc/arm-none-eabi/10.3.1/../../../../arm-none-eabi/lib/thumb/v6-m/nofp/libc_nano.a(lib_a-sccl.o)
                              /opt/st/stm32cubeide_1.9.0/plugins/com.st.stm32cube.ide.mcu.externaltools.gnu-tools-for-stm32.10.3-2021.10.linux64_1.0.0.202111181127/tools/bin/../lib/gcc/arm-none-eabi/10.3.1/../../../../arm-none-eabi/lib/thumb/v6-m/nofp/libc_nano.a(lib_a-nano-svfscanf.o) (__sccl)
/opt/st/stm32cubeide_1.9.0/plugins/com.st.stm32cube.ide.mcu.externaltools.gnu-tools-for-stm32.10.3-2021.10.linux64_1.0.0.202111181127/tools/bin/../lib/gcc/arm-none-eabi/10.3.1/../../../../arm-none-eabi/lib/thumb/v6-m/nofp/libc_nano.a(lib_a-ungetc.o)
                              /opt/st/stm32cubeide_1.9.0/plugins/com.st.stm32cube.ide.mcu.externaltools.gnu-tools-for-stm32.10.3-2021.10.linux64_1.0.0.202111181127/tools/bin/../lib/gcc/arm-none-eabi/10.3.1/../../../../arm-none-eabi/lib/thumb/v6-m/nofp/libc_nano.a(lib_a-nano-svfscanf.o) (__submore)
/opt/st/stm32cubeide_1.9.0/plugins/com.st.stm32cube.ide.mcu.externaltools.gnu-tools-for-stm32.10.3-2021.10.linux64_1.0.0.202111181127/tools/bin/../lib/gcc/arm-none-eabi/10.3.1/../../../../arm-none-eabi/lib/thumb/v6-m/nofp/libc_nano.a(lib_a-wbuf.o)
                              /opt/st/stm32cubeide_1.9.0/plugins/com.st.stm32cube.ide.mcu.externaltools.gnu-tools-for-stm32.10.3-2021.10.linux64_1.0.0.202111181127/tools/bin/../lib/gcc/arm-none-eabi/10.3.1/../../../../arm-none-eabi/lib/thumb/v6-m/nofp/libc_nano.a(lib_a-nano-vfprintf.o) (__swbuf_r)
/opt/st/stm32cubeide_1.9.0/plugins/com.st.stm32cube.ide.mcu.externaltools.gnu-tools-for-stm32.10.3-2021.10.linux64_1.0.0.202111181127/tools/bin/../lib/gcc/arm-none-eabi/10.3.1/../../../../arm-none-eabi/lib/thumb/v6-m/nofp/libc_nano.a(lib_a-wsetup.o)
                              /opt/st/stm32cubeide_1.9.0/plugins/com.st.stm32cube.ide.mcu.externaltools.gnu-tools-for-stm32.10.3-2021.10.linux64_1.0.0.202111181127/tools/bin/../lib/gcc/arm-none-eabi/10.3.1/../../../../arm-none-eabi/lib/thumb/v6-m/nofp/libc_nano.a(lib_a-nano-vfprintf.o) (__swsetup_r)
/opt/st/stm32cubeide_1.9.0/plugins/com.st.stm32cube.ide.mcu.externaltools.gnu-tools-for-stm32.10.3-2021.10.linux64_1.0.0.202111181127/tools/bin/../lib/gcc/arm-none-eabi/10.3.1/../../../../arm-none-eabi/lib/thumb/v6-m/nofp/libc_nano.a(lib_a-abort.o)
                              /opt/st/stm32cubeide_1.9.0/plugins/com.st.stm32cube.ide.mcu.externaltools.gnu-tools-for-stm32.10.3-2021.10.linux64_1.0.0.202111181127/tools/bin/../lib/gcc/arm-none-eabi/10.3.1/../../../../arm-none-eabi/lib/thumb/v6-m/nofp/libc_nano.a(lib_a-assert.o) (abort)
/opt/st/stm32cubeide_1.9.0/plugins/com.st.stm32cube.ide.mcu.externaltools.gnu-tools-for-stm32.10.3-2021.10.linux64_1.0.0.202111181127/tools/bin/../lib/gcc/arm-none-eabi/10.3.1/../../../../arm-none-eabi/lib/thumb/v6-m/nofp/libc_nano.a(lib_a-fflush.o)
                              /opt/st/stm32cubeide_1.9.0/plugins/com.st.stm32cube.ide.mcu.externaltools.gnu-tools-for-stm32.10.3-2021.10.linux64_1.0.0.202111181127/tools/bin/../lib/gcc/arm-none-eabi/10.3.1/../../../../arm-none-eabi/lib/thumb/v6-m/nofp/libc_nano.a(lib_a-ungetc.o) (_fflush_r)
/opt/st/stm32cubeide_1.9.0/plugins/com.st.stm32cube.ide.mcu.externaltools.gnu-tools-for-stm32.10.3-2021.10.linux64_1.0.0.202111181127/tools/bin/../lib/gcc/arm-none-eabi/10.3.1/../../../../arm-none-eabi/lib/thumb/v6-m/nofp/libc_nano.a(lib_a-findfp.o)
                              /opt/st/stm32cubeide_1.9.0/plugins/com.st.stm32cube.ide.mcu.externaltools.gnu-tools-for-stm32.10.3-2021.10.linux64_1.0.0.202111181127/tools/bin/../lib/gcc/arm-none-eabi/10.3.1/../../../../arm-none-eabi/lib/thumb/v6-m/nofp/libc_nano.a(lib_a-nano-vfprintf.o) (__sinit)
/opt/st/stm32cubeide_1.9.0/plugins/com.st.stm32cube.ide.mcu.externaltools.gnu-tools-for-stm32.10.3-2021.10.linux64_1.0.0.202111181127/tools/bin/../lib/gcc/arm-none-eabi/10.3.1/../../../../arm-none-eabi/lib/thumb/v6-m/nofp/libc_nano.a(lib_a-fvwrite.o)
                              /opt/st/stm32cubeide_1.9.0/plugins/com.st.stm32cube.ide.mcu.externaltools.gnu-tools-for-stm32.10.3-2021.10.linux64_1.0.0.202111181127/tools/bin/../lib/gcc/arm-none-eabi/10.3.1/../../../../arm-none-eabi/lib/thumb/v6-m/nofp/libc_nano.a(lib_a-nano-vfprintf.o) (__sfvwrite_r)
/opt/st/stm32cubeide_1.9.0/plugins/com.st.stm32cube.ide.mcu.externaltools.gnu-tools-for-stm32.10.3-2021.10.linux64_1.0.0.202111181127/tools/bin/../lib/gcc/arm-none-eabi/10.3.1/../../../../arm-none-eabi/lib/thumb/v6-m/nofp/libc_nano.a(lib_a-fwalk.o)
                              /opt/st/stm32cubeide_1.9.0/plugins/com.st.stm32cube.ide.mcu.externaltools.gnu-tools-for-stm32.10.3-2021.10.linux64_1.0.0.202111181127/tools/bin/../lib/gcc/arm-none-eabi/10.3.1/../../../../arm-none-eabi/lib/thumb/v6-m/nofp/libc_nano.a(lib_a-findfp.o) (_fwalk)
/opt/st/stm32cubeide_1.9.0/plugins/com.st.stm32cube.ide.mcu.externaltools.gnu-tools-for-stm32.10.3-2021.10.linux64_1.0.0.202111181127/tools/bin/../lib/gcc/arm-none-eabi/10.3.1/../../../../arm-none-eabi/lib/thumb/v6-m/nofp/libc_nano.a(lib_a-makebuf.o)
                              /opt/st/stm32cubeide_1.9.0/plugins/com.st.stm32cube.ide.mcu.externaltools.gnu-tools-for-stm32.10.3-2021.10.linux64_1.0.0.202111181127/tools/bin/../lib/gcc/arm-none-eabi/10.3.1/../../../../arm-none-eabi/lib/thumb/v6-m/nofp/libc_nano.a(lib_a-wsetup.o) (__smakebuf_r)
/opt/st/stm32cubeide_1.9.0/plugins/com.st.stm32cube.ide.mcu.externaltools.gnu-tools-for-stm32.10.3-2021.10.linux64_1.0.0.202111181127/tools/bin/../lib/gcc/arm-none-eabi/10.3.1/../../../../arm-none-eabi/lib/thumb/v6-m/nofp/libc_nano.a(lib_a-nano-msizer.o)
                              /opt/st/stm32cubeide_1.9.0/plugins/com.st.stm32cube.ide.mcu.externaltools.gnu-tools-for-stm32.10.3-2021.10.linux64_1.0.0.202111181127/tools/bin/../lib/gcc/arm-none-eabi/10.3.1/../../../../arm-none-eabi/lib/thumb/v6-m/nofp/libc_nano.a(lib_a-nano-reallocr.o) (_malloc_usable_size_r)
/opt/st/stm32cubeide_1.9.0/plugins/com.st.stm32cube.ide.mcu.externaltools.gnu-tools-for-stm32.10.3-2021.10.linux64_1.0.0.202111181127/tools/bin/../lib/gcc/arm-none-eabi/10.3.1/../../../../arm-none-eabi/lib/thumb/v6-m/nofp/libc_nano.a(lib_a-signal.o)
                              /opt/st/stm32cubeide_1.9.0/plugins/com.st.stm32cube.ide.mcu.externaltools.gnu-tools-for-stm32.10.3-2021.10.linux64_1.0.0.202111181127/tools/bin/../lib/gcc/arm-none-eabi/10.3.1/../../../../arm-none-eabi/lib/thumb/v6-m/nofp/libc_nano.a(lib_a-abort.o) (raise)
/opt/st/stm32cubeide_1.9.0/plugins/com.st.stm32cube.ide.mcu.externaltools.gnu-tools-for-stm32.10.3-2021.10.linux64_1.0.0.202111181127/tools/bin/../lib/gcc/arm-none-eabi/10.3.1/../../../../arm-none-eabi/lib/thumb/v6-m/nofp/libc_nano.a(lib_a-signalr.o)
                              /opt/st/stm32cubeide_1.9.0/plugins/com.st.stm32cube.ide.mcu.externaltools.gnu-tools-for-stm32.10.3-2021.10.linux64_1.0.0.202111181127/tools/bin/../lib/gcc/arm-none-eabi/10.3.1/../../../../arm-none-eabi/lib/thumb/v6-m/nofp/libc_nano.a(lib_a-signal.o) (_kill_r)
/opt/st/stm32cubeide_1.9.0/plugins/com.st.stm32cube.ide.mcu.externaltools.gnu-tools-for-stm32.10.3-2021.10.linux64_1.0.0.202111181127/tools/bin/../lib/gcc/arm-none-eabi/10.3.1/../../../../arm-none-eabi/lib/thumb/v6-m/nofp/libc_nano.a(lib_a-fstatr.o)
                              /opt/st/stm32cubeide_1.9.0/plugins/com.st.stm32cube.ide.mcu.externaltools.gnu-tools-for-stm32.10.3-2021.10.linux64_1.0.0.202111181127/tools/bin/../lib/gcc/arm-none-eabi/10.3.1/../../../../arm-none-eabi/lib/thumb/v6-m/nofp/libc_nano.a(lib_a-makebuf.o) (_fstat_r)
/opt/st/stm32cubeide_1.9.0/plugins/com.st.stm32cube.ide.mcu.externaltools.gnu-tools-for-stm32.10.3-2021.10.linux64_1.0.0.202111181127/tools/bin/../lib/gcc/arm-none-eabi/10.3.1/../../../../arm-none-eabi/lib/thumb/v6-m/nofp/libc_nano.a(lib_a-isattyr.o)
                              /opt/st/stm32cubeide_1.9.0/plugins/com.st.stm32cube.ide.mcu.externaltools.gnu-tools-for-stm32.10.3-2021.10.linux64_1.0.0.202111181127/tools/bin/../lib/gcc/arm-none-eabi/10.3.1/../../../../arm-none-eabi/lib/thumb/v6-m/nofp/libc_nano.a(lib_a-makebuf.o) (_isatty_r)
/opt/st/stm32cubeide_1.9.0/plugins/com.st.stm32cube.ide.mcu.externaltools.gnu-tools-for-stm32.10.3-2021.10.linux64_1.0.0.202111181127/tools/bin/../lib/gcc/arm-none-eabi/10.3.1/../../../../arm-none-eabi/lib/thumb/v6-m/nofp/libm.a(lib_a-s_ceil.o)
                              ./Drivers/BSP/Components/sx1276/sx1276.o (ceil)
/opt/st/stm32cubeide_1.9.0/plugins/com.st.stm32cube.ide.mcu.externaltools.gnu-tools-for-stm32.10.3-2021.10.linux64_1.0.0.202111181127/tools/bin/../lib/gcc/arm-none-eabi/10.3.1/../../../../arm-none-eabi/lib/thumb/v6-m/nofp/libm.a(lib_a-s_floor.o)
                              ./App/LoRaWAN/src/hw_rtc.o (floor)
/opt/st/stm32cubeide_1.9.0/plugins/com.st.stm32cube.ide.mcu.externaltools.gnu-tools-for-stm32.10.3-2021.10.linux64_1.0.0.202111181127/tools/bin/../lib/gcc/arm-none-eabi/10.3.1/../../../../arm-none-eabi/lib/thumb/v6-m/nofp/libm.a(lib_a-s_round.o)
                              ./Drivers/BSP/Components/sx1276/sx1276.o (round)
/opt/st/stm32cubeide_1.9.0/plugins/com.st.stm32cube.ide.mcu.externaltools.gnu-tools-for-stm32.10.3-2021.10.linux64_1.0.0.202111181127/tools/bin/../lib/gcc/arm-none-eabi/10.3.1/thumb/v6-m/nofp/libgcc.a(_thumb1_case_uqi.o)
                              /opt/st/stm32cubeide_1.9.0/plugins/com.st.stm32cube.ide.mcu.externaltools.gnu-tools-for-stm32.10.3-2021.10.linux64_1.0.0.202111181127/tools/bin/../lib/gcc/arm-none-eabi/10.3.1/../../../../arm-none-eabi/lib/thumb/v6-m/nofp/libc_nano.a(lib_a-strtod.o) (__gnu_thumb1_case_uqi)
/opt/st/stm32cubeide_1.9.0/plugins/com.st.stm32cube.ide.mcu.externaltools.gnu-tools-for-stm32.10.3-2021.10.linux64_1.0.0.202111181127/tools/bin/../lib/gcc/arm-none-eabi/10.3.1/thumb/v6-m/nofp/libgcc.a(_thumb1_case_shi.o)
                              /opt/st/stm32cubeide_1.9.0/plugins/com.st.stm32cube.ide.mcu.externaltools.gnu-tools-for-stm32.10.3-2021.10.linux64_1.0.0.202111181127/tools/bin/../lib/gcc/arm-none-eabi/10.3.1/../../../../arm-none-eabi/lib/thumb/v6-m/nofp/libc_nano.a(lib_a-nano-vfprintf_i.o) (__gnu_thumb1_case_shi)
/opt/st/stm32cubeide_1.9.0/plugins/com.st.stm32cube.ide.mcu.externaltools.gnu-tools-for-stm32.10.3-2021.10.linux64_1.0.0.202111181127/tools/bin/../lib/gcc/arm-none-eabi/10.3.1/thumb/v6-m/nofp/libgcc.a(_udivsi3.o)
                              ./App/Aquaponics/aquaponics.o (__aeabi_uidiv)
/opt/st/stm32cubeide_1.9.0/plugins/com.st.stm32cube.ide.mcu.externaltools.gnu-tools-for-stm32.10.3-2021.10.linux64_1.0.0.202111181127/tools/bin/../lib/gcc/arm-none-eabi/10.3.1/thumb/v6-m/nofp/libgcc.a(_divsi3.o)
                              ./App/Aquaponics/aquaponics.o (__aeabi_idiv)
/opt/st/stm32cubeide_1.9.0/plugins/com.st.stm32cube.ide.mcu.externaltools.gnu-tools-for-stm32.10.3-2021.10.linux64_1.0.0.202111181127/tools/bin/../lib/gcc/arm-none-eabi/10.3.1/thumb/v6-m/nofp/libgcc.a(_dvmd_tls.o)
                              /opt/st/stm32cubeide_1.9.0/plugins/com.st.stm32cube.ide.mcu.externaltools.gnu-tools-for-stm32.10.3-2021.10.linux64_1.0.0.202111181127/tools/bin/../lib/gcc/arm-none-eabi/10.3.1/thumb/v6-m/nofp/libgcc.a(_udivsi3.o) (__aeabi_idiv0)
/opt/st/stm32cubeide_1.9.0/plugins/com.st.stm32cube.ide.mcu.externaltools.gnu-tools-for-stm32.10.3-2021.10.linux64_1.0.0.202111181127/tools/bin/../lib/gcc/arm-none-eabi/10.3.1/thumb/v6-m/nofp/libgcc.a(_arm_cmpdf2.o)
                              /opt/st/stm32cubeide_1.9.0/plugins/com.st.stm32cube.ide.mcu.externaltools.gnu-tools-for-stm32.10.3-2021.10.linux64_1.0.0.202111181127/tools/bin/../lib/gcc/arm-none-eabi/10.3.1/../../../../arm-none-eabi/lib/thumb/v6-m/nofp/libc_nano.a(lib_a-nano-vfprintf_float.o) (__aeabi_dcmpeq)
/opt/st/stm32cubeide_1.9.0/plugins/com.st.stm32cube.ide.mcu.externaltools.gnu-tools-for-stm32.10.3-2021.10.linux64_1.0.0.202111181127/tools/bin/../lib/gcc/arm-none-eabi/10.3.1/thumb/v6-m/nofp/libgcc.a(_arm_cmpsf2.o)
                              ./App/Aquaponics/aquaponics.o (__aeabi_fcmpeq)
/opt/st/stm32cubeide_1.9.0/plugins/com.st.stm32cube.ide.mcu.externaltools.gnu-tools-for-stm32.10.3-2021.10.linux64_1.0.0.202111181127/tools/bin/../lib/gcc/arm-none-eabi/10.3.1/thumb/v6-m/nofp/libgcc.a(_aeabi_uldivmod.o)
                              ./App/LoRaWAN/src/hw_rtc.o (__aeabi_uldivmod)
/opt/st/stm32cubeide_1.9.0/plugins/com.st.stm32cube.ide.mcu.externaltools.gnu-tools-for-stm32.10.3-2021.10.linux64_1.0.0.202111181127/tools/bin/../lib/gcc/arm-none-eabi/10.3.1/thumb/v6-m/nofp/libgcc.a(_muldi3.o)
                              /opt/st/stm32cubeide_1.9.0/plugins/com.st.stm32cube.ide.mcu.externaltools.gnu-tools-for-stm32.10.3-2021.10.linux64_1.0.0.202111181127/tools/bin/../lib/gcc/arm-none-eabi/10.3.1/../../../../arm-none-eabi/lib/thumb/v6-m/nofp/libc_nano.a(lib_a-mktime.o) (__aeabi_lmul)
/opt/st/stm32cubeide_1.9.0/plugins/com.st.stm32cube.ide.mcu.externaltools.gnu-tools-for-stm32.10.3-2021.10.linux64_1.0.0.202111181127/tools/bin/../lib/gcc/arm-none-eabi/10.3.1/thumb/v6-m/nofp/libgcc.a(_fixunssfsi.o)
                              ./App/Aquaponics/aquaponics.o (__aeabi_f2uiz)
/opt/st/stm32cubeide_1.9.0/plugins/com.st.stm32cube.ide.mcu.externaltools.gnu-tools-for-stm32.10.3-2021.10.linux64_1.0.0.202111181127/tools/bin/../lib/gcc/arm-none-eabi/10.3.1/thumb/v6-m/nofp/libgcc.a(_fixunsdfsi.o)
                              ./App/Aquaponics/aquaponics.o (__aeabi_d2uiz)
/opt/st/stm32cubeide_1.9.0/plugins/com.st.stm32cube.ide.mcu.externaltools.gnu-tools-for-stm32.10.3-2021.10.linux64_1.0.0.202111181127/tools/bin/../lib/gcc/arm-none-eabi/10.3.1/thumb/v6-m/nofp/libgcc.a(_fixdfdi.o)
                              /opt/st/stm32cubeide_1.9.0/plugins/com.st.stm32cube.ide.mcu.externaltools.gnu-tools-for-stm32.10.3-2021.10.linux64_1.0.0.202111181127/tools/bin/../lib/gcc/arm-none-eabi/10.3.1/../../../../arm-none-eabi/lib/thumb/v6-m/nofp/libc_nano.a(lib_a-strtod.o) (__aeabi_d2lz)
/opt/st/stm32cubeide_1.9.0/plugins/com.st.stm32cube.ide.mcu.externaltools.gnu-tools-for-stm32.10.3-2021.10.linux64_1.0.0.202111181127/tools/bin/../lib/gcc/arm-none-eabi/10.3.1/thumb/v6-m/nofp/libgcc.a(_fixunsdfdi.o)
                              /opt/st/stm32cubeide_1.9.0/plugins/com.st.stm32cube.ide.mcu.externaltools.gnu-tools-for-stm32.10.3-2021.10.linux64_1.0.0.202111181127/tools/bin/../lib/gcc/arm-none-eabi/10.3.1/thumb/v6-m/nofp/libgcc.a(_fixdfdi.o) (__aeabi_d2ulz)
/opt/st/stm32cubeide_1.9.0/plugins/com.st.stm32cube.ide.mcu.externaltools.gnu-tools-for-stm32.10.3-2021.10.linux64_1.0.0.202111181127/tools/bin/../lib/gcc/arm-none-eabi/10.3.1/thumb/v6-m/nofp/libgcc.a(_floatdidf.o)
                              /opt/st/stm32cubeide_1.9.0/plugins/com.st.stm32cube.ide.mcu.externaltools.gnu-tools-for-stm32.10.3-2021.10.linux64_1.0.0.202111181127/tools/bin/../lib/gcc/arm-none-eabi/10.3.1/../../../../arm-none-eabi/lib/thumb/v6-m/nofp/libc_nano.a(lib_a-strtod.o) (__aeabi_l2d)
/opt/st/stm32cubeide_1.9.0/plugins/com.st.stm32cube.ide.mcu.externaltools.gnu-tools-for-stm32.10.3-2021.10.linux64_1.0.0.202111181127/tools/bin/../lib/gcc/arm-none-eabi/10.3.1/thumb/v6-m/nofp/libgcc.a(_udivmoddi4.o)
                              /opt/st/stm32cubeide_1.9.0/plugins/com.st.stm32cube.ide.mcu.externaltools.gnu-tools-for-stm32.10.3-2021.10.linux64_1.0.0.202111181127/tools/bin/../lib/gcc/arm-none-eabi/10.3.1/thumb/v6-m/nofp/libgcc.a(_aeabi_uldivmod.o) (__udivmoddi4)
/opt/st/stm32cubeide_1.9.0/plugins/com.st.stm32cube.ide.mcu.externaltools.gnu-tools-for-stm32.10.3-2021.10.linux64_1.0.0.202111181127/tools/bin/../lib/gcc/arm-none-eabi/10.3.1/thumb/v6-m/nofp/libgcc.a(addsf3.o)
                              ./App/Aquaponics/aquaponics.o (__aeabi_fadd)
/opt/st/stm32cubeide_1.9.0/plugins/com.st.stm32cube.ide.mcu.externaltools.gnu-tools-for-stm32.10.3-2021.10.linux64_1.0.0.202111181127/tools/bin/../lib/gcc/arm-none-eabi/10.3.1/thumb/v6-m/nofp/libgcc.a(divsf3.o)
                              ./App/Aquaponics/aquaponics.o (__aeabi_fdiv)
/opt/st/stm32cubeide_1.9.0/plugins/com.st.stm32cube.ide.mcu.externaltools.gnu-tools-for-stm32.10.3-2021.10.linux64_1.0.0.202111181127/tools/bin/../lib/gcc/arm-none-eabi/10.3.1/thumb/v6-m/nofp/libgcc.a(eqsf2.o)
                              /opt/st/stm32cubeide_1.9.0/plugins/com.st.stm32cube.ide.mcu.externaltools.gnu-tools-for-stm32.10.3-2021.10.linux64_1.0.0.202111181127/tools/bin/../lib/gcc/arm-none-eabi/10.3.1/thumb/v6-m/nofp/libgcc.a(_arm_cmpsf2.o) (__eqsf2)
/opt/st/stm32cubeide_1.9.0/plugins/com.st.stm32cube.ide.mcu.externaltools.gnu-tools-for-stm32.10.3-2021.10.linux64_1.0.0.202111181127/tools/bin/../lib/gcc/arm-none-eabi/10.3.1/thumb/v6-m/nofp/libgcc.a(gesf2.o)
                              /opt/st/stm32cubeide_1.9.0/plugins/com.st.stm32cube.ide.mcu.externaltools.gnu-tools-for-stm32.10.3-2021.10.linux64_1.0.0.202111181127/tools/bin/../lib/gcc/arm-none-eabi/10.3.1/thumb/v6-m/nofp/libgcc.a(_arm_cmpsf2.o) (__gesf2)
/opt/st/stm32cubeide_1.9.0/plugins/com.st.stm32cube.ide.mcu.externaltools.gnu-tools-for-stm32.10.3-2021.10.linux64_1.0.0.202111181127/tools/bin/../lib/gcc/arm-none-eabi/10.3.1/thumb/v6-m/nofp/libgcc.a(lesf2.o)
                              /opt/st/stm32cubeide_1.9.0/plugins/com.st.stm32cube.ide.mcu.externaltools.gnu-tools-for-stm32.10.3-2021.10.linux64_1.0.0.202111181127/tools/bin/../lib/gcc/arm-none-eabi/10.3.1/thumb/v6-m/nofp/libgcc.a(_arm_cmpsf2.o) (__lesf2)
/opt/st/stm32cubeide_1.9.0/plugins/com.st.stm32cube.ide.mcu.externaltools.gnu-tools-for-stm32.10.3-2021.10.linux64_1.0.0.202111181127/tools/bin/../lib/gcc/arm-none-eabi/10.3.1/thumb/v6-m/nofp/libgcc.a(mulsf3.o)
                              ./App/Aquaponics/aquaponics.o (__aeabi_fmul)
/opt/st/stm32cubeide_1.9.0/plugins/com.st.stm32cube.ide.mcu.externaltools.gnu-tools-for-stm32.10.3-2021.10.linux64_1.0.0.202111181127/tools/bin/../lib/gcc/arm-none-eabi/10.3.1/thumb/v6-m/nofp/libgcc.a(subsf3.o)
                              ./App/LoRaWAN/src/hw_rtc.o (__aeabi_fsub)
/opt/st/stm32cubeide_1.9.0/plugins/com.st.stm32cube.ide.mcu.externaltools.gnu-tools-for-stm32.10.3-2021.10.linux64_1.0.0.202111181127/tools/bin/../lib/gcc/arm-none-eabi/10.3.1/thumb/v6-m/nofp/libgcc.a(unordsf2.o)
                              /opt/st/stm32cubeide_1.9.0/plugins/com.st.stm32cube.ide.mcu.externaltools.gnu-tools-for-stm32.10.3-2021.10.linux64_1.0.0.202111181127/tools/bin/../lib/gcc/arm-none-eabi/10.3.1/../../../../arm-none-eabi/lib/thumb/v6-m/nofp/libc_nano.a(lib_a-strtod.o) (__aeabi_fcmpun)
/opt/st/stm32cubeide_1.9.0/plugins/com.st.stm32cube.ide.mcu.externaltools.gnu-tools-for-stm32.10.3-2021.10.linux64_1.0.0.202111181127/tools/bin/../lib/gcc/arm-none-eabi/10.3.1/thumb/v6-m/nofp/libgcc.a(fixsfsi.o)
                              /opt/st/stm32cubeide_1.9.0/plugins/com.st.stm32cube.ide.mcu.externaltools.gnu-tools-for-stm32.10.3-2021.10.linux64_1.0.0.202111181127/tools/bin/../lib/gcc/arm-none-eabi/10.3.1/thumb/v6-m/nofp/libgcc.a(_fixunssfsi.o) (__aeabi_f2iz)
/opt/st/stm32cubeide_1.9.0/plugins/com.st.stm32cube.ide.mcu.externaltools.gnu-tools-for-stm32.10.3-2021.10.linux64_1.0.0.202111181127/tools/bin/../lib/gcc/arm-none-eabi/10.3.1/thumb/v6-m/nofp/libgcc.a(floatsisf.o)
                              ./Drivers/Middlewares/LoRaWAN/Mac/region/RegionKR920.o (__aeabi_i2f)
/opt/st/stm32cubeide_1.9.0/plugins/com.st.stm32cube.ide.mcu.externaltools.gnu-tools-for-stm32.10.3-2021.10.linux64_1.0.0.202111181127/tools/bin/../lib/gcc/arm-none-eabi/10.3.1/thumb/v6-m/nofp/libgcc.a(floatunsisf.o)
                              ./App/Aquaponics/aquaponics.o (__aeabi_ui2f)
/opt/st/stm32cubeide_1.9.0/plugins/com.st.stm32cube.ide.mcu.externaltools.gnu-tools-for-stm32.10.3-2021.10.linux64_1.0.0.202111181127/tools/bin/../lib/gcc/arm-none-eabi/10.3.1/thumb/v6-m/nofp/libgcc.a(adddf3.o)
                              ./App/Aquaponics/aquaponics.o (__aeabi_dadd)
/opt/st/stm32cubeide_1.9.0/plugins/com.st.stm32cube.ide.mcu.externaltools.gnu-tools-for-stm32.10.3-2021.10.linux64_1.0.0.202111181127/tools/bin/../lib/gcc/arm-none-eabi/10.3.1/thumb/v6-m/nofp/libgcc.a(divdf3.o)
                              ./App/Aquaponics/aquaponics.o (__aeabi_ddiv)
/opt/st/stm32cubeide_1.9.0/plugins/com.st.stm32cube.ide.mcu.externaltools.gnu-tools-for-stm32.10.3-2021.10.linux64_1.0.0.202111181127/tools/bin/../lib/gcc/arm-none-eabi/10.3.1/thumb/v6-m/nofp/libgcc.a(eqdf2.o)
                              /opt/st/stm32cubeide_1.9.0/plugins/com.st.stm32cube.ide.mcu.externaltools.gnu-tools-for-stm32.10.3-2021.10.linux64_1.0.0.202111181127/tools/bin/../lib/gcc/arm-none-eabi/10.3.1/thumb/v6-m/nofp/libgcc.a(_arm_cmpdf2.o) (__eqdf2)
/opt/st/stm32cubeide_1.9.0/plugins/com.st.stm32cube.ide.mcu.externaltools.gnu-tools-for-stm32.10.3-2021.10.linux64_1.0.0.202111181127/tools/bin/../lib/gcc/arm-none-eabi/10.3.1/thumb/v6-m/nofp/libgcc.a(gedf2.o)
                              /opt/st/stm32cubeide_1.9.0/plugins/com.st.stm32cube.ide.mcu.externaltools.gnu-tools-for-stm32.10.3-2021.10.linux64_1.0.0.202111181127/tools/bin/../lib/gcc/arm-none-eabi/10.3.1/thumb/v6-m/nofp/libgcc.a(_arm_cmpdf2.o) (__gedf2)
/opt/st/stm32cubeide_1.9.0/plugins/com.st.stm32cube.ide.mcu.externaltools.gnu-tools-for-stm32.10.3-2021.10.linux64_1.0.0.202111181127/tools/bin/../lib/gcc/arm-none-eabi/10.3.1/thumb/v6-m/nofp/libgcc.a(ledf2.o)
                              /opt/st/stm32cubeide_1.9.0/plugins/com.st.stm32cube.ide.mcu.externaltools.gnu-tools-for-stm32.10.3-2021.10.linux64_1.0.0.202111181127/tools/bin/../lib/gcc/arm-none-eabi/10.3.1/thumb/v6-m/nofp/libgcc.a(_arm_cmpdf2.o) (__ledf2)
/opt/st/stm32cubeide_1.9.0/plugins/com.st.stm32cube.ide.mcu.externaltools.gnu-tools-for-stm32.10.3-2021.10.linux64_1.0.0.202111181127/tools/bin/../lib/gcc/arm-none-eabi/10.3.1/thumb/v6-m/nofp/libgcc.a(muldf3.o)
                              ./App/Aquaponics/aquaponics.o (__aeabi_dmul)
/opt/st/stm32cubeide_1.9.0/plugins/com.st.stm32cube.ide.mcu.externaltools.gnu-tools-for-stm32.10.3-2021.10.linux64_1.0.0.202111181127/tools/bin/../lib/gcc/arm-none-eabi/10.3.1/thumb/v6-m/nofp/libgcc.a(subdf3.o)
                              ./App/Aquaponics/aquaponics.o (__aeabi_dsub)
/opt/st/stm32cubeide_1.9.0/plugins/com.st.stm32cube.ide.mcu.externaltools.gnu-tools-for-stm32.10.3-2021.10.linux64_1.0.0.202111181127/tools/bin/../lib/gcc/arm-none-eabi/10.3.1/thumb/v6-m/nofp/libgcc.a(unorddf2.o)
                              /opt/st/stm32cubeide_1.9.0/plugins/com.st.stm32cube.ide.mcu.externaltools.gnu-tools-for-stm32.10.3-2021.10.linux64_1.0.0.202111181127/tools/bin/../lib/gcc/arm-none-eabi/10.3.1/../../../../arm-none-eabi/lib/thumb/v6-m/nofp/libc_nano.a(lib_a-nano-vfprintf_float.o) (__aeabi_dcmpun)
/opt/st/stm32cubeide_1.9.0/plugins/com.st.stm32cube.ide.mcu.externaltools.gnu-tools-for-stm32.10.3-2021.10.linux64_1.0.0.202111181127/tools/bin/../lib/gcc/arm-none-eabi/10.3.1/thumb/v6-m/nofp/libgcc.a(fixdfsi.o)
                              ./Drivers/Middlewares/LoRaWAN/Mac/region/RegionCommon.o (__aeabi_d2iz)
/opt/st/stm32cubeide_1.9.0/plugins/com.st.stm32cube.ide.mcu.externaltools.gnu-tools-for-stm32.10.3-2021.10.linux64_1.0.0.202111181127/tools/bin/../lib/gcc/arm-none-eabi/10.3.1/thumb/v6-m/nofp/libgcc.a(floatsidf.o)
                              ./App/Aquaponics/aquaponics.o (__aeabi_i2d)
/opt/st/stm32cubeide_1.9.0/plugins/com.st.stm32cube.ide.mcu.externaltools.gnu-tools-for-stm32.10.3-2021.10.linux64_1.0.0.202111181127/tools/bin/../lib/gcc/arm-none-eabi/10.3.1/thumb/v6-m/nofp/libgcc.a(floatunsidf.o)
                              ./Drivers/BSP/Components/sx1276/sx1276.o (__aeabi_ui2d)
/opt/st/stm32cubeide_1.9.0/plugins/com.st.stm32cube.ide.mcu.externaltools.gnu-tools-for-stm32.10.3-2021.10.linux64_1.0.0.202111181127/tools/bin/../lib/gcc/arm-none-eabi/10.3.1/thumb/v6-m/nofp/libgcc.a(extendsfdf2.o)
                              ./App/Aquaponics/aquaponics.o (__aeabi_f2d)
/opt/st/stm32cubeide_1.9.0/plugins/com.st.stm32cube.ide.mcu.externaltools.gnu-tools-for-stm32.10.3-2021.10.linux64_1.0.0.202111181127/tools/bin/../lib/gcc/arm-none-eabi/10.3.1/thumb/v6-m/nofp/libgcc.a(truncdfsf2.o)
                              ./App/Aquaponics/aquaponics.o (__aeabi_d2f)
/opt/st/stm32cubeide_1.9.0/plugins/com.st.stm32cube.ide.mcu.externaltools.gnu-tools-for-stm32.10.3-2021.10.linux64_1.0.0.202111181127/tools/bin/../lib/gcc/arm-none-eabi/10.3.1/thumb/v6-m/nofp/libgcc.a(_clzsi2.o)
                              /opt/st/stm32cubeide_1.9.0/plugins/com.st.stm32cube.ide.mcu.externaltools.gnu-tools-for-stm32.10.3-2021.10.linux64_1.0.0.202111181127/tools/bin/../lib/gcc/arm-none-eabi/10.3.1/thumb/v6-m/nofp/libgcc.a(addsf3.o) (__clzsi2)
/opt/st/stm32cubeide_1.9.0/plugins/com.st.stm32cube.ide.mcu.externaltools.gnu-tools-for-stm32.10.3-2021.10.linux64_1.0.0.202111181127/tools/bin/../lib/gcc/arm-none-eabi/10.3.1/thumb/v6-m/nofp/libgcc.a(_clzdi2.o)
                              /opt/st/stm32cubeide_1.9.0/plugins/com.st.stm32cube.ide.mcu.externaltools.gnu-tools-for-stm32.10.3-2021.10.linux64_1.0.0.202111181127/tools/bin/../lib/gcc/arm-none-eabi/10.3.1/thumb/v6-m/nofp/libgcc.a(_udivmoddi4.o) (__clzdi2)
/opt/st/stm32cubeide_1.9.0/plugins/com.st.stm32cube.ide.mcu.externaltools.gnu-tools-for-stm32.10.3-2021.10.linux64_1.0.0.202111181127/tools/bin/../lib/gcc/arm-none-eabi/10.3.1/../../../../arm-none-eabi/lib/thumb/v6-m/nofp/libnosys.a(close.o)
                              /opt/st/stm32cubeide_1.9.0/plugins/com.st.stm32cube.ide.mcu.externaltools.gnu-tools-for-stm32.10.3-2021.10.linux64_1.0.0.202111181127/tools/bin/../lib/gcc/arm-none-eabi/10.3.1/../../../../arm-none-eabi/lib/thumb/v6-m/nofp/libc_nano.a(lib_a-closer.o) (_close)
/opt/st/stm32cubeide_1.9.0/plugins/com.st.stm32cube.ide.mcu.externaltools.gnu-tools-for-stm32.10.3-2021.10.linux64_1.0.0.202111181127/tools/bin/../lib/gcc/arm-none-eabi/10.3.1/../../../../arm-none-eabi/lib/thumb/v6-m/nofp/libnosys.a(fstat.o)
                              /opt/st/stm32cubeide_1.9.0/plugins/com.st.stm32cube.ide.mcu.externaltools.gnu-tools-for-stm32.10.3-2021.10.linux64_1.0.0.202111181127/tools/bin/../lib/gcc/arm-none-eabi/10.3.1/../../../../arm-none-eabi/lib/thumb/v6-m/nofp/libc_nano.a(lib_a-fstatr.o) (_fstat)
/opt/st/stm32cubeide_1.9.0/plugins/com.st.stm32cube.ide.mcu.externaltools.gnu-tools-for-stm32.10.3-2021.10.linux64_1.0.0.202111181127/tools/bin/../lib/gcc/arm-none-eabi/10.3.1/../../../../arm-none-eabi/lib/thumb/v6-m/nofp/libnosys.a(getpid.o)
                              /opt/st/stm32cubeide_1.9.0/plugins/com.st.stm32cube.ide.mcu.externaltools.gnu-tools-for-stm32.10.3-2021.10.linux64_1.0.0.202111181127/tools/bin/../lib/gcc/arm-none-eabi/10.3.1/../../../../arm-none-eabi/lib/thumb/v6-m/nofp/libc_nano.a(lib_a-signalr.o) (_getpid)
/opt/st/stm32cubeide_1.9.0/plugins/com.st.stm32cube.ide.mcu.externaltools.gnu-tools-for-stm32.10.3-2021.10.linux64_1.0.0.202111181127/tools/bin/../lib/gcc/arm-none-eabi/10.3.1/../../../../arm-none-eabi/lib/thumb/v6-m/nofp/libnosys.a(isatty.o)
                              /opt/st/stm32cubeide_1.9.0/plugins/com.st.stm32cube.ide.mcu.externaltools.gnu-tools-for-stm32.10.3-2021.10.linux64_1.0.0.202111181127/tools/bin/../lib/gcc/arm-none-eabi/10.3.1/../../../../arm-none-eabi/lib/thumb/v6-m/nofp/libc_nano.a(lib_a-isattyr.o) (_isatty)
/opt/st/stm32cubeide_1.9.0/plugins/com.st.stm32cube.ide.mcu.externaltools.gnu-tools-for-stm32.10.3-2021.10.linux64_1.0.0.202111181127/tools/bin/../lib/gcc/arm-none-eabi/10.3.1/../../../../arm-none-eabi/lib/thumb/v6-m/nofp/libnosys.a(kill.o)
                              /opt/st/stm32cubeide_1.9.0/plugins/com.st.stm32cube.ide.mcu.externaltools.gnu-tools-for-stm32.10.3-2021.10.linux64_1.0.0.202111181127/tools/bin/../lib/gcc/arm-none-eabi/10.3.1/../../../../arm-none-eabi/lib/thumb/v6-m/nofp/libc_nano.a(lib_a-signalr.o) (_kill)
/opt/st/stm32cubeide_1.9.0/plugins/com.st.stm32cube.ide.mcu.externaltools.gnu-tools-for-stm32.10.3-2021.10.linux64_1.0.0.202111181127/tools/bin/../lib/gcc/arm-none-eabi/10.3.1/../../../../arm-none-eabi/lib/thumb/v6-m/nofp/libnosys.a(lseek.o)
                              /opt/st/stm32cubeide_1.9.0/plugins/com.st.stm32cube.ide.mcu.externaltools.gnu-tools-for-stm32.10.3-2021.10.linux64_1.0.0.202111181127/tools/bin/../lib/gcc/arm-none-eabi/10.3.1/../../../../arm-none-eabi/lib/thumb/v6-m/nofp/libc_nano.a(lib_a-lseekr.o) (_lseek)
/opt/st/stm32cubeide_1.9.0/plugins/com.st.stm32cube.ide.mcu.externaltools.gnu-tools-for-stm32.10.3-2021.10.linux64_1.0.0.202111181127/tools/bin/../lib/gcc/arm-none-eabi/10.3.1/../../../../arm-none-eabi/lib/thumb/v6-m/nofp/libnosys.a(read.o)
                              /opt/st/stm32cubeide_1.9.0/plugins/com.st.stm32cube.ide.mcu.externaltools.gnu-tools-for-stm32.10.3-2021.10.linux64_1.0.0.202111181127/tools/bin/../lib/gcc/arm-none-eabi/10.3.1/../../../../arm-none-eabi/lib/thumb/v6-m/nofp/libc_nano.a(lib_a-readr.o) (_read)
/opt/st/stm32cubeide_1.9.0/plugins/com.st.stm32cube.ide.mcu.externaltools.gnu-tools-for-stm32.10.3-2021.10.linux64_1.0.0.202111181127/tools/bin/../lib/gcc/arm-none-eabi/10.3.1/../../../../arm-none-eabi/lib/thumb/v6-m/nofp/libnosys.a(sbrk.o)
                              /opt/st/stm32cubeide_1.9.0/plugins/com.st.stm32cube.ide.mcu.externaltools.gnu-tools-for-stm32.10.3-2021.10.linux64_1.0.0.202111181127/tools/bin/../lib/gcc/arm-none-eabi/10.3.1/../../../../arm-none-eabi/lib/thumb/v6-m/nofp/libc_nano.a(lib_a-sbrkr.o) (_sbrk)
/opt/st/stm32cubeide_1.9.0/plugins/com.st.stm32cube.ide.mcu.externaltools.gnu-tools-for-stm32.10.3-2021.10.linux64_1.0.0.202111181127/tools/bin/../lib/gcc/arm-none-eabi/10.3.1/../../../../arm-none-eabi/lib/thumb/v6-m/nofp/libnosys.a(write.o)
                              /opt/st/stm32cubeide_1.9.0/plugins/com.st.stm32cube.ide.mcu.externaltools.gnu-tools-for-stm32.10.3-2021.10.linux64_1.0.0.202111181127/tools/bin/../lib/gcc/arm-none-eabi/10.3.1/../../../../arm-none-eabi/lib/thumb/v6-m/nofp/libc_nano.a(lib_a-writer.o) (_write)
/opt/st/stm32cubeide_1.9.0/plugins/com.st.stm32cube.ide.mcu.externaltools.gnu-tools-for-stm32.10.3-2021.10.linux64_1.0.0.202111181127/tools/bin/../lib/gcc/arm-none-eabi/10.3.1/../../../../arm-none-eabi/lib/thumb/v6-m/nofp/libnosys.a(_exit.o)
                              /opt/st/stm32cubeide_1.9.0/plugins/com.st.stm32cube.ide.mcu.externaltools.gnu-tools-for-stm32.10.3-2021.10.linux64_1.0.0.202111181127/tools/bin/../lib/gcc/arm-none-eabi/10.3.1/../../../../arm-none-eabi/lib/thumb/v6-m/nofp/libc_nano.a(lib_a-exit.o) (_exit)

Discarded input sections

 .text          0x0000000000000000        0x0 /opt/st/stm32cubeide_1.9.0/plugins/com.st.stm32cube.ide.mcu.externaltools.gnu-tools-for-stm32.10.3-2021.10.linux64_1.0.0.202111181127/tools/bin/../lib/gcc/arm-none-eabi/10.3.1/thumb/v6-m/nofp/crti.o
 .data          0x0000000000000000        0x0 /opt/st/stm32cubeide_1.9.0/plugins/com.st.stm32cube.ide.mcu.externaltools.gnu-tools-for-stm32.10.3-2021.10.linux64_1.0.0.202111181127/tools/bin/../lib/gcc/arm-none-eabi/10.3.1/thumb/v6-m/nofp/crti.o
 .bss           0x0000000000000000        0x0 /opt/st/stm32cubeide_1.9.0/plugins/com.st.stm32cube.ide.mcu.externaltools.gnu-tools-for-stm32.10.3-2021.10.linux64_1.0.0.202111181127/tools/bin/../lib/gcc/arm-none-eabi/10.3.1/thumb/v6-m/nofp/crti.o
 .data          0x0000000000000000        0x4 /opt/st/stm32cubeide_1.9.0/plugins/com.st.stm32cube.ide.mcu.externaltools.gnu-tools-for-stm32.10.3-2021.10.linux64_1.0.0.202111181127/tools/bin/../lib/gcc/arm-none-eabi/10.3.1/thumb/v6-m/nofp/crtbegin.o
 .rodata        0x0000000000000000       0x24 /opt/st/stm32cubeide_1.9.0/plugins/com.st.stm32cube.ide.mcu.externaltools.gnu-tools-for-stm32.10.3-2021.10.linux64_1.0.0.202111181127/tools/bin/../lib/gcc/arm-none-eabi/10.3.1/thumb/v6-m/nofp/crtbegin.o
 .text          0x0000000000000000       0x80 /opt/st/stm32cubeide_1.9.0/plugins/com.st.stm32cube.ide.mcu.externaltools.gnu-tools-for-stm32.10.3-2021.10.linux64_1.0.0.202111181127/tools/bin/../lib/gcc/arm-none-eabi/10.3.1/../../../../arm-none-eabi/lib/thumb/v6-m/nofp/crt0.o
 .data          0x0000000000000000        0x0 /opt/st/stm32cubeide_1.9.0/plugins/com.st.stm32cube.ide.mcu.externaltools.gnu-tools-for-stm32.10.3-2021.10.linux64_1.0.0.202111181127/tools/bin/../lib/gcc/arm-none-eabi/10.3.1/../../../../arm-none-eabi/lib/thumb/v6-m/nofp/crt0.o
 .bss           0x0000000000000000        0x0 /opt/st/stm32cubeide_1.9.0/plugins/com.st.stm32cube.ide.mcu.externaltools.gnu-tools-for-stm32.10.3-2021.10.linux64_1.0.0.202111181127/tools/bin/../lib/gcc/arm-none-eabi/10.3.1/../../../../arm-none-eabi/lib/thumb/v6-m/nofp/crt0.o
 .ARM.extab     0x0000000000000000        0x0 /opt/st/stm32cubeide_1.9.0/plugins/com.st.stm32cube.ide.mcu.externaltools.gnu-tools-for-stm32.10.3-2021.10.linux64_1.0.0.202111181127/tools/bin/../lib/gcc/arm-none-eabi/10.3.1/../../../../arm-none-eabi/lib/thumb/v6-m/nofp/crt0.o
 .ARM.exidx     0x0000000000000000       0x10 /opt/st/stm32cubeide_1.9.0/plugins/com.st.stm32cube.ide.mcu.externaltools.gnu-tools-for-stm32.10.3-2021.10.linux64_1.0.0.202111181127/tools/bin/../lib/gcc/arm-none-eabi/10.3.1/../../../../arm-none-eabi/lib/thumb/v6-m/nofp/crt0.o
 .ARM.attributes
                0x0000000000000000       0x1b /opt/st/stm32cubeide_1.9.0/plugins/com.st.stm32cube.ide.mcu.externaltools.gnu-tools-for-stm32.10.3-2021.10.linux64_1.0.0.202111181127/tools/bin/../lib/gcc/arm-none-eabi/10.3.1/../../../../arm-none-eabi/lib/thumb/v6-m/nofp/crt0.o
 .group         0x0000000000000000        0xc ./App/Aquaponics/aquaponics.o
 .group         0x0000000000000000        0xc ./App/Aquaponics/aquaponics.o
 .group         0x0000000000000000        0xc ./App/Aquaponics/aquaponics.o
 .group         0x0000000000000000        0xc ./App/Aquaponics/aquaponics.o
 .group         0x0000000000000000        0xc ./App/Aquaponics/aquaponics.o
 .group         0x0000000000000000        0xc ./App/Aquaponics/aquaponics.o
Memory Configuration

Name             Origin             Length             Attributes
RAM              0x0000000020000000 0x0000000000005000 xrw
FLASH            0x0000000008000000 0x0000000000030000 xr
*default*        0x0000000000000000 0xffffffffffffffff

Linker script and memory map

LOAD /opt/st/stm32cubeide_1.9.0/plugins/com.st.stm32cube.ide.mcu.externaltools.gnu-tools-for-stm32.10.3-2021.10.linux64_1.0.0.202111181127/tools/bin/../lib/gcc/arm-none-eabi/10.3.1/thumb/v6-m/nofp/crti.o
LOAD /opt/st/stm32cubeide_1.9.0/plugins/com.st.stm32cube.ide.mcu.externaltools.gnu-tools-for-stm32.10.3-2021.10.linux64_1.0.0.202111181127/tools/bin/../lib/gcc/arm-none-eabi/10.3.1/thumb/v6-m/nofp/crtbegin.o
LOAD /opt/st/stm32cubeide_1.9.0/plugins/com.st.stm32cube.ide.mcu.externaltools.gnu-tools-for-stm32.10.3-2021.10.linux64_1.0.0.202111181127/tools/bin/../lib/gcc/arm-none-eabi/10.3.1/../../../../arm-none-eabi/lib/thumb/v6-m/nofp/crt0.o
LOAD ./App/Aquaponics/aquaponics.o
LOAD ./App/Aquaponics/i2c.o
LOAD ./App/Aquaponics/timer.o
LOAD ./App/Core/Src/mlm32l0xx_hal_msp.o
LOAD ./App/Core/Src/mlm32l0xx_hw.o
LOAD ./App/Core/Src/mlm32l0xx_it.o
LOAD ./App/LoRaWAN/src/debug.o
LOAD ./App/LoRaWAN/src/hw_gpio.o
LOAD ./App/LoRaWAN/src/hw_rtc.o
LOAD ./App/LoRaWAN/src/hw_spi.o
LOAD ./App/LoRaWAN/src/main.o
LOAD ./App/LoRaWAN/src/vcom.o
LOAD ./App/Startup/startup_stm32l072czyx.o
LOAD ./Drivers/BSP/B-L072Z-LRWAN1/b-l072z-lrwan1.o
LOAD ./Drivers/BSP/CMWX1ZZABZ-0xx/mlm32l07x01.o
LOAD ./Drivers/BSP/Components/sx1276/sx1276.o
LOAD ./Drivers/CMSIS/Device/ST/STM32L0xx/Source/system_stm32l0xx.o
LOAD ./Drivers/Middlewares/LoRaWAN/Crypto/aes.o
LOAD ./Drivers/Middlewares/LoRaWAN/Crypto/cmac.o
LOAD ./Drivers/Middlewares/LoRaWAN/Crypto/soft-se.o
LOAD ./Drivers/Middlewares/LoRaWAN/Mac/LoRaMac.o
LOAD ./Drivers/Middlewares/LoRaWAN/Mac/LoRaMacAdr.o
LOAD ./Drivers/Middlewares/LoRaWAN/Mac/LoRaMacClassB.o
LOAD ./Drivers/Middlewares/LoRaWAN/Mac/LoRaMacCommands.o
LOAD ./Drivers/Middlewares/LoRaWAN/Mac/LoRaMacConfirmQueue.o
LOAD ./Drivers/Middlewares/LoRaWAN/Mac/LoRaMacCrypto.o
LOAD ./Drivers/Middlewares/LoRaWAN/Mac/LoRaMacParser.o
LOAD ./Drivers/Middlewares/LoRaWAN/Mac/LoRaMacSerializer.o
LOAD ./Drivers/Middlewares/LoRaWAN/Mac/region/Region.o
LOAD ./Drivers/Middlewares/LoRaWAN/Mac/region/RegionAS923.o
LOAD ./Drivers/Middlewares/LoRaWAN/Mac/region/RegionAU915.o
LOAD ./Drivers/Middlewares/LoRaWAN/Mac/region/RegionCN470.o
LOAD ./Drivers/Middlewares/LoRaWAN/Mac/region/RegionCN779.o
LOAD ./Drivers/Middlewares/LoRaWAN/Mac/region/RegionCommon.o
LOAD ./Drivers/Middlewares/LoRaWAN/Mac/region/RegionEU433.o
LOAD ./Drivers/Middlewares/LoRaWAN/Mac/region/RegionEU868.o
LOAD ./Drivers/Middlewares/LoRaWAN/Mac/region/RegionIN865.o
LOAD ./Drivers/Middlewares/LoRaWAN/Mac/region/RegionKR920.o
LOAD ./Drivers/Middlewares/LoRaWAN/Mac/region/RegionRU864.o
LOAD ./Drivers/Middlewares/LoRaWAN/Mac/region/RegionUS915.o
LOAD ./Drivers/Middlewares/LoRaWAN/Patterns/Basic/lora-test.o
LOAD ./Drivers/Middlewares/LoRaWAN/Patterns/Basic/lora.o
LOAD ./Drivers/Middlewares/LoRaWAN/Utilities/low_power_manager.o
LOAD ./Drivers/Middlewares/LoRaWAN/Utilities/queue.o
LOAD ./Drivers/Middlewares/LoRaWAN/Utilities/systime.o
LOAD ./Drivers/Middlewares/LoRaWAN/Utilities/timeServer.o
LOAD ./Drivers/Middlewares/LoRaWAN/Utilities/trace.o
LOAD ./Drivers/Middlewares/LoRaWAN/Utilities/utilities.o
LOAD ./Drivers/STM32L0xx_HAL_Driver/Src/stm32l0xx_hal.o
LOAD ./Drivers/STM32L0xx_HAL_Driver/Src/stm32l0xx_hal_adc.o
LOAD ./Drivers/STM32L0xx_HAL_Driver/Src/stm32l0xx_hal_adc_ex.o
LOAD ./Drivers/STM32L0xx_HAL_Driver/Src/stm32l0xx_hal_comp.o
LOAD ./Drivers/STM32L0xx_HAL_Driver/Src/stm32l0xx_hal_comp_ex.o
LOAD ./Drivers/STM32L0xx_HAL_Driver/Src/stm32l0xx_hal_cortex.o
LOAD ./Drivers/STM32L0xx_HAL_Driver/Src/stm32l0xx_hal_crc.o
LOAD ./Drivers/STM32L0xx_HAL_Driver/Src/stm32l0xx_hal_crc_ex.o
LOAD ./Drivers/STM32L0xx_HAL_Driver/Src/stm32l0xx_hal_cryp.o
LOAD ./Drivers/STM32L0xx_HAL_Driver/Src/stm32l0xx_hal_cryp_ex.o
LOAD ./Drivers/STM32L0xx_HAL_Driver/Src/stm32l0xx_hal_dac.o
LOAD ./Drivers/STM32L0xx_HAL_Driver/Src/stm32l0xx_hal_dac_ex.o
LOAD ./Drivers/STM32L0xx_HAL_Driver/Src/stm32l0xx_hal_dma.o
LOAD ./Drivers/STM32L0xx_HAL_Driver/Src/stm32l0xx_hal_firewall.o
LOAD ./Drivers/STM32L0xx_HAL_Driver/Src/stm32l0xx_hal_flash.o
LOAD ./Drivers/STM32L0xx_HAL_Driver/Src/stm32l0xx_hal_flash_ex.o
LOAD ./Drivers/STM32L0xx_HAL_Driver/Src/stm32l0xx_hal_flash_ramfunc.o
LOAD ./Drivers/STM32L0xx_HAL_Driver/Src/stm32l0xx_hal_gpio.o
LOAD ./Drivers/STM32L0xx_HAL_Driver/Src/stm32l0xx_hal_i2c.o
LOAD ./Drivers/STM32L0xx_HAL_Driver/Src/stm32l0xx_hal_i2c_ex.o
LOAD ./Drivers/STM32L0xx_HAL_Driver/Src/stm32l0xx_hal_i2s.o
LOAD ./Drivers/STM32L0xx_HAL_Driver/Src/stm32l0xx_hal_irda.o
LOAD ./Drivers/STM32L0xx_HAL_Driver/Src/stm32l0xx_hal_iwdg.o
LOAD ./Drivers/STM32L0xx_HAL_Driver/Src/stm32l0xx_hal_lcd.o
LOAD ./Drivers/STM32L0xx_HAL_Driver/Src/stm32l0xx_hal_lptim.o
LOAD ./Drivers/STM32L0xx_HAL_Driver/Src/stm32l0xx_hal_pcd.o
LOAD ./Drivers/STM32L0xx_HAL_Driver/Src/stm32l0xx_hal_pcd_ex.o
LOAD ./Drivers/STM32L0xx_HAL_Driver/Src/stm32l0xx_hal_pwr.o
LOAD ./Drivers/STM32L0xx_HAL_Driver/Src/stm32l0xx_hal_pwr_ex.o
LOAD ./Drivers/STM32L0xx_HAL_Driver/Src/stm32l0xx_hal_rcc.o
LOAD ./Drivers/STM32L0xx_HAL_Driver/Src/stm32l0xx_hal_rcc_ex.o
LOAD ./Drivers/STM32L0xx_HAL_Driver/Src/stm32l0xx_hal_rng.o
LOAD ./Drivers/STM32L0xx_HAL_Driver/Src/stm32l0xx_hal_rtc.o
LOAD ./Drivers/STM32L0xx_HAL_Driver/Src/stm32l0xx_hal_rtc_ex.o
LOAD ./Drivers/STM32L0xx_HAL_Driver/Src/stm32l0xx_hal_smartcard.o
LOAD ./Drivers/STM32L0xx_HAL_Driver/Src/stm32l0xx_hal_smartcard_ex.o
LOAD ./Drivers/STM32L0xx_HAL_Driver/Src/stm32l0xx_hal_smbus.o
LOAD ./Drivers/STM32L0xx_HAL_Driver/Src/stm32l0xx_hal_spi.o
LOAD ./Drivers/STM32L0xx_HAL_Driver/Src/stm32l0xx_hal_tim.o
LOAD ./Drivers/STM32L0xx_HAL_Driver/Src/stm32l0xx_hal_tim_ex.o
LOAD ./Drivers/STM32L0xx_HAL_Driver/Src/stm32l0xx_hal_tsc.o
LOAD ./Drivers/STM32L0xx_HAL_Driver/Src/stm32l0xx_hal_uart.o
LOAD ./Drivers/STM32L0xx_HAL_Driver/Src/stm32l0xx_hal_uart_ex.o
LOAD ./Drivers/STM32L0xx_HAL_Driver/Src/stm32l0xx_hal_usart.o
LOAD ./Drivers/STM32L0xx_HAL_Driver/Src/stm32l0xx_hal_wwdg.o
LOAD ./Drivers/STM32L0xx_HAL_Driver/Src/stm32l0xx_ll_adc.o
LOAD ./Drivers/STM32L0xx_HAL_Driver/Src/stm32l0xx_ll_comp.o
LOAD ./Drivers/STM32L0xx_HAL_Driver/Src/stm32l0xx_ll_crc.o
LOAD ./Drivers/STM32L0xx_HAL_Driver/Src/stm32l0xx_ll_crs.o
LOAD ./Drivers/STM32L0xx_HAL_Driver/Src/stm32l0xx_ll_dac.o
LOAD ./Drivers/STM32L0xx_HAL_Driver/Src/stm32l0xx_ll_dma.o
LOAD ./Drivers/STM32L0xx_HAL_Driver/Src/stm32l0xx_ll_exti.o
LOAD ./Drivers/STM32L0xx_HAL_Driver/Src/stm32l0xx_ll_gpio.o
LOAD ./Drivers/STM32L0xx_HAL_Driver/Src/stm32l0xx_ll_i2c.o
LOAD ./Drivers/STM32L0xx_HAL_Driver/Src/stm32l0xx_ll_lptim.o
LOAD ./Drivers/STM32L0xx_HAL_Driver/Src/stm32l0xx_ll_lpuart.o
LOAD ./Drivers/STM32L0xx_HAL_Driver/Src/stm32l0xx_ll_pwr.o
LOAD ./Drivers/STM32L0xx_HAL_Driver/Src/stm32l0xx_ll_rcc.o
LOAD ./Drivers/STM32L0xx_HAL_Driver/Src/stm32l0xx_ll_rng.o
LOAD ./Drivers/STM32L0xx_HAL_Driver/Src/stm32l0xx_ll_rtc.o
LOAD ./Drivers/STM32L0xx_HAL_Driver/Src/stm32l0xx_ll_spi.o
LOAD ./Drivers/STM32L0xx_HAL_Driver/Src/stm32l0xx_ll_tim.o
LOAD ./Drivers/STM32L0xx_HAL_Driver/Src/stm32l0xx_ll_usart.o
LOAD ./Drivers/STM32L0xx_HAL_Driver/Src/stm32l0xx_ll_usb.o
LOAD ./Drivers/STM32L0xx_HAL_Driver/Src/stm32l0xx_ll_utils.o
START GROUP
LOAD /opt/st/stm32cubeide_1.9.0/plugins/com.st.stm32cube.ide.mcu.externaltools.gnu-tools-for-stm32.10.3-2021.10.linux64_1.0.0.202111181127/tools/bin/../lib/gcc/arm-none-eabi/10.3.1/../../../../arm-none-eabi/lib/thumb/v6-m/nofp/libc_nano.a
LOAD /opt/st/stm32cubeide_1.9.0/plugins/com.st.stm32cube.ide.mcu.externaltools.gnu-tools-for-stm32.10.3-2021.10.linux64_1.0.0.202111181127/tools/bin/../lib/gcc/arm-none-eabi/10.3.1/../../../../arm-none-eabi/lib/thumb/v6-m/nofp/libm.a
END GROUP
START GROUP
LOAD /opt/st/stm32cubeide_1.9.0/plugins/com.st.stm32cube.ide.mcu.externaltools.gnu-tools-for-stm32.10.3-2021.10.linux64_1.0.0.202111181127/tools/bin/../lib/gcc/arm-none-eabi/10.3.1/thumb/v6-m/nofp/libgcc.a
LOAD /opt/st/stm32cubeide_1.9.0/plugins/com.st.stm32cube.ide.mcu.externaltools.gnu-tools-for-stm32.10.3-2021.10.linux64_1.0.0.202111181127/tools/bin/../lib/gcc/arm-none-eabi/10.3.1/../../../../arm-none-eabi/lib/thumb/v6-m/nofp/libc_nano.a
END GROUP
START GROUP
LOAD /opt/st/stm32cubeide_1.9.0/plugins/com.st.stm32cube.ide.mcu.externaltools.gnu-tools-for-stm32.10.3-2021.10.linux64_1.0.0.202111181127/tools/bin/../lib/gcc/arm-none-eabi/10.3.1/thumb/v6-m/nofp/libgcc.a
LOAD /opt/st/stm32cubeide_1.9.0/plugins/com.st.stm32cube.ide.mcu.externaltools.gnu-tools-for-stm32.10.3-2021.10.linux64_1.0.0.202111181127/tools/bin/../lib/gcc/arm-none-eabi/10.3.1/../../../../arm-none-eabi/lib/thumb/v6-m/nofp/libc_nano.a
LOAD /opt/st/stm32cubeide_1.9.0/plugins/com.st.stm32cube.ide.mcu.externaltools.gnu-tools-for-stm32.10.3-2021.10.linux64_1.0.0.202111181127/tools/bin/../lib/gcc/arm-none-eabi/10.3.1/../../../../arm-none-eabi/lib/thumb/v6-m/nofp/libnosys.a
END GROUP
START GROUP
LOAD /opt/st/stm32cubeide_1.9.0/plugins/com.st.stm32cube.ide.mcu.externaltools.gnu-tools-for-stm32.10.3-2021.10.linux64_1.0.0.202111181127/tools/bin/../lib/gcc/arm-none-eabi/10.3.1/thumb/v6-m/nofp/libgcc.a
LOAD /opt/st/stm32cubeide_1.9.0/plugins/com.st.stm32cube.ide.mcu.externaltools.gnu-tools-for-stm32.10.3-2021.10.linux64_1.0.0.202111181127/tools/bin/../lib/gcc/arm-none-eabi/10.3.1/../../../../arm-none-eabi/lib/thumb/v6-m/nofp/libc_nano.a
LOAD /opt/st/stm32cubeide_1.9.0/plugins/com.st.stm32cube.ide.mcu.externaltools.gnu-tools-for-stm32.10.3-2021.10.linux64_1.0.0.202111181127/tools/bin/../lib/gcc/arm-none-eabi/10.3.1/../../../../arm-none-eabi/lib/thumb/v6-m/nofp/libnosys.a
END GROUP
LOAD /opt/st/stm32cubeide_1.9.0/plugins/com.st.stm32cube.ide.mcu.externaltools.gnu-tools-for-stm32.10.3-2021.10.linux64_1.0.0.202111181127/tools/bin/../lib/gcc/arm-none-eabi/10.3.1/thumb/v6-m/nofp/crtend.o
LOAD /opt/st/stm32cubeide_1.9.0/plugins/com.st.stm32cube.ide.mcu.externaltools.gnu-tools-for-stm32.10.3-2021.10.linux64_1.0.0.202111181127/tools/bin/../lib/gcc/arm-none-eabi/10.3.1/thumb/v6-m/nofp/crtn.o
                0x0000000020005000                _estack = (ORIGIN (RAM) + LENGTH (RAM))
                0x0000000000000200                _Min_Heap_Size = 0x200
                0x0000000000000400                _Min_Stack_Size = 0x400

.isr_vector     0x0000000008000000       0xc0
                0x0000000008000000                . = ALIGN (0x4)
 *(.isr_vector)
 .isr_vector    0x0000000008000000       0xc0 ./App/Startup/startup_stm32l072czyx.o
                0x0000000008000000                g_pfnVectors
                0x00000000080000c0                . = ALIGN (0x4)

.text           0x00000000080000c0    0x219e0
                0x00000000080000c0                . = ALIGN (0x4)
 *(.text)
 .text          0x00000000080000c0       0x48 /opt/st/stm32cubeide_1.9.0/plugins/com.st.stm32cube.ide.mcu.externaltools.gnu-tools-for-stm32.10.3-2021.10.linux64_1.0.0.202111181127/tools/bin/../lib/gcc/arm-none-eabi/10.3.1/thumb/v6-m/nofp/crtbegin.o
 .text          0x0000000008000108        0xe /opt/st/stm32cubeide_1.9.0/plugins/com.st.stm32cube.ide.mcu.externaltools.gnu-tools-for-stm32.10.3-2021.10.linux64_1.0.0.202111181127/tools/bin/../lib/gcc/arm-none-eabi/10.3.1/../../../../arm-none-eabi/lib/thumb/v6-m/nofp/libc_nano.a(lib_a-strlen.o)
                0x0000000008000108                strlen
 .text          0x0000000008000116       0x14 /opt/st/stm32cubeide_1.9.0/plugins/com.st.stm32cube.ide.mcu.externaltools.gnu-tools-for-stm32.10.3-2021.10.linux64_1.0.0.202111181127/tools/bin/../lib/gcc/arm-none-eabi/10.3.1/../../../../arm-none-eabi/lib/thumb/v6-m/nofp/libc_nano.a(lib_a-strcmp.o)
                0x0000000008000116                strcmp
 *fill*         0x000000000800012a        0x2 
 .text          0x000000000800012c       0x14 /opt/st/stm32cubeide_1.9.0/plugins/com.st.stm32cube.ide.mcu.externaltools.gnu-tools-for-stm32.10.3-2021.10.linux64_1.0.0.202111181127/tools/bin/../lib/gcc/arm-none-eabi/10.3.1/thumb/v6-m/nofp/libgcc.a(_thumb1_case_uqi.o)
                0x000000000800012c                __gnu_thumb1_case_uqi
 .text          0x0000000008000140       0x14 /opt/st/stm32cubeide_1.9.0/plugins/com.st.stm32cube.ide.mcu.externaltools.gnu-tools-for-stm32.10.3-2021.10.linux64_1.0.0.202111181127/tools/bin/../lib/gcc/arm-none-eabi/10.3.1/thumb/v6-m/nofp/libgcc.a(_thumb1_case_shi.o)
                0x0000000008000140                __gnu_thumb1_case_shi
 .text          0x0000000008000154      0x114 /opt/st/stm32cubeide_1.9.0/plugins/com.st.stm32cube.ide.mcu.externaltools.gnu-tools-for-stm32.10.3-2021.10.linux64_1.0.0.202111181127/tools/bin/../lib/gcc/arm-none-eabi/10.3.1/thumb/v6-m/nofp/libgcc.a(_udivsi3.o)
                0x0000000008000154                __udivsi3
                0x0000000008000154                __aeabi_uidiv
                0x0000000008000260                __aeabi_uidivmod
 .text          0x0000000008000268      0x1d4 /opt/st/stm32cubeide_1.9.0/plugins/com.st.stm32cube.ide.mcu.externaltools.gnu-tools-for-stm32.10.3-2021.10.linux64_1.0.0.202111181127/tools/bin/../lib/gcc/arm-none-eabi/10.3.1/thumb/v6-m/nofp/libgcc.a(_divsi3.o)
                0x0000000008000268                __aeabi_idiv
                0x0000000008000268                __divsi3
                0x0000000008000434                __aeabi_idivmod
 .text          0x000000000800043c        0x4 /opt/st/stm32cubeide_1.9.0/plugins/com.st.stm32cube.ide.mcu.externaltools.gnu-tools-for-stm32.10.3-2021.10.linux64_1.0.0.202111181127/tools/bin/../lib/gcc/arm-none-eabi/10.3.1/thumb/v6-m/nofp/libgcc.a(_dvmd_tls.o)
                0x000000000800043c                __aeabi_ldiv0
                0x000000000800043c                __aeabi_idiv0
 .text          0x0000000008000440       0x7c /opt/st/stm32cubeide_1.9.0/plugins/com.st.stm32cube.ide.mcu.externaltools.gnu-tools-for-stm32.10.3-2021.10.linux64_1.0.0.202111181127/tools/bin/../lib/gcc/arm-none-eabi/10.3.1/thumb/v6-m/nofp/libgcc.a(_arm_cmpdf2.o)
                0x0000000008000440                __aeabi_cdrcmple
                0x0000000008000450                __aeabi_cdcmple
                0x0000000008000450                __aeabi_cdcmpeq
                0x0000000008000460                __aeabi_dcmpeq
                0x000000000800046c                __aeabi_dcmplt
                0x0000000008000480                __aeabi_dcmple
                0x0000000008000494                __aeabi_dcmpgt
                0x00000000080004a8                __aeabi_dcmpge
 .text          0x00000000080004bc       0x74 /opt/st/stm32cubeide_1.9.0/plugins/com.st.stm32cube.ide.mcu.externaltools.gnu-tools-for-stm32.10.3-2021.10.linux64_1.0.0.202111181127/tools/bin/../lib/gcc/arm-none-eabi/10.3.1/thumb/v6-m/nofp/libgcc.a(_arm_cmpsf2.o)
                0x00000000080004bc                __aeabi_cfrcmple
                0x00000000080004c4                __aeabi_cfcmple
                0x00000000080004c4                __aeabi_cfcmpeq
                0x00000000080004d4                __aeabi_fcmpeq
                0x00000000080004e0                __aeabi_fcmplt
                0x00000000080004f4                __aeabi_fcmple
                0x0000000008000508                __aeabi_fcmpgt
                0x000000000800051c                __aeabi_fcmpge
 .text          0x0000000008000530       0x40 /opt/st/stm32cubeide_1.9.0/plugins/com.st.stm32cube.ide.mcu.externaltools.gnu-tools-for-stm32.10.3-2021.10.linux64_1.0.0.202111181127/tools/bin/../lib/gcc/arm-none-eabi/10.3.1/thumb/v6-m/nofp/libgcc.a(_aeabi_uldivmod.o)
                0x0000000008000530                __aeabi_uldivmod
 .text          0x0000000008000570       0x5c /opt/st/stm32cubeide_1.9.0/plugins/com.st.stm32cube.ide.mcu.externaltools.gnu-tools-for-stm32.10.3-2021.10.linux64_1.0.0.202111181127/tools/bin/../lib/gcc/arm-none-eabi/10.3.1/thumb/v6-m/nofp/libgcc.a(_muldi3.o)
                0x0000000008000570                __aeabi_lmul
                0x0000000008000570                __muldi3
 .text          0x00000000080005cc       0x30 /opt/st/stm32cubeide_1.9.0/plugins/com.st.stm32cube.ide.mcu.externaltools.gnu-tools-for-stm32.10.3-2021.10.linux64_1.0.0.202111181127/tools/bin/../lib/gcc/arm-none-eabi/10.3.1/thumb/v6-m/nofp/libgcc.a(_fixunssfsi.o)
                0x00000000080005cc                __aeabi_f2uiz
                0x00000000080005cc                __fixunssfsi
 .text          0x00000000080005fc       0x3c /opt/st/stm32cubeide_1.9.0/plugins/com.st.stm32cube.ide.mcu.externaltools.gnu-tools-for-stm32.10.3-2021.10.linux64_1.0.0.202111181127/tools/bin/../lib/gcc/arm-none-eabi/10.3.1/thumb/v6-m/nofp/libgcc.a(_fixunsdfsi.o)
                0x00000000080005fc                __fixunsdfsi
                0x00000000080005fc                __aeabi_d2uiz
 .text          0x0000000008000638       0x3c /opt/st/stm32cubeide_1.9.0/plugins/com.st.stm32cube.ide.mcu.externaltools.gnu-tools-for-stm32.10.3-2021.10.linux64_1.0.0.202111181127/tools/bin/../lib/gcc/arm-none-eabi/10.3.1/thumb/v6-m/nofp/libgcc.a(_fixdfdi.o)
                0x0000000008000638                __aeabi_d2lz
                0x0000000008000638                __fixdfdi
 .text          0x0000000008000674       0x3c /opt/st/stm32cubeide_1.9.0/plugins/com.st.stm32cube.ide.mcu.externaltools.gnu-tools-for-stm32.10.3-2021.10.linux64_1.0.0.202111181127/tools/bin/../lib/gcc/arm-none-eabi/10.3.1/thumb/v6-m/nofp/libgcc.a(_fixunsdfdi.o)
                0x0000000008000674                __aeabi_d2ulz
                0x0000000008000674                __fixunsdfdi
 .text          0x00000000080006b0       0x2c /opt/st/stm32cubeide_1.9.0/plugins/com.st.stm32cube.ide.mcu.externaltools.gnu-tools-for-stm32.10.3-2021.10.linux64_1.0.0.202111181127/tools/bin/../lib/gcc/arm-none-eabi/10.3.1/thumb/v6-m/nofp/libgcc.a(_floatdidf.o)
                0x00000000080006b0                __floatdidf
                0x00000000080006b0                __aeabi_l2d
 .text          0x00000000080006dc      0x198 /opt/st/stm32cubeide_1.9.0/plugins/com.st.stm32cube.ide.mcu.externaltools.gnu-tools-for-stm32.10.3-2021.10.linux64_1.0.0.202111181127/tools/bin/../lib/gcc/arm-none-eabi/10.3.1/thumb/v6-m/nofp/libgcc.a(_udivmoddi4.o)
                0x00000000080006dc                __udivmoddi4
 .text          0x0000000008000874      0x33c /opt/st/stm32cubeide_1.9.0/plugins/com.st.stm32cube.ide.mcu.externaltools.gnu-tools-for-stm32.10.3-2021.10.linux64_1.0.0.202111181127/tools/bin/../lib/gcc/arm-none-eabi/10.3.1/thumb/v6-m/nofp/libgcc.a(addsf3.o)
                0x0000000008000874                __aeabi_fadd
 .text          0x0000000008000bb0      0x230 /opt/st/stm32cubeide_1.9.0/plugins/com.st.stm32cube.ide.mcu.externaltools.gnu-tools-for-stm32.10.3-2021.10.linux64_1.0.0.202111181127/tools/bin/../lib/gcc/arm-none-eabi/10.3.1/thumb/v6-m/nofp/libgcc.a(divsf3.o)
                0x0000000008000bb0                __aeabi_fdiv
 .text          0x0000000008000de0       0x4c /opt/st/stm32cubeide_1.9.0/plugins/com.st.stm32cube.ide.mcu.externaltools.gnu-tools-for-stm32.10.3-2021.10.linux64_1.0.0.202111181127/tools/bin/../lib/gcc/arm-none-eabi/10.3.1/thumb/v6-m/nofp/libgcc.a(eqsf2.o)
                0x0000000008000de0                __nesf2
                0x0000000008000de0                __eqsf2
 .text          0x0000000008000e2c       0x8c /opt/st/stm32cubeide_1.9.0/plugins/com.st.stm32cube.ide.mcu.externaltools.gnu-tools-for-stm32.10.3-2021.10.linux64_1.0.0.202111181127/tools/bin/../lib/gcc/arm-none-eabi/10.3.1/thumb/v6-m/nofp/libgcc.a(gesf2.o)
                0x0000000008000e2c                __gtsf2
                0x0000000008000e2c                __gesf2
 .text          0x0000000008000eb8       0x88 /opt/st/stm32cubeide_1.9.0/plugins/com.st.stm32cube.ide.mcu.externaltools.gnu-tools-for-stm32.10.3-2021.10.linux64_1.0.0.202111181127/tools/bin/../lib/gcc/arm-none-eabi/10.3.1/thumb/v6-m/nofp/libgcc.a(lesf2.o)
                0x0000000008000eb8                __lesf2
                0x0000000008000eb8                __ltsf2
 .text          0x0000000008000f40      0x24c /opt/st/stm32cubeide_1.9.0/plugins/com.st.stm32cube.ide.mcu.externaltools.gnu-tools-for-stm32.10.3-2021.10.linux64_1.0.0.202111181127/tools/bin/../lib/gcc/arm-none-eabi/10.3.1/thumb/v6-m/nofp/libgcc.a(mulsf3.o)
                0x0000000008000f40                __aeabi_fmul
 .text          0x000000000800118c      0x35c /opt/st/stm32cubeide_1.9.0/plugins/com.st.stm32cube.ide.mcu.externaltools.gnu-tools-for-stm32.10.3-2021.10.linux64_1.0.0.202111181127/tools/bin/../lib/gcc/arm-none-eabi/10.3.1/thumb/v6-m/nofp/libgcc.a(subsf3.o)
                0x000000000800118c                __aeabi_fsub
 .text          0x00000000080014e8       0x40 /opt/st/stm32cubeide_1.9.0/plugins/com.st.stm32cube.ide.mcu.externaltools.gnu-tools-for-stm32.10.3-2021.10.linux64_1.0.0.202111181127/tools/bin/../lib/gcc/arm-none-eabi/10.3.1/thumb/v6-m/nofp/libgcc.a(fixsfsi.o)
                0x00000000080014e8                __aeabi_f2iz
 .text          0x0000000008001528       0x84 /opt/st/stm32cubeide_1.9.0/plugins/com.st.stm32cube.ide.mcu.externaltools.gnu-tools-for-stm32.10.3-2021.10.linux64_1.0.0.202111181127/tools/bin/../lib/gcc/arm-none-eabi/10.3.1/thumb/v6-m/nofp/libgcc.a(floatunsisf.o)
                0x0000000008001528                __aeabi_ui2f
 .text          0x00000000080015ac      0x678 /opt/st/stm32cubeide_1.9.0/plugins/com.st.stm32cube.ide.mcu.externaltools.gnu-tools-for-stm32.10.3-2021.10.linux64_1.0.0.202111181127/tools/bin/../lib/gcc/arm-none-eabi/10.3.1/thumb/v6-m/nofp/libgcc.a(adddf3.o)
                0x00000000080015ac                __aeabi_dadd
 .text          0x0000000008001c24      0x5ec /opt/st/stm32cubeide_1.9.0/plugins/com.st.stm32cube.ide.mcu.externaltools.gnu-tools-for-stm32.10.3-2021.10.linux64_1.0.0.202111181127/tools/bin/../lib/gcc/arm-none-eabi/10.3.1/thumb/v6-m/nofp/libgcc.a(divdf3.o)
                0x0000000008001c24                __aeabi_ddiv
 .text          0x0000000008002210       0x84 /opt/st/stm32cubeide_1.9.0/plugins/com.st.stm32cube.ide.mcu.externaltools.gnu-tools-for-stm32.10.3-2021.10.linux64_1.0.0.202111181127/tools/bin/../lib/gcc/arm-none-eabi/10.3.1/thumb/v6-m/nofp/libgcc.a(eqdf2.o)
                0x0000000008002210                __eqdf2
                0x0000000008002210                __nedf2
 .text          0x0000000008002294       0xcc /opt/st/stm32cubeide_1.9.0/plugins/com.st.stm32cube.ide.mcu.externaltools.gnu-tools-for-stm32.10.3-2021.10.linux64_1.0.0.202111181127/tools/bin/../lib/gcc/arm-none-eabi/10.3.1/thumb/v6-m/nofp/libgcc.a(gedf2.o)
                0x0000000008002294                __gtdf2
                0x0000000008002294                __gedf2
 .text          0x0000000008002360       0xc8 /opt/st/stm32cubeide_1.9.0/plugins/com.st.stm32cube.ide.mcu.externaltools.gnu-tools-for-stm32.10.3-2021.10.linux64_1.0.0.202111181127/tools/bin/../lib/gcc/arm-none-eabi/10.3.1/thumb/v6-m/nofp/libgcc.a(ledf2.o)
                0x0000000008002360                __ltdf2
                0x0000000008002360                __ledf2
 .text          0x0000000008002428      0x4d8 /opt/st/stm32cubeide_1.9.0/plugins/com.st.stm32cube.ide.mcu.externaltools.gnu-tools-for-stm32.10.3-2021.10.linux64_1.0.0.202111181127/tools/bin/../lib/gcc/arm-none-eabi/10.3.1/thumb/v6-m/nofp/libgcc.a(muldf3.o)
                0x0000000008002428                __aeabi_dmul
 .text          0x0000000008002900      0x724 /opt/st/stm32cubeide_1.9.0/plugins/com.st.stm32cube.ide.mcu.externaltools.gnu-tools-for-stm32.10.3-2021.10.linux64_1.0.0.202111181127/tools/bin/../lib/gcc/arm-none-eabi/10.3.1/thumb/v6-m/nofp/libgcc.a(subdf3.o)
                0x0000000008002900                __aeabi_dsub
 .text          0x0000000008003024       0x3c /opt/st/stm32cubeide_1.9.0/plugins/com.st.stm32cube.ide.mcu.externaltools.gnu-tools-for-stm32.10.3-2021.10.linux64_1.0.0.202111181127/tools/bin/../lib/gcc/arm-none-eabi/10.3.1/thumb/v6-m/nofp/libgcc.a(unorddf2.o)
                0x0000000008003024                __aeabi_dcmpun
 .text          0x0000000008003060       0x6c /opt/st/stm32cubeide_1.9.0/plugins/com.st.stm32cube.ide.mcu.externaltools.gnu-tools-for-stm32.10.3-2021.10.linux64_1.0.0.202111181127/tools/bin/../lib/gcc/arm-none-eabi/10.3.1/thumb/v6-m/nofp/libgcc.a(fixdfsi.o)
                0x0000000008003060                __aeabi_d2iz
 .text          0x00000000080030cc       0x60 /opt/st/stm32cubeide_1.9.0/plugins/com.st.stm32cube.ide.mcu.externaltools.gnu-tools-for-stm32.10.3-2021.10.linux64_1.0.0.202111181127/tools/bin/../lib/gcc/arm-none-eabi/10.3.1/thumb/v6-m/nofp/libgcc.a(floatsidf.o)
                0x00000000080030cc                __aeabi_i2d
 .text          0x000000000800312c       0x4c /opt/st/stm32cubeide_1.9.0/plugins/com.st.stm32cube.ide.mcu.externaltools.gnu-tools-for-stm32.10.3-2021.10.linux64_1.0.0.202111181127/tools/bin/../lib/gcc/arm-none-eabi/10.3.1/thumb/v6-m/nofp/libgcc.a(floatunsidf.o)
                0x000000000800312c                __aeabi_ui2d
 .text          0x0000000008003178       0x90 /opt/st/stm32cubeide_1.9.0/plugins/com.st.stm32cube.ide.mcu.externaltools.gnu-tools-for-stm32.10.3-2021.10.linux64_1.0.0.202111181127/tools/bin/../lib/gcc/arm-none-eabi/10.3.1/thumb/v6-m/nofp/libgcc.a(extendsfdf2.o)
                0x0000000008003178                __aeabi_f2d
 .text          0x0000000008003208      0x110 /opt/st/stm32cubeide_1.9.0/plugins/com.st.stm32cube.ide.mcu.externaltools.gnu-tools-for-stm32.10.3-2021.10.linux64_1.0.0.202111181127/tools/bin/../lib/gcc/arm-none-eabi/10.3.1/thumb/v6-m/nofp/libgcc.a(truncdfsf2.o)
                0x0000000008003208                __aeabi_d2f
 .text          0x0000000008003318       0x3c /opt/st/stm32cubeide_1.9.0/plugins/com.st.stm32cube.ide.mcu.externaltools.gnu-tools-for-stm32.10.3-2021.10.linux64_1.0.0.202111181127/tools/bin/../lib/gcc/arm-none-eabi/10.3.1/thumb/v6-m/nofp/libgcc.a(_clzsi2.o)
                0x0000000008003318                __clzsi2
 .text          0x0000000008003354       0x18 /opt/st/stm32cubeide_1.9.0/plugins/com.st.stm32cube.ide.mcu.externaltools.gnu-tools-for-stm32.10.3-2021.10.linux64_1.0.0.202111181127/tools/bin/../lib/gcc/arm-none-eabi/10.3.1/thumb/v6-m/nofp/libgcc.a(_clzdi2.o)
                0x0000000008003354                __clzdi2
 *(.text*)
 .text.delay    0x000000000800336c       0x34 ./App/Aquaponics/aquaponics.o
                0x000000000800336c                delay
 .text.Set_Pin_Output
                0x00000000080033a0       0x46 ./App/Aquaponics/aquaponics.o
                0x00000000080033a0                Set_Pin_Output
 .text.Set_Pin_Input
                0x00000000080033e6       0x46 ./App/Aquaponics/aquaponics.o
                0x00000000080033e6                Set_Pin_Input
 .text.DS18B20_Start
                0x000000000800342c       0x74 ./App/Aquaponics/aquaponics.o
                0x000000000800342c                DS18B20_Start
 .text.DS18B20_Write
                0x00000000080034a0       0x9c ./App/Aquaponics/aquaponics.o
                0x00000000080034a0                DS18B20_Write
 .text.DS18B20_Read
                0x000000000800353c       0x8c ./App/Aquaponics/aquaponics.o
                0x000000000800353c                DS18B20_Read
 .text.dataTemp
                0x00000000080035c8       0xcc ./App/Aquaponics/aquaponics.o
                0x00000000080035c8                dataTemp
 .text.getWaterLevel_Low
                0x0000000008003694       0x28 ./App/Aquaponics/aquaponics.o
                0x0000000008003694                getWaterLevel_Low
 .text.getWaterLevel_High
                0x00000000080036bc       0x2c ./App/Aquaponics/aquaponics.o
                0x00000000080036bc                getWaterLevel_High
 .text.waterLevel
                0x00000000080036e8       0x58 ./App/Aquaponics/aquaponics.o
                0x00000000080036e8                waterLevel
 .text.downlinkRectification
                0x0000000008003740      0x1b4 ./App/Aquaponics/aquaponics.o
                0x0000000008003740                downlinkRectification
 .text.aquaponicsGPIOinit
                0x00000000080038f4       0x78 ./App/Aquaponics/aquaponics.o
                0x00000000080038f4                aquaponicsGPIOinit
 .text.pH_test  0x000000000800396c      0x174 ./App/Aquaponics/aquaponics.o
                0x000000000800396c                pH_test
 .text.flowSensorInterruptEnable
                0x0000000008003ae0       0x58 ./App/Aquaponics/aquaponics.o
                0x0000000008003ae0                flowSensorInterruptEnable
 .text.waterPulseCount
                0x0000000008003b38       0x30 ./App/Aquaponics/aquaponics.o
                0x0000000008003b38                waterPulseCount
 .text.flowSensor
                0x0000000008003b68       0xd4 ./App/Aquaponics/aquaponics.o
                0x0000000008003b68                flowSensor
 .text.electricalConductivity
                0x0000000008003c3c      0x288 ./App/Aquaponics/aquaponics.o
                0x0000000008003c3c                electricalConductivity
 .text.dissolvedOxygen
                0x0000000008003ec4       0x84 ./App/Aquaponics/aquaponics.o
                0x0000000008003ec4                dissolvedOxygen
 .text.readDO   0x0000000008003f48       0x60 ./App/Aquaponics/aquaponics.o
                0x0000000008003f48                readDO
 .text.aquaponicsInit
                0x0000000008003fa8       0x1a ./App/Aquaponics/aquaponics.o
                0x0000000008003fa8                aquaponicsInit
 *fill*         0x0000000008003fc2        0x2 
 .text.readSystemParameters
                0x0000000008003fc4       0x60 ./App/Aquaponics/aquaponics.o
                0x0000000008003fc4                readSystemParameters
 .text.MX_I2C1_Init
                0x0000000008004024       0x80 ./App/Aquaponics/i2c.o
                0x0000000008004024                MX_I2C1_Init
 .text.HAL_I2C_MspInit
                0x00000000080040a4       0x8c ./App/Aquaponics/i2c.o
                0x00000000080040a4                HAL_I2C_MspInit
 .text.MX_TIM6_Init
                0x0000000008004130       0x78 ./App/Aquaponics/timer.o
                0x0000000008004130                MX_TIM6_Init
 .text.HAL_TIM_Base_MspInit
                0x00000000080041a8       0x30 ./App/Aquaponics/timer.o
                0x00000000080041a8                HAL_TIM_Base_MspInit
 .text.HAL_InitTick
                0x00000000080041d8       0x12 ./App/Core/Src/mlm32l0xx_hal_msp.o
                0x00000000080041d8                HAL_InitTick
 .text.HAL_Delay
                0x00000000080041ea       0x18 ./App/Core/Src/mlm32l0xx_hal_msp.o
                0x00000000080041ea                HAL_Delay
 *fill*         0x0000000008004202        0x2 
 .text.HAL_MspInit
                0x0000000008004204       0x48 ./App/Core/Src/mlm32l0xx_hal_msp.o
                0x0000000008004204                HAL_MspInit
 .text.HAL_RTC_MspInit
                0x000000000800424c       0x98 ./App/Core/Src/mlm32l0xx_hal_msp.o
                0x000000000800424c                HAL_RTC_MspInit
 .text.HAL_RTC_AlarmAEventCallback
                0x00000000080042e4       0x14 ./App/Core/Src/mlm32l0xx_hal_msp.o
                0x00000000080042e4                HAL_RTC_AlarmAEventCallback
 .text.HAL_GPIO_EXTI_Callback
                0x00000000080042f8       0x1e ./App/Core/Src/mlm32l0xx_hal_msp.o
                0x00000000080042f8                HAL_GPIO_EXTI_Callback
 .text.MSP_GetIRQn
                0x0000000008004316       0x38 ./App/Core/Src/mlm32l0xx_hal_msp.o
                0x0000000008004316                MSP_GetIRQn
 *fill*         0x000000000800434e        0x2 
 .text.HW_Init  0x0000000008004350       0x58 ./App/Core/Src/mlm32l0xx_hw.o
                0x0000000008004350                HW_Init
 .text.HW_GpioInit
                0x00000000080043a8      0x110 ./App/Core/Src/mlm32l0xx_hw.o
                0x00000000080043a8                HW_GpioInit
 .text.SystemClock_Config
                0x00000000080044b8       0xdc ./App/Core/Src/mlm32l0xx_hw.o
                0x00000000080044b8                SystemClock_Config
 .text.HW_GetRandomSeed
                0x0000000008004594       0x28 ./App/Core/Src/mlm32l0xx_hw.o
                0x0000000008004594                HW_GetRandomSeed
 .text.HW_GetUniqueId
                0x00000000080045bc       0xa4 ./App/Core/Src/mlm32l0xx_hw.o
                0x00000000080045bc                HW_GetUniqueId
 .text.HW_GetTemperatureLevel
                0x0000000008004660       0xbc ./App/Core/Src/mlm32l0xx_hw.o
                0x0000000008004660                HW_GetTemperatureLevel
 .text.HW_GetBatteryLevel
                0x000000000800471c       0x5c ./App/Core/Src/mlm32l0xx_hw.o
                0x000000000800471c                HW_GetBatteryLevel
 .text.HW_AdcInit
                0x0000000008004778       0xa8 ./App/Core/Src/mlm32l0xx_hw.o
                0x0000000008004778                HW_AdcInit
 .text.HW_AdcReadChannel
                0x0000000008004820       0xfc ./App/Core/Src/mlm32l0xx_hw.o
                0x0000000008004820                HW_AdcReadChannel
 .text.NMI_Handler
                0x000000000800491c        0xa ./App/Core/Src/mlm32l0xx_it.o
                0x000000000800491c                NMI_Handler
 .text.HardFault_Handler
                0x0000000008004926        0x8 ./App/Core/Src/mlm32l0xx_it.o
                0x0000000008004926                HardFault_Handler
 .text.SVC_Handler
                0x000000000800492e        0xa ./App/Core/Src/mlm32l0xx_it.o
                0x000000000800492e                SVC_Handler
 .text.PendSV_Handler
                0x0000000008004938        0xa ./App/Core/Src/mlm32l0xx_it.o
                0x0000000008004938                PendSV_Handler
 .text.SysTick_Handler
                0x0000000008004942        0xe ./App/Core/Src/mlm32l0xx_it.o
                0x0000000008004942                SysTick_Handler
 .text.USART2_IRQHandler
                0x0000000008004950        0xe ./App/Core/Src/mlm32l0xx_it.o
                0x0000000008004950                USART2_IRQHandler
 .text.DMA1_Channel4_5_6_7_IRQHandler
                0x000000000800495e        0xe ./App/Core/Src/mlm32l0xx_it.o
                0x000000000800495e                DMA1_Channel4_5_6_7_IRQHandler
 .text.RTC_IRQHandler
                0x000000000800496c        0xe ./App/Core/Src/mlm32l0xx_it.o
                0x000000000800496c                RTC_IRQHandler
 .text.EXTI0_1_IRQHandler
                0x000000000800497a       0x16 ./App/Core/Src/mlm32l0xx_it.o
                0x000000000800497a                EXTI0_1_IRQHandler
 .text.EXTI2_3_IRQHandler
                0x0000000008004990       0x16 ./App/Core/Src/mlm32l0xx_it.o
                0x0000000008004990                EXTI2_3_IRQHandler
 .text.EXTI4_15_IRQHandler
                0x00000000080049a6       0x72 ./App/Core/Src/mlm32l0xx_it.o
                0x00000000080049a6                EXTI4_15_IRQHandler
 .text.DBG_Init
                0x0000000008004a18       0xb4 ./App/LoRaWAN/src/debug.o
                0x0000000008004a18                DBG_Init
 .text.Error_Handler
                0x0000000008004acc       0x14 ./App/LoRaWAN/src/debug.o
                0x0000000008004acc                Error_Handler
 .text.HW_GPIO_Init
                0x0000000008004ae0       0xec ./App/LoRaWAN/src/hw_gpio.o
                0x0000000008004ae0                HW_GPIO_Init
 .text.HW_GPIO_SetIrq
                0x0000000008004bcc       0x78 ./App/LoRaWAN/src/hw_gpio.o
                0x0000000008004bcc                HW_GPIO_SetIrq
 .text.HW_GPIO_IrqHandler
                0x0000000008004c44       0x40 ./App/LoRaWAN/src/hw_gpio.o
                0x0000000008004c44                HW_GPIO_IrqHandler
 .text.HW_GPIO_Write
                0x0000000008004c84       0x2a ./App/LoRaWAN/src/hw_gpio.o
                0x0000000008004c84                HW_GPIO_Write
 *fill*         0x0000000008004cae        0x2 
 .text.HW_GPIO_GetBitPos
                0x0000000008004cb0       0x90 ./App/LoRaWAN/src/hw_gpio.o
 .text.LL_RTC_TIME_GetSubSecond
                0x0000000008004d40       0x18 ./App/LoRaWAN/src/hw_rtc.o
 .text.HW_RTC_Init
                0x0000000008004d58       0x30 ./App/LoRaWAN/src/hw_rtc.o
                0x0000000008004d58                HW_RTC_Init
 .text.HW_RTC_SetConfig
                0x0000000008004d88       0xb0 ./App/LoRaWAN/src/hw_rtc.o
 .text.HW_RTC_GetMinimumTimeout
                0x0000000008004e38        0xc ./App/LoRaWAN/src/hw_rtc.o
                0x0000000008004e38                HW_RTC_GetMinimumTimeout
 .text.HW_RTC_ms2Tick
                0x0000000008004e44       0x32 ./App/LoRaWAN/src/hw_rtc.o
                0x0000000008004e44                HW_RTC_ms2Tick
 .text.HW_RTC_Tick2ms
                0x0000000008004e76       0x40 ./App/LoRaWAN/src/hw_rtc.o
                0x0000000008004e76                HW_RTC_Tick2ms
 *fill*         0x0000000008004eb6        0x2 
 .text.HW_RTC_SetAlarm
                0x0000000008004eb8       0x60 ./App/LoRaWAN/src/hw_rtc.o
                0x0000000008004eb8                HW_RTC_SetAlarm
 .text.HW_RTC_GetTimerElapsedTime
                0x0000000008004f18       0x30 ./App/LoRaWAN/src/hw_rtc.o
                0x0000000008004f18                HW_RTC_GetTimerElapsedTime
 .text.HW_RTC_GetTimerValue
                0x0000000008004f48       0x26 ./App/LoRaWAN/src/hw_rtc.o
                0x0000000008004f48                HW_RTC_GetTimerValue
 *fill*         0x0000000008004f6e        0x2 
 .text.HW_RTC_StopAlarm
                0x0000000008004f70       0x40 ./App/LoRaWAN/src/hw_rtc.o
                0x0000000008004f70                HW_RTC_StopAlarm
 .text.HW_RTC_IrqHandler
                0x0000000008004fb0       0x68 ./App/LoRaWAN/src/hw_rtc.o
                0x0000000008004fb0                HW_RTC_IrqHandler
 .text.HW_RTC_DelayMs
                0x0000000008005018       0x42 ./App/LoRaWAN/src/hw_rtc.o
                0x0000000008005018                HW_RTC_DelayMs
 *fill*         0x000000000800505a        0x2 
 .text.HW_RTC_SetTimerContext
                0x000000000800505c       0x30 ./App/LoRaWAN/src/hw_rtc.o
                0x000000000800505c                HW_RTC_SetTimerContext
 .text.HW_RTC_GetTimerContext
                0x000000000800508c       0x14 ./App/LoRaWAN/src/hw_rtc.o
                0x000000000800508c                HW_RTC_GetTimerContext
 .text.HW_RTC_SetAlarmConfig
                0x00000000080050a0       0x1c ./App/LoRaWAN/src/hw_rtc.o
 .text.HW_RTC_StartWakeUpAlarm
                0x00000000080050bc      0x2cc ./App/LoRaWAN/src/hw_rtc.o
 .text.HW_RTC_GetCalendarValue
                0x0000000008005388      0x158 ./App/LoRaWAN/src/hw_rtc.o
 .text.HW_RTC_GetCalendarTime
                0x00000000080054e0       0x54 ./App/LoRaWAN/src/hw_rtc.o
                0x00000000080054e0                HW_RTC_GetCalendarTime
 .text.HW_RTC_BKUPWrite
                0x0000000008005534       0x30 ./App/LoRaWAN/src/hw_rtc.o
                0x0000000008005534                HW_RTC_BKUPWrite
 .text.HW_RTC_BKUPRead
                0x0000000008005564       0x38 ./App/LoRaWAN/src/hw_rtc.o
                0x0000000008005564                HW_RTC_BKUPRead
 .text.HW_SPI_Init
                0x000000000800559c       0x8c ./App/LoRaWAN/src/hw_spi.o
                0x000000000800559c                HW_SPI_Init
 .text.HW_SPI_IoInit
                0x0000000008005628       0x8c ./App/LoRaWAN/src/hw_spi.o
                0x0000000008005628                HW_SPI_IoInit
 .text.HW_SPI_InOut
                0x00000000080056b4       0x30 ./App/LoRaWAN/src/hw_spi.o
                0x00000000080056b4                HW_SPI_InOut
 .text.SpiFrequency
                0x00000000080056e4       0x70 ./App/LoRaWAN/src/hw_spi.o
 .text.main     0x0000000008005754       0xfc ./App/LoRaWAN/src/main.o
                0x0000000008005754                main
 .text.LoraMacProcessNotify
                0x0000000008005850       0x14 ./App/LoRaWAN/src/main.o
 .text.LORA_HasJoined
                0x0000000008005864       0x10 ./App/LoRaWAN/src/main.o
 .text.Send     0x0000000008005874      0x328 ./App/LoRaWAN/src/main.o
 .text.LORA_RxData
                0x0000000008005b9c      0x1d8 ./App/LoRaWAN/src/main.o
 .text.OnTxTimerEvent
                0x0000000008005d74       0x34 ./App/LoRaWAN/src/main.o
 .text.LoraStartTx
                0x0000000008005da8       0x90 ./App/LoRaWAN/src/main.o
 .text.LORA_ConfirmClass
                0x0000000008005e38       0x4c ./App/LoRaWAN/src/main.o
 .text.LORA_TxNeeded
                0x0000000008005e84       0x24 ./App/LoRaWAN/src/main.o
 .text.OnCheckTimerEvent
                0x0000000008005ea8       0x3c ./App/LoRaWAN/src/main.o
 .text.StartTimer
                0x0000000008005ee4       0x48 ./App/LoRaWAN/src/main.o
 .text.MX_GPIO_Init
                0x0000000008005f2c       0xa4 ./App/LoRaWAN/src/main.o
 .text.LORA_GetBatteryLevel
                0x0000000008005fd0       0x8c ./App/LoRaWAN/src/main.o
 .text.bcdToDec
                0x000000000800605c       0x32 ./App/LoRaWAN/src/main.o
                0x000000000800605c                bcdToDec
 *fill*         0x000000000800608e        0x2 
 .text.Get_Time
                0x0000000008006090      0x108 ./App/LoRaWAN/src/main.o
                0x0000000008006090                Get_Time
 .text.readRTC  0x0000000008006198        0xe ./App/LoRaWAN/src/main.o
                0x0000000008006198                readRTC
 .text.OnTimerLedEvent
                0x00000000080061a6       0x16 ./App/LoRaWAN/src/main.o
 .text.vcom_Init
                0x00000000080061bc       0x60 ./App/LoRaWAN/src/vcom.o
                0x00000000080061bc                vcom_Init
 .text.vcom_Trace
                0x000000000800621c       0x28 ./App/LoRaWAN/src/vcom.o
                0x000000000800621c                vcom_Trace
 .text.HAL_UART_TxCpltCallback
                0x0000000008006244       0x1c ./App/LoRaWAN/src/vcom.o
                0x0000000008006244                HAL_UART_TxCpltCallback
 .text.vcom_DMA_TX_IRQHandler
                0x0000000008006260       0x18 ./App/LoRaWAN/src/vcom.o
                0x0000000008006260                vcom_DMA_TX_IRQHandler
 .text.vcom_IRQHandler
                0x0000000008006278       0x18 ./App/LoRaWAN/src/vcom.o
                0x0000000008006278                vcom_IRQHandler
 .text.HAL_UART_MspInit
                0x0000000008006290       0xf0 ./App/LoRaWAN/src/vcom.o
                0x0000000008006290                HAL_UART_MspInit
 .text.vcom_IoInit
                0x0000000008006380       0x98 ./App/LoRaWAN/src/vcom.o
                0x0000000008006380                vcom_IoInit
 .text.Reset_Handler
                0x0000000008006418       0x50 ./App/Startup/startup_stm32l072czyx.o
                0x0000000008006418                Reset_Handler
 .text.Default_Handler
                0x0000000008006468        0x2 ./App/Startup/startup_stm32l072czyx.o
                0x0000000008006468                TSC_IRQHandler
                0x0000000008006468                ADC1_COMP_IRQHandler
                0x0000000008006468                PVD_IRQHandler
                0x0000000008006468                I2C1_IRQHandler
                0x0000000008006468                RCC_CRS_IRQHandler
                0x0000000008006468                SPI1_IRQHandler
                0x0000000008006468                TIM6_DAC_IRQHandler
                0x0000000008006468                I2C2_IRQHandler
                0x0000000008006468                TIM3_IRQHandler
                0x0000000008006468                DMA1_Channel1_IRQHandler
                0x0000000008006468                USART4_5_IRQHandler
                0x0000000008006468                Default_Handler
                0x0000000008006468                TIM22_IRQHandler
                0x0000000008006468                TIM7_IRQHandler
                0x0000000008006468                USB_IRQHandler
                0x0000000008006468                I2C3_IRQHandler
                0x0000000008006468                SPI2_IRQHandler
                0x0000000008006468                TIM21_IRQHandler
                0x0000000008006468                WWDG_IRQHandler
                0x0000000008006468                TIM2_IRQHandler
                0x0000000008006468                DMA1_Channel2_3_IRQHandler
                0x0000000008006468                FLASH_IRQHandler
                0x0000000008006468                USART1_IRQHandler
                0x0000000008006468                RNG_LPUART1_IRQHandler
                0x0000000008006468                LPTIM1_IRQHandler
 *fill*         0x000000000800646a        0x2 
 .text.BSP_LED_Init
                0x000000000800646c       0xdc ./Drivers/BSP/B-L072Z-LRWAN1/b-l072z-lrwan1.o
                0x000000000800646c                BSP_LED_Init
 .text.BSP_LED_On
                0x0000000008006548       0x38 ./Drivers/BSP/B-L072Z-LRWAN1/b-l072z-lrwan1.o
                0x0000000008006548                BSP_LED_On
 .text.BSP_LED_Off
                0x0000000008006580       0x38 ./Drivers/BSP/B-L072Z-LRWAN1/b-l072z-lrwan1.o
                0x0000000008006580                BSP_LED_Off
 .text.SX1276GetWakeTime
                0x00000000080065b8        0xc ./Drivers/BSP/CMWX1ZZABZ-0xx/mlm32l07x01.o
                0x00000000080065b8                SX1276GetWakeTime
 .text.SX1276SetXO
                0x00000000080065c4       0x44 ./Drivers/BSP/CMWX1ZZABZ-0xx/mlm32l07x01.o
                0x00000000080065c4                SX1276SetXO
 .text.SX1276IoInit
                0x0000000008006608       0x94 ./Drivers/BSP/CMWX1ZZABZ-0xx/mlm32l07x01.o
                0x0000000008006608                SX1276IoInit
 .text.SX1276IoIrqInit
                0x000000000800669c       0x58 ./Drivers/BSP/CMWX1ZZABZ-0xx/mlm32l07x01.o
                0x000000000800669c                SX1276IoIrqInit
 .text.SX1276IoDeInit
                0x00000000080066f4       0x68 ./Drivers/BSP/CMWX1ZZABZ-0xx/mlm32l07x01.o
                0x00000000080066f4                SX1276IoDeInit
 .text.SX1276SetRfTxPower
                0x000000000800675c      0x1c0 ./Drivers/BSP/CMWX1ZZABZ-0xx/mlm32l07x01.o
                0x000000000800675c                SX1276SetRfTxPower
 .text.SX1276GetPaSelect
                0x000000000800691c       0x24 ./Drivers/BSP/CMWX1ZZABZ-0xx/mlm32l07x01.o
                0x000000000800691c                SX1276GetPaSelect
 .text.SX1276SetAntSwLowPower
                0x0000000008006940       0x2c ./Drivers/BSP/CMWX1ZZABZ-0xx/mlm32l07x01.o
                0x0000000008006940                SX1276SetAntSwLowPower
 .text.SX1276AntSwInit
                0x000000000800696c       0x80 ./Drivers/BSP/CMWX1ZZABZ-0xx/mlm32l07x01.o
 .text.SX1276AntSwDeInit
                0x00000000080069ec       0x80 ./Drivers/BSP/CMWX1ZZABZ-0xx/mlm32l07x01.o
 .text.SX1276SetAntSw
                0x0000000008006a6c       0x74 ./Drivers/BSP/CMWX1ZZABZ-0xx/mlm32l07x01.o
                0x0000000008006a6c                SX1276SetAntSw
 .text.SX1276CheckRfFrequency
                0x0000000008006ae0       0x12 ./Drivers/BSP/CMWX1ZZABZ-0xx/mlm32l07x01.o
                0x0000000008006ae0                SX1276CheckRfFrequency
 *fill*         0x0000000008006af2        0x2 
 .text.SX1276BoardInit
                0x0000000008006af4       0x1c ./Drivers/BSP/Components/sx1276/sx1276.o
                0x0000000008006af4                SX1276BoardInit
 .text.SX1276Init
                0x0000000008006b10       0xfc ./Drivers/BSP/Components/sx1276/sx1276.o
                0x0000000008006b10                SX1276Init
 .text.SX1276GetStatus
                0x0000000008006c0c       0x14 ./Drivers/BSP/Components/sx1276/sx1276.o
                0x0000000008006c0c                SX1276GetStatus
 .text.SX1276SetChannel
                0x0000000008006c20       0x8c ./Drivers/BSP/Components/sx1276/sx1276.o
                0x0000000008006c20                SX1276SetChannel
 .text.SX1276IsChannelFree
                0x0000000008006cac       0xb8 ./Drivers/BSP/Components/sx1276/sx1276.o
                0x0000000008006cac                SX1276IsChannelFree
 .text.SX1276Random
                0x0000000008006d64       0x68 ./Drivers/BSP/Components/sx1276/sx1276.o
                0x0000000008006d64                SX1276Random
 .text.RxChainCalibration
                0x0000000008006dcc       0xf8 ./Drivers/BSP/Components/sx1276/sx1276.o
                0x0000000008006dcc                RxChainCalibration
 .text.GetFskBandwidthRegValue
                0x0000000008006ec4       0x6c ./Drivers/BSP/Components/sx1276/sx1276.o
 .text.SX1276SetRxConfig
                0x0000000008006f30      0x4e8 ./Drivers/BSP/Components/sx1276/sx1276.o
                0x0000000008006f30                SX1276SetRxConfig
 .text.SX1276SetTxConfig
                0x0000000008007418      0x444 ./Drivers/BSP/Components/sx1276/sx1276.o
                0x0000000008007418                SX1276SetTxConfig
 .text.SX1276GetTimeOnAir
                0x000000000800785c      0x314 ./Drivers/BSP/Components/sx1276/sx1276.o
                0x000000000800785c                SX1276GetTimeOnAir
 .text.SX1276Send
                0x0000000008007b70      0x180 ./Drivers/BSP/Components/sx1276/sx1276.o
                0x0000000008007b70                SX1276Send
 .text.SX1276SetSleep
                0x0000000008007cf0       0x4c ./Drivers/BSP/Components/sx1276/sx1276.o
                0x0000000008007cf0                SX1276SetSleep
 .text.SX1276SetStby
                0x0000000008007d3c       0x40 ./Drivers/BSP/Components/sx1276/sx1276.o
                0x0000000008007d3c                SX1276SetStby
 .text.SX1276SetRx
                0x0000000008007d7c      0x31c ./Drivers/BSP/Components/sx1276/sx1276.o
                0x0000000008007d7c                SX1276SetRx
 .text.SX1276SetTx
                0x0000000008008098      0x100 ./Drivers/BSP/Components/sx1276/sx1276.o
                0x0000000008008098                SX1276SetTx
 .text.SX1276StartCad
                0x0000000008008198       0x50 ./Drivers/BSP/Components/sx1276/sx1276.o
                0x0000000008008198                SX1276StartCad
 .text.SX1276SetTxContinuousWave
                0x00000000080081e8       0xc4 ./Drivers/BSP/Components/sx1276/sx1276.o
                0x00000000080081e8                SX1276SetTxContinuousWave
 .text.SX1276ReadRssi
                0x00000000080082ac       0x98 ./Drivers/BSP/Components/sx1276/sx1276.o
                0x00000000080082ac                SX1276ReadRssi
 .text.SX1276Reset
                0x0000000008008344       0x68 ./Drivers/BSP/Components/sx1276/sx1276.o
                0x0000000008008344                SX1276Reset
 .text.SX1276SetOpMode
                0x00000000080083ac       0xa0 ./Drivers/BSP/Components/sx1276/sx1276.o
                0x00000000080083ac                SX1276SetOpMode
 .text.SX1276SetModem
                0x000000000800844c       0xb4 ./Drivers/BSP/Components/sx1276/sx1276.o
                0x000000000800844c                SX1276SetModem
 .text.SX1276Write
                0x0000000008008500       0x28 ./Drivers/BSP/Components/sx1276/sx1276.o
                0x0000000008008500                SX1276Write
 .text.SX1276Read
                0x0000000008008528       0x28 ./Drivers/BSP/Components/sx1276/sx1276.o
                0x0000000008008528                SX1276Read
 .text.SX1276WriteBuffer
                0x0000000008008550       0x84 ./Drivers/BSP/Components/sx1276/sx1276.o
                0x0000000008008550                SX1276WriteBuffer
 .text.SX1276ReadBuffer
                0x00000000080085d4       0x88 ./Drivers/BSP/Components/sx1276/sx1276.o
                0x00000000080085d4                SX1276ReadBuffer
 .text.SX1276WriteFifo
                0x000000000800865c       0x24 ./Drivers/BSP/Components/sx1276/sx1276.o
                0x000000000800865c                SX1276WriteFifo
 .text.SX1276ReadFifo
                0x0000000008008680       0x24 ./Drivers/BSP/Components/sx1276/sx1276.o
                0x0000000008008680                SX1276ReadFifo
 .text.SX1276SetMaxPayloadLength
                0x00000000080086a4       0x64 ./Drivers/BSP/Components/sx1276/sx1276.o
                0x00000000080086a4                SX1276SetMaxPayloadLength
 .text.SX1276SetPublicNetwork
                0x0000000008008708       0x44 ./Drivers/BSP/Components/sx1276/sx1276.o
                0x0000000008008708                SX1276SetPublicNetwork
 .text.SX1276GetWakeupTime
                0x000000000800874c       0x1c ./Drivers/BSP/Components/sx1276/sx1276.o
                0x000000000800874c                SX1276GetWakeupTime
 .text.SX1276OnTimeoutIrq
                0x0000000008008768      0x160 ./Drivers/BSP/Components/sx1276/sx1276.o
                0x0000000008008768                SX1276OnTimeoutIrq
 .text.SX1276OnDio0Irq
                0x00000000080088c8      0x45c ./Drivers/BSP/Components/sx1276/sx1276.o
                0x00000000080088c8                SX1276OnDio0Irq
 .text.SX1276OnDio1Irq
                0x0000000008008d24      0x1ac ./Drivers/BSP/Components/sx1276/sx1276.o
                0x0000000008008d24                SX1276OnDio1Irq
 .text.SX1276OnDio2Irq
                0x0000000008008ed0      0x190 ./Drivers/BSP/Components/sx1276/sx1276.o
                0x0000000008008ed0                SX1276OnDio2Irq
 .text.SX1276OnDio3Irq
                0x0000000008009060       0x8c ./Drivers/BSP/Components/sx1276/sx1276.o
                0x0000000008009060                SX1276OnDio3Irq
 .text.SX1276OnDio4Irq
                0x00000000080090ec       0x3c ./Drivers/BSP/Components/sx1276/sx1276.o
                0x00000000080090ec                SX1276OnDio4Irq
 .text.SystemInit
                0x0000000008009128       0x7c ./Drivers/CMSIS/Device/ST/STM32L0xx/Source/system_stm32l0xx.o
                0x0000000008009128                SystemInit
 .text.copy_block
                0x00000000080091a4       0xb0 ./Drivers/Middlewares/LoRaWAN/Crypto/aes.o
 .text.copy_block_nn
                0x0000000008009254       0x38 ./Drivers/Middlewares/LoRaWAN/Crypto/aes.o
 .text.xor_block
                0x000000000800928c      0x16c ./Drivers/Middlewares/LoRaWAN/Crypto/aes.o
 .text.copy_and_key
                0x00000000080093f8      0x16e ./Drivers/Middlewares/LoRaWAN/Crypto/aes.o
 .text.add_round_key
                0x0000000008009566       0x1e ./Drivers/Middlewares/LoRaWAN/Crypto/aes.o
 .text.shift_sub_rows
                0x0000000008009584      0x144 ./Drivers/Middlewares/LoRaWAN/Crypto/aes.o
 .text.mix_sub_columns
                0x00000000080096c8      0x3cc ./Drivers/Middlewares/LoRaWAN/Crypto/aes.o
 .text.aes_set_key
                0x0000000008009a94      0x278 ./Drivers/Middlewares/LoRaWAN/Crypto/aes.o
                0x0000000008009a94                aes_set_key
 .text.aes_encrypt
                0x0000000008009d0c       0x94 ./Drivers/Middlewares/LoRaWAN/Crypto/aes.o
                0x0000000008009d0c                aes_encrypt
 .text.AES_CMAC_Init
                0x0000000008009da0       0x34 ./Drivers/Middlewares/LoRaWAN/Crypto/cmac.o
                0x0000000008009da0                AES_CMAC_Init
 .text.AES_CMAC_SetKey
                0x0000000008009dd4       0x1e ./Drivers/Middlewares/LoRaWAN/Crypto/cmac.o
                0x0000000008009dd4                AES_CMAC_SetKey
 .text.AES_CMAC_Update
                0x0000000008009df2      0x176 ./Drivers/Middlewares/LoRaWAN/Crypto/cmac.o
                0x0000000008009df2                AES_CMAC_Update
 .text.AES_CMAC_Final
                0x0000000008009f68      0x2d6 ./Drivers/Middlewares/LoRaWAN/Crypto/cmac.o
                0x0000000008009f68                AES_CMAC_Final
 *fill*         0x000000000800a23e        0x2 
 .text.GetKeyByID
                0x000000000800a240       0x7c ./Drivers/Middlewares/LoRaWAN/Crypto/soft-se.o
                0x000000000800a240                GetKeyByID
 .text.DummyCB  0x000000000800a2bc        0xa ./Drivers/Middlewares/LoRaWAN/Crypto/soft-se.o
 *fill*         0x000000000800a2c6        0x2 
 .text.ComputeCmac
                0x000000000800a2c8       0xc0 ./Drivers/Middlewares/LoRaWAN/Crypto/soft-se.o
 .text.SecureElementInit
                0x000000000800a388      0x384 ./Drivers/Middlewares/LoRaWAN/Crypto/soft-se.o
                0x000000000800a388                SecureElementInit
 .text.SecureElementRestoreNvmCtx
                0x000000000800a70c       0x30 ./Drivers/Middlewares/LoRaWAN/Crypto/soft-se.o
                0x000000000800a70c                SecureElementRestoreNvmCtx
 .text.SecureElementGetNvmCtx
                0x000000000800a73c       0x20 ./Drivers/Middlewares/LoRaWAN/Crypto/soft-se.o
                0x000000000800a73c                SecureElementGetNvmCtx
 .text.SecureElementSetKey
                0x000000000800a75c      0x114 ./Drivers/Middlewares/LoRaWAN/Crypto/soft-se.o
                0x000000000800a75c                SecureElementSetKey
 .text.SecureElementComputeAesCmac
                0x000000000800a870       0x42 ./Drivers/Middlewares/LoRaWAN/Crypto/soft-se.o
                0x000000000800a870                SecureElementComputeAesCmac
 .text.SecureElementVerifyAesCmac
                0x000000000800a8b2       0x82 ./Drivers/Middlewares/LoRaWAN/Crypto/soft-se.o
                0x000000000800a8b2                SecureElementVerifyAesCmac
 .text.SecureElementAesEncrypt
                0x000000000800a934       0xd4 ./Drivers/Middlewares/LoRaWAN/Crypto/soft-se.o
                0x000000000800a934                SecureElementAesEncrypt
 .text.SecureElementDeriveAndStoreKey
                0x000000000800aa08       0xba ./Drivers/Middlewares/LoRaWAN/Crypto/soft-se.o
                0x000000000800aa08                SecureElementDeriveAndStoreKey
 *fill*         0x000000000800aac2        0x2 
 .text.SecureElementRandomNumber
                0x000000000800aac4       0x2c ./Drivers/Middlewares/LoRaWAN/Crypto/soft-se.o
                0x000000000800aac4                SecureElementRandomNumber
 .text.SecureElementSetDevEui
                0x000000000800aaf0       0x38 ./Drivers/Middlewares/LoRaWAN/Crypto/soft-se.o
                0x000000000800aaf0                SecureElementSetDevEui
 .text.SecureElementGetDevEui
                0x000000000800ab28       0x10 ./Drivers/Middlewares/LoRaWAN/Crypto/soft-se.o
                0x000000000800ab28                SecureElementGetDevEui
 .text.SecureElementSetJoinEui
                0x000000000800ab38       0x38 ./Drivers/Middlewares/LoRaWAN/Crypto/soft-se.o
                0x000000000800ab38                SecureElementSetJoinEui
 .text.SecureElementGetJoinEui
                0x000000000800ab70       0x10 ./Drivers/Middlewares/LoRaWAN/Crypto/soft-se.o
                0x000000000800ab70                SecureElementGetJoinEui
 .text.OnRadioTxDone
                0x000000000800ab80       0x9c ./Drivers/Middlewares/LoRaWAN/Mac/LoRaMac.o
 .text.OnRadioRxDone
                0x000000000800ac1c       0xc0 ./Drivers/Middlewares/LoRaWAN/Mac/LoRaMac.o
 .text.OnRadioTxTimeout
                0x000000000800acdc       0x74 ./Drivers/Middlewares/LoRaWAN/Mac/LoRaMac.o
 .text.OnRadioRxError
                0x000000000800ad50       0x44 ./Drivers/Middlewares/LoRaWAN/Mac/LoRaMac.o
 .text.OnRadioRxTimeout
                0x000000000800ad94       0x74 ./Drivers/Middlewares/LoRaWAN/Mac/LoRaMac.o
 .text.UpdateRxSlotIdleState
                0x000000000800ae08       0x38 ./Drivers/Middlewares/LoRaWAN/Mac/LoRaMac.o
 .text.ProcessRadioTxDone
                0x000000000800ae40      0x158 ./Drivers/Middlewares/LoRaWAN/Mac/LoRaMac.o
 .text.PrepareRxDoneAbort
                0x000000000800af98       0x58 ./Drivers/Middlewares/LoRaWAN/Mac/LoRaMac.o
 .text.ProcessRadioRxDone
                0x000000000800aff0      0xa70 ./Drivers/Middlewares/LoRaWAN/Mac/LoRaMac.o
 .text.ProcessRadioTxTimeout
                0x000000000800ba60       0x6c ./Drivers/Middlewares/LoRaWAN/Mac/LoRaMac.o
 .text.HandleRadioRxErrorTimeout
                0x000000000800bacc      0x128 ./Drivers/Middlewares/LoRaWAN/Mac/LoRaMac.o
 .text.ProcessRadioRxError
                0x000000000800bbf4       0x12 ./Drivers/Middlewares/LoRaWAN/Mac/LoRaMac.o
 .text.ProcessRadioRxTimeout
                0x000000000800bc06       0x12 ./Drivers/Middlewares/LoRaWAN/Mac/LoRaMac.o
 .text.LoRaMacHandleIrqEvents
                0x000000000800bc18       0x98 ./Drivers/Middlewares/LoRaWAN/Mac/LoRaMac.o
 .text.LoRaMacIsBusy
                0x000000000800bcb0       0x30 ./Drivers/Middlewares/LoRaWAN/Mac/LoRaMac.o
                0x000000000800bcb0                LoRaMacIsBusy
 .text.LoRaMacEnableRequests
                0x000000000800bce0       0x28 ./Drivers/Middlewares/LoRaWAN/Mac/LoRaMac.o
 .text.LoRaMacHandleRequestEvents
                0x000000000800bd08       0xcc ./Drivers/Middlewares/LoRaWAN/Mac/LoRaMac.o
 .text.LoRaMacHandleScheduleUplinkEvent
                0x000000000800bdd4       0x38 ./Drivers/Middlewares/LoRaWAN/Mac/LoRaMac.o
 .text.LoRaMacHandleIndicationEvents
                0x000000000800be0c       0xb0 ./Drivers/Middlewares/LoRaWAN/Mac/LoRaMac.o
 .text.LoRaMacHandleMcpsRequest
                0x000000000800bebc      0x104 ./Drivers/Middlewares/LoRaWAN/Mac/LoRaMac.o
 .text.LoRaMacHandleMlmeRequest
                0x000000000800bfc0       0x84 ./Drivers/Middlewares/LoRaWAN/Mac/LoRaMac.o
 .text.LoRaMacCheckForBeaconAcquisition
                0x000000000800c044       0x58 ./Drivers/Middlewares/LoRaWAN/Mac/LoRaMac.o
 .text.LoRaMacCheckForRxAbort
                0x000000000800c09c       0x48 ./Drivers/Middlewares/LoRaWAN/Mac/LoRaMac.o
 .text.LoRaMacProcess
                0x000000000800c0e4       0x8c ./Drivers/Middlewares/LoRaWAN/Mac/LoRaMac.o
                0x000000000800c0e4                LoRaMacProcess
 .text.OnTxDelayedTimerEvent
                0x000000000800c170       0x8c ./Drivers/Middlewares/LoRaWAN/Mac/LoRaMac.o
 .text.OnRxWindow1TimerEvent
                0x000000000800c1fc       0x98 ./Drivers/Middlewares/LoRaWAN/Mac/LoRaMac.o
 .text.OnRxWindow2TimerEvent
                0x000000000800c294       0xa4 ./Drivers/Middlewares/LoRaWAN/Mac/LoRaMac.o
 .text.OnAckTimeoutTimerEvent
                0x000000000800c338       0x84 ./Drivers/Middlewares/LoRaWAN/Mac/LoRaMac.o
 .text.GetFCntDown
                0x000000000800c3bc       0xc4 ./Drivers/Middlewares/LoRaWAN/Mac/LoRaMac.o
 .text.SwitchClass
                0x000000000800c480      0x294 ./Drivers/Middlewares/LoRaWAN/Mac/LoRaMac.o
 .text.GetMaxAppPayloadWithoutFOptsLength
                0x000000000800c714       0x78 ./Drivers/Middlewares/LoRaWAN/Mac/LoRaMac.o
 .text.ValidatePayloadLength
                0x000000000800c78c       0x78 ./Drivers/Middlewares/LoRaWAN/Mac/LoRaMac.o
 .text.SetMlmeScheduleUplinkIndication
                0x000000000800c804       0x20 ./Drivers/Middlewares/LoRaWAN/Mac/LoRaMac.o
 .text.ProcessMacCommands
                0x000000000800c824      0xac8 ./Drivers/Middlewares/LoRaWAN/Mac/LoRaMac.o
 .text.Send     0x000000000800d2ec      0x26c ./Drivers/Middlewares/LoRaWAN/Mac/LoRaMac.o
                0x000000000800d2ec                Send
 .text.SendReJoinReq
                0x000000000800d558       0xc8 ./Drivers/Middlewares/LoRaWAN/Mac/LoRaMac.o
                0x000000000800d558                SendReJoinReq
 .text.ScheduleTx
                0x000000000800d620      0x2d4 ./Drivers/Middlewares/LoRaWAN/Mac/LoRaMac.o
 .text.SecureFrame
                0x000000000800d8f4       0xdc ./Drivers/Middlewares/LoRaWAN/Mac/LoRaMac.o
 .text.CalculateBackOff
                0x000000000800d9d0       0xe0 ./Drivers/Middlewares/LoRaWAN/Mac/LoRaMac.o
 .text.RemoveMacCommands
                0x000000000800dab0       0x50 ./Drivers/Middlewares/LoRaWAN/Mac/LoRaMac.o
 .text.ResetMacParameters
                0x000000000800db00      0x1f8 ./Drivers/Middlewares/LoRaWAN/Mac/LoRaMac.o
 .text.RxWindowSetup
                0x000000000800dcf8       0x68 ./Drivers/Middlewares/LoRaWAN/Mac/LoRaMac.o
 .text.OpenContinuousRxCWindow
                0x000000000800dd60       0x64 ./Drivers/Middlewares/LoRaWAN/Mac/LoRaMac.o
 .text.PrepareFrame
                0x000000000800ddc4      0x2a4 ./Drivers/Middlewares/LoRaWAN/Mac/LoRaMac.o
                0x000000000800ddc4                PrepareFrame
 .text.SendFrameOnChannel
                0x000000000800e068      0x1a8 ./Drivers/Middlewares/LoRaWAN/Mac/LoRaMac.o
                0x000000000800e068                SendFrameOnChannel
 .text.SetTxContinuousWave
                0x000000000800e210       0x9c ./Drivers/Middlewares/LoRaWAN/Mac/LoRaMac.o
                0x000000000800e210                SetTxContinuousWave
 .text.SetTxContinuousWave1
                0x000000000800e2ac       0x50 ./Drivers/Middlewares/LoRaWAN/Mac/LoRaMac.o
                0x000000000800e2ac                SetTxContinuousWave1
 .text.GetCtxs  0x000000000800e2fc       0xac ./Drivers/Middlewares/LoRaWAN/Mac/LoRaMac.o
                0x000000000800e2fc                GetCtxs
 .text.RestoreCtxs
                0x000000000800e3a8       0xe4 ./Drivers/Middlewares/LoRaWAN/Mac/LoRaMac.o
                0x000000000800e3a8                RestoreCtxs
 .text.DetermineFrameType
                0x000000000800e48c       0x9a ./Drivers/Middlewares/LoRaWAN/Mac/LoRaMac.o
                0x000000000800e48c                DetermineFrameType
 *fill*         0x000000000800e526        0x2 
 .text.CheckRetransUnconfirmedUplink
                0x000000000800e528       0x68 ./Drivers/Middlewares/LoRaWAN/Mac/LoRaMac.o
 .text.CheckRetransConfirmedUplink
                0x000000000800e590       0x50 ./Drivers/Middlewares/LoRaWAN/Mac/LoRaMac.o
 .text.StopRetransmission
                0x000000000800e5e0       0x98 ./Drivers/Middlewares/LoRaWAN/Mac/LoRaMac.o
 .text.AckTimeoutRetriesProcess
                0x000000000800e678       0x9c ./Drivers/Middlewares/LoRaWAN/Mac/LoRaMac.o
 .text.AckTimeoutRetriesFinalize
                0x000000000800e714       0x78 ./Drivers/Middlewares/LoRaWAN/Mac/LoRaMac.o
 .text.CallNvmCtxCallback
                0x000000000800e78c       0x44 ./Drivers/Middlewares/LoRaWAN/Mac/LoRaMac.o
 .text.EventMacNvmCtxChanged
                0x000000000800e7d0       0x10 ./Drivers/Middlewares/LoRaWAN/Mac/LoRaMac.o
 .text.EventRegionNvmCtxChanged
                0x000000000800e7e0       0x10 ./Drivers/Middlewares/LoRaWAN/Mac/LoRaMac.o
 .text.EventCryptoNvmCtxChanged
                0x000000000800e7f0       0x10 ./Drivers/Middlewares/LoRaWAN/Mac/LoRaMac.o
 .text.EventSecureElementNvmCtxChanged
                0x000000000800e800       0x10 ./Drivers/Middlewares/LoRaWAN/Mac/LoRaMac.o
 .text.EventCommandsNvmCtxChanged
                0x000000000800e810       0x10 ./Drivers/Middlewares/LoRaWAN/Mac/LoRaMac.o
 .text.EventClassBNvmCtxChanged
                0x000000000800e820       0x10 ./Drivers/Middlewares/LoRaWAN/Mac/LoRaMac.o
 .text.EventConfirmQueueNvmCtxChanged
                0x000000000800e830       0x10 ./Drivers/Middlewares/LoRaWAN/Mac/LoRaMac.o
 .text.IsRequestPending
                0x000000000800e840       0x38 ./Drivers/Middlewares/LoRaWAN/Mac/LoRaMac.o
 .text.LoRaMacInitialization
                0x000000000800e878      0x750 ./Drivers/Middlewares/LoRaWAN/Mac/LoRaMac.o
                0x000000000800e878                LoRaMacInitialization
 .text.LoRaMacStart
                0x000000000800efc8       0x1c ./Drivers/Middlewares/LoRaWAN/Mac/LoRaMac.o
                0x000000000800efc8                LoRaMacStart
 .text.LoRaMacQueryTxPossible
                0x000000000800efe4      0x15c ./Drivers/Middlewares/LoRaWAN/Mac/LoRaMac.o
                0x000000000800efe4                LoRaMacQueryTxPossible
 .text.LoRaMacMibGetRequestConfirm
                0x000000000800f140      0x2b8 ./Drivers/Middlewares/LoRaWAN/Mac/LoRaMac.o
                0x000000000800f140                LoRaMacMibGetRequestConfirm
 .text.LoRaMacMibSetRequestConfirm
                0x000000000800f3f8      0x9e8 ./Drivers/Middlewares/LoRaWAN/Mac/LoRaMac.o
                0x000000000800f3f8                LoRaMacMibSetRequestConfirm
 .text.LoRaMacMlmeRequest
                0x000000000800fde0      0x2a4 ./Drivers/Middlewares/LoRaWAN/Mac/LoRaMac.o
                0x000000000800fde0                LoRaMacMlmeRequest
 .text.LoRaMacMcpsRequest
                0x0000000008010084      0x28c ./Drivers/Middlewares/LoRaWAN/Mac/LoRaMac.o
                0x0000000008010084                LoRaMacMcpsRequest
 .text.CalcNextV10X
                0x0000000008010310      0x1aa ./Drivers/Middlewares/LoRaWAN/Mac/LoRaMacAdr.o
 .text.LoRaMacAdrCalcNext
                0x00000000080104ba       0x30 ./Drivers/Middlewares/LoRaWAN/Mac/LoRaMacAdr.o
                0x00000000080104ba                LoRaMacAdrCalcNext
 .text.LoRaMacClassBInit
                0x00000000080104ea       0x14 ./Drivers/Middlewares/LoRaWAN/Mac/LoRaMacClassB.o
                0x00000000080104ea                LoRaMacClassBInit
 .text.LoRaMacClassBRestoreNvmCtx
                0x00000000080104fe       0x12 ./Drivers/Middlewares/LoRaWAN/Mac/LoRaMacClassB.o
                0x00000000080104fe                LoRaMacClassBRestoreNvmCtx
 .text.LoRaMacClassBGetNvmCtx
                0x0000000008010510       0x18 ./Drivers/Middlewares/LoRaWAN/Mac/LoRaMacClassB.o
                0x0000000008010510                LoRaMacClassBGetNvmCtx
 .text.LoRaMacClassBSetBeaconState
                0x0000000008010528       0x14 ./Drivers/Middlewares/LoRaWAN/Mac/LoRaMacClassB.o
                0x0000000008010528                LoRaMacClassBSetBeaconState
 .text.LoRaMacClassBSetPingSlotState
                0x000000000801053c       0x14 ./Drivers/Middlewares/LoRaWAN/Mac/LoRaMacClassB.o
                0x000000000801053c                LoRaMacClassBSetPingSlotState
 .text.LoRaMacClassBSetMulticastSlotState
                0x0000000008010550       0x14 ./Drivers/Middlewares/LoRaWAN/Mac/LoRaMacClassB.o
                0x0000000008010550                LoRaMacClassBSetMulticastSlotState
 .text.LoRaMacClassBIsAcquisitionInProgress
                0x0000000008010564        0xc ./Drivers/Middlewares/LoRaWAN/Mac/LoRaMacClassB.o
                0x0000000008010564                LoRaMacClassBIsAcquisitionInProgress
 .text.LoRaMacClassBBeaconTimerEvent
                0x0000000008010570       0x10 ./Drivers/Middlewares/LoRaWAN/Mac/LoRaMacClassB.o
                0x0000000008010570                LoRaMacClassBBeaconTimerEvent
 .text.LoRaMacClassBPingSlotTimerEvent
                0x0000000008010580       0x10 ./Drivers/Middlewares/LoRaWAN/Mac/LoRaMacClassB.o
                0x0000000008010580                LoRaMacClassBPingSlotTimerEvent
 .text.LoRaMacClassBMulticastSlotTimerEvent
                0x0000000008010590       0x10 ./Drivers/Middlewares/LoRaWAN/Mac/LoRaMacClassB.o
                0x0000000008010590                LoRaMacClassBMulticastSlotTimerEvent
 .text.LoRaMacClassBRxBeacon
                0x00000000080105a0       0x18 ./Drivers/Middlewares/LoRaWAN/Mac/LoRaMacClassB.o
                0x00000000080105a0                LoRaMacClassBRxBeacon
 .text.LoRaMacClassBIsBeaconExpected
                0x00000000080105b8        0xc ./Drivers/Middlewares/LoRaWAN/Mac/LoRaMacClassB.o
                0x00000000080105b8                LoRaMacClassBIsBeaconExpected
 .text.LoRaMacClassBIsPingExpected
                0x00000000080105c4        0xc ./Drivers/Middlewares/LoRaWAN/Mac/LoRaMacClassB.o
                0x00000000080105c4                LoRaMacClassBIsPingExpected
 .text.LoRaMacClassBIsMulticastExpected
                0x00000000080105d0        0xc ./Drivers/Middlewares/LoRaWAN/Mac/LoRaMacClassB.o
                0x00000000080105d0                LoRaMacClassBIsMulticastExpected
 .text.LoRaMacClassBIsBeaconModeActive
                0x00000000080105dc        0xc ./Drivers/Middlewares/LoRaWAN/Mac/LoRaMacClassB.o
                0x00000000080105dc                LoRaMacClassBIsBeaconModeActive
 .text.LoRaMacClassBSetPingSlotInfo
                0x00000000080105e8       0x14 ./Drivers/Middlewares/LoRaWAN/Mac/LoRaMacClassB.o
                0x00000000080105e8                LoRaMacClassBSetPingSlotInfo
 .text.LoRaMacClassBHaltBeaconing
                0x00000000080105fc        0xa ./Drivers/Middlewares/LoRaWAN/Mac/LoRaMacClassB.o
                0x00000000080105fc                LoRaMacClassBHaltBeaconing
 .text.LoRaMacClassBResumeBeaconing
                0x0000000008010606        0xa ./Drivers/Middlewares/LoRaWAN/Mac/LoRaMacClassB.o
                0x0000000008010606                LoRaMacClassBResumeBeaconing
 .text.LoRaMacClassBSwitchClass
                0x0000000008010610       0x16 ./Drivers/Middlewares/LoRaWAN/Mac/LoRaMacClassB.o
                0x0000000008010610                LoRaMacClassBSwitchClass
 .text.LoRaMacClassBMibGetRequestConfirm
                0x0000000008010626       0x12 ./Drivers/Middlewares/LoRaWAN/Mac/LoRaMacClassB.o
                0x0000000008010626                LoRaMacClassBMibGetRequestConfirm
 .text.LoRaMacMibClassBSetRequestConfirm
                0x0000000008010638       0x12 ./Drivers/Middlewares/LoRaWAN/Mac/LoRaMacClassB.o
                0x0000000008010638                LoRaMacMibClassBSetRequestConfirm
 .text.LoRaMacClassBPingSlotInfoAns
                0x000000000801064a        0xa ./Drivers/Middlewares/LoRaWAN/Mac/LoRaMacClassB.o
                0x000000000801064a                LoRaMacClassBPingSlotInfoAns
 .text.LoRaMacClassBPingSlotChannelReq
                0x0000000008010654       0x18 ./Drivers/Middlewares/LoRaWAN/Mac/LoRaMacClassB.o
                0x0000000008010654                LoRaMacClassBPingSlotChannelReq
 .text.LoRaMacClassBBeaconTimingAns
                0x000000000801066c       0x1c ./Drivers/Middlewares/LoRaWAN/Mac/LoRaMacClassB.o
                0x000000000801066c                LoRaMacClassBBeaconTimingAns
 .text.LoRaMacClassBDeviceTimeAns
                0x0000000008010688        0xa ./Drivers/Middlewares/LoRaWAN/Mac/LoRaMacClassB.o
                0x0000000008010688                LoRaMacClassBDeviceTimeAns
 .text.LoRaMacClassBBeaconFreqReq
                0x0000000008010692       0x12 ./Drivers/Middlewares/LoRaWAN/Mac/LoRaMacClassB.o
                0x0000000008010692                LoRaMacClassBBeaconFreqReq
 .text.LoRaMacClassBIsUplinkCollision
                0x00000000080106a4       0x12 ./Drivers/Middlewares/LoRaWAN/Mac/LoRaMacClassB.o
                0x00000000080106a4                LoRaMacClassBIsUplinkCollision
 .text.LoRaMacClassBStopRxSlots
                0x00000000080106b6        0xa ./Drivers/Middlewares/LoRaWAN/Mac/LoRaMacClassB.o
                0x00000000080106b6                LoRaMacClassBStopRxSlots
 .text.LoRaMacClassBProcess
                0x00000000080106c0        0xa ./Drivers/Middlewares/LoRaWAN/Mac/LoRaMacClassB.o
                0x00000000080106c0                LoRaMacClassBProcess
 .text.IsSlotFree
                0x00000000080106ca       0x4a ./Drivers/Middlewares/LoRaWAN/Mac/LoRaMacCommands.o
 .text.MallocNewMacCommandSlot
                0x0000000008010714       0x60 ./Drivers/Middlewares/LoRaWAN/Mac/LoRaMacCommands.o
 .text.FreeMacCommandSlot
                0x0000000008010774       0x28 ./Drivers/Middlewares/LoRaWAN/Mac/LoRaMacCommands.o
 .text.LinkedListInit
                0x000000000801079c       0x28 ./Drivers/Middlewares/LoRaWAN/Mac/LoRaMacCommands.o
 .text.LinkedListAdd
                0x00000000080107c4       0x4e ./Drivers/Middlewares/LoRaWAN/Mac/LoRaMacCommands.o
 .text.LinkedListGetPrevious
                0x0000000008010812       0x50 ./Drivers/Middlewares/LoRaWAN/Mac/LoRaMacCommands.o
 .text.LinkedListRemove
                0x0000000008010862       0x6a ./Drivers/Middlewares/LoRaWAN/Mac/LoRaMacCommands.o
 .text.IsSticky
                0x00000000080108cc       0x40 ./Drivers/Middlewares/LoRaWAN/Mac/LoRaMacCommands.o
 .text.NvmCtxCallback
                0x000000000801090c       0x1c ./Drivers/Middlewares/LoRaWAN/Mac/LoRaMacCommands.o
 .text.LoRaMacCommandsInit
                0x0000000008010928       0x34 ./Drivers/Middlewares/LoRaWAN/Mac/LoRaMacCommands.o
                0x0000000008010928                LoRaMacCommandsInit
 .text.LoRaMacCommandsRestoreNvmCtx
                0x000000000801095c       0x2c ./Drivers/Middlewares/LoRaWAN/Mac/LoRaMacCommands.o
                0x000000000801095c                LoRaMacCommandsRestoreNvmCtx
 .text.LoRaMacCommandsGetNvmCtx
                0x0000000008010988       0x1c ./Drivers/Middlewares/LoRaWAN/Mac/LoRaMacCommands.o
                0x0000000008010988                LoRaMacCommandsGetNvmCtx
 .text.LoRaMacCommandsAddCmd
                0x00000000080109a4       0xa4 ./Drivers/Middlewares/LoRaWAN/Mac/LoRaMacCommands.o
                0x00000000080109a4                LoRaMacCommandsAddCmd
 .text.LoRaMacCommandsRemoveCmd
                0x0000000008010a48       0x70 ./Drivers/Middlewares/LoRaWAN/Mac/LoRaMacCommands.o
                0x0000000008010a48                LoRaMacCommandsRemoveCmd
 .text.LoRaMacCommandsRemoveNoneStickyCmds
                0x0000000008010ab8       0x50 ./Drivers/Middlewares/LoRaWAN/Mac/LoRaMacCommands.o
                0x0000000008010ab8                LoRaMacCommandsRemoveNoneStickyCmds
 .text.LoRaMacCommandsRemoveStickyAnsCmds
                0x0000000008010b08       0x48 ./Drivers/Middlewares/LoRaWAN/Mac/LoRaMacCommands.o
                0x0000000008010b08                LoRaMacCommandsRemoveStickyAnsCmds
 .text.LoRaMacCommandsGetSizeSerializedCmds
                0x0000000008010b50       0x2c ./Drivers/Middlewares/LoRaWAN/Mac/LoRaMacCommands.o
                0x0000000008010b50                LoRaMacCommandsGetSizeSerializedCmds
 .text.LoRaMacCommandsSerializeCmds
                0x0000000008010b7c       0x9c ./Drivers/Middlewares/LoRaWAN/Mac/LoRaMacCommands.o
                0x0000000008010b7c                LoRaMacCommandsSerializeCmds
 .text.LoRaMacCommandsStickyCmdsPending
                0x0000000008010c18       0x4c ./Drivers/Middlewares/LoRaWAN/Mac/LoRaMacCommands.o
                0x0000000008010c18                LoRaMacCommandsStickyCmdsPending
 .text.IncreaseBufferPointer
                0x0000000008010c64       0x30 ./Drivers/Middlewares/LoRaWAN/Mac/LoRaMacConfirmQueue.o
 .text.GetElement
                0x0000000008010c94       0x48 ./Drivers/Middlewares/LoRaWAN/Mac/LoRaMacConfirmQueue.o
 .text.LoRaMacConfirmQueueInit
                0x0000000008010cdc       0x60 ./Drivers/Middlewares/LoRaWAN/Mac/LoRaMacConfirmQueue.o
                0x0000000008010cdc                LoRaMacConfirmQueueInit
 .text.LoRaMacConfirmQueueRestoreNvmCtx
                0x0000000008010d3c       0x2c ./Drivers/Middlewares/LoRaWAN/Mac/LoRaMacConfirmQueue.o
                0x0000000008010d3c                LoRaMacConfirmQueueRestoreNvmCtx
 .text.LoRaMacConfirmQueueGetNvmCtx
                0x0000000008010d68       0x1c ./Drivers/Middlewares/LoRaWAN/Mac/LoRaMacConfirmQueue.o
                0x0000000008010d68                LoRaMacConfirmQueueGetNvmCtx
 .text.LoRaMacConfirmQueueAdd
                0x0000000008010d84       0x68 ./Drivers/Middlewares/LoRaWAN/Mac/LoRaMacConfirmQueue.o
                0x0000000008010d84                LoRaMacConfirmQueueAdd
 .text.LoRaMacConfirmQueueRemoveFirst
                0x0000000008010dec       0x3c ./Drivers/Middlewares/LoRaWAN/Mac/LoRaMacConfirmQueue.o
                0x0000000008010dec                LoRaMacConfirmQueueRemoveFirst
 .text.LoRaMacConfirmQueueSetStatus
                0x0000000008010e28       0x58 ./Drivers/Middlewares/LoRaWAN/Mac/LoRaMacConfirmQueue.o
                0x0000000008010e28                LoRaMacConfirmQueueSetStatus
 .text.LoRaMacConfirmQueueGetStatus
                0x0000000008010e80       0x4c ./Drivers/Middlewares/LoRaWAN/Mac/LoRaMacConfirmQueue.o
                0x0000000008010e80                LoRaMacConfirmQueueGetStatus
 .text.LoRaMacConfirmQueueSetStatusCmn
                0x0000000008010ecc       0x64 ./Drivers/Middlewares/LoRaWAN/Mac/LoRaMacConfirmQueue.o
                0x0000000008010ecc                LoRaMacConfirmQueueSetStatusCmn
 .text.LoRaMacConfirmQueueIsCmdActive
                0x0000000008010f30       0x34 ./Drivers/Middlewares/LoRaWAN/Mac/LoRaMacConfirmQueue.o
                0x0000000008010f30                LoRaMacConfirmQueueIsCmdActive
 .text.LoRaMacConfirmQueueHandleCb
                0x0000000008010f64       0xc4 ./Drivers/Middlewares/LoRaWAN/Mac/LoRaMacConfirmQueue.o
                0x0000000008010f64                LoRaMacConfirmQueueHandleCb
 .text.LoRaMacConfirmQueueGetCnt
                0x0000000008011028       0x14 ./Drivers/Middlewares/LoRaWAN/Mac/LoRaMacConfirmQueue.o
                0x0000000008011028                LoRaMacConfirmQueueGetCnt
 .text.LoRaMacConfirmQueueIsFull
                0x000000000801103c       0x20 ./Drivers/Middlewares/LoRaWAN/Mac/LoRaMacConfirmQueue.o
                0x000000000801103c                LoRaMacConfirmQueueIsFull
 .text.PayloadEncrypt
                0x000000000801105c      0x18c ./Drivers/Middlewares/LoRaWAN/Mac/LoRaMacCrypto.o
 .text.PrepareB0
                0x00000000080111e8      0x120 ./Drivers/Middlewares/LoRaWAN/Mac/LoRaMacCrypto.o
 .text.ComputeCmacB0
                0x0000000008011308       0x8e ./Drivers/Middlewares/LoRaWAN/Mac/LoRaMacCrypto.o
 *fill*         0x0000000008011396        0x2 
 .text.VerifyCmacB0
                0x0000000008011398      0x134 ./Drivers/Middlewares/LoRaWAN/Mac/LoRaMacCrypto.o
 .text.GetKeyAddrItem
                0x00000000080114cc       0x64 ./Drivers/Middlewares/LoRaWAN/Mac/LoRaMacCrypto.o
 .text.DeriveSessionKey10x
                0x0000000008011530       0xc4 ./Drivers/Middlewares/LoRaWAN/Mac/LoRaMacCrypto.o
 .text.GetLastFcntDown
                0x00000000080115f4       0xb8 ./Drivers/Middlewares/LoRaWAN/Mac/LoRaMacCrypto.o
 .text.CheckFCntDown
                0x00000000080116ac       0x46 ./Drivers/Middlewares/LoRaWAN/Mac/LoRaMacCrypto.o
 *fill*         0x00000000080116f2        0x2 
 .text.UpdateFCntDown
                0x00000000080116f4       0x80 ./Drivers/Middlewares/LoRaWAN/Mac/LoRaMacCrypto.o
 .text.ResetFCnts
                0x0000000008011774       0x70 ./Drivers/Middlewares/LoRaWAN/Mac/LoRaMacCrypto.o
 .text.DummyCB  0x00000000080117e4        0xa ./Drivers/Middlewares/LoRaWAN/Mac/LoRaMacCrypto.o
 *fill*         0x00000000080117ee        0x2 
 .text.LoRaMacCryptoInit
                0x00000000080117f0       0x6c ./Drivers/Middlewares/LoRaWAN/Mac/LoRaMacCrypto.o
                0x00000000080117f0                LoRaMacCryptoInit
 .text.LoRaMacCryptoSetLrWanVersion
                0x000000000801185c       0x20 ./Drivers/Middlewares/LoRaWAN/Mac/LoRaMacCrypto.o
                0x000000000801185c                LoRaMacCryptoSetLrWanVersion
 .text.LoRaMacCryptoRestoreNvmCtx
                0x000000000801187c       0x2c ./Drivers/Middlewares/LoRaWAN/Mac/LoRaMacCrypto.o
                0x000000000801187c                LoRaMacCryptoRestoreNvmCtx
 .text.LoRaMacCryptoGetNvmCtx
                0x00000000080118a8       0x1c ./Drivers/Middlewares/LoRaWAN/Mac/LoRaMacCrypto.o
                0x00000000080118a8                LoRaMacCryptoGetNvmCtx
 .text.LoRaMacCryptoGetFCntUp
                0x00000000080118c4       0x2c ./Drivers/Middlewares/LoRaWAN/Mac/LoRaMacCrypto.o
                0x00000000080118c4                LoRaMacCryptoGetFCntUp
 .text.LoRaMacCryptoGetFCntDown
                0x00000000080118f0      0x11c ./Drivers/Middlewares/LoRaWAN/Mac/LoRaMacCrypto.o
                0x00000000080118f0                LoRaMacCryptoGetFCntDown
 .text.LoRaMacCryptoSetMulticastReference
                0x0000000008011a0c       0x50 ./Drivers/Middlewares/LoRaWAN/Mac/LoRaMacCrypto.o
                0x0000000008011a0c                LoRaMacCryptoSetMulticastReference
 .text.LoRaMacCryptoSetKey
                0x0000000008011a5c       0x5e ./Drivers/Middlewares/LoRaWAN/Mac/LoRaMacCrypto.o
                0x0000000008011a5c                LoRaMacCryptoSetKey
 *fill*         0x0000000008011aba        0x2 
 .text.LoRaMacCryptoPrepareJoinRequest
                0x0000000008011abc       0x94 ./Drivers/Middlewares/LoRaWAN/Mac/LoRaMacCrypto.o
                0x0000000008011abc                LoRaMacCryptoPrepareJoinRequest
 .text.LoRaMacCryptoHandleJoinAccept
                0x0000000008011b50      0x3b4 ./Drivers/Middlewares/LoRaWAN/Mac/LoRaMacCrypto.o
                0x0000000008011b50                LoRaMacCryptoHandleJoinAccept
 .text.LoRaMacCryptoSecureMessage
                0x0000000008011f04      0x11c ./Drivers/Middlewares/LoRaWAN/Mac/LoRaMacCrypto.o
                0x0000000008011f04                LoRaMacCryptoSecureMessage
 .text.LoRaMacCryptoUnsecureMessage
                0x0000000008012020      0x190 ./Drivers/Middlewares/LoRaWAN/Mac/LoRaMacCrypto.o
                0x0000000008012020                LoRaMacCryptoUnsecureMessage
 .text.LoRaMacCryptoDeriveMcRootKey
                0x00000000080121b0       0x84 ./Drivers/Middlewares/LoRaWAN/Mac/LoRaMacCrypto.o
                0x00000000080121b0                LoRaMacCryptoDeriveMcRootKey
 .text.LoRaMacCryptoDeriveMcKEKey
                0x0000000008012234       0x54 ./Drivers/Middlewares/LoRaWAN/Mac/LoRaMacCrypto.o
                0x0000000008012234                LoRaMacCryptoDeriveMcKEKey
 .text.LoRaMacParserJoinAccept
                0x0000000008012288      0x1e0 ./Drivers/Middlewares/LoRaWAN/Mac/LoRaMacParser.o
                0x0000000008012288                LoRaMacParserJoinAccept
 .text.LoRaMacParserData
                0x0000000008012468      0x220 ./Drivers/Middlewares/LoRaWAN/Mac/LoRaMacParser.o
                0x0000000008012468                LoRaMacParserData
 .text.LoRaMacSerializerJoinRequest
                0x0000000008012688      0x136 ./Drivers/Middlewares/LoRaWAN/Mac/LoRaMacSerializer.o
                0x0000000008012688                LoRaMacSerializerJoinRequest
 .text.LoRaMacSerializerData
                0x00000000080127be      0x256 ./Drivers/Middlewares/LoRaWAN/Mac/LoRaMacSerializer.o
                0x00000000080127be                LoRaMacSerializerData
 .text.RegionIsActive
                0x0000000008012a14       0x22 ./Drivers/Middlewares/LoRaWAN/Mac/region/Region.o
                0x0000000008012a14                RegionIsActive
 .text.RegionGetPhyParam
                0x0000000008012a36       0x4e ./Drivers/Middlewares/LoRaWAN/Mac/region/Region.o
                0x0000000008012a36                RegionGetPhyParam
 .text.RegionSetBandTxDone
                0x0000000008012a84       0x28 ./Drivers/Middlewares/LoRaWAN/Mac/region/Region.o
                0x0000000008012a84                RegionSetBandTxDone
 .text.RegionInitDefaults
                0x0000000008012aac       0x2a ./Drivers/Middlewares/LoRaWAN/Mac/region/Region.o
                0x0000000008012aac                RegionInitDefaults
 .text.RegionGetNvmCtx
                0x0000000008012ad6       0x2c ./Drivers/Middlewares/LoRaWAN/Mac/region/Region.o
                0x0000000008012ad6                RegionGetNvmCtx
 .text.RegionVerify
                0x0000000008012b02       0x3a ./Drivers/Middlewares/LoRaWAN/Mac/region/Region.o
                0x0000000008012b02                RegionVerify
 .text.RegionApplyCFList
                0x0000000008012b3c       0x2a ./Drivers/Middlewares/LoRaWAN/Mac/region/Region.o
                0x0000000008012b3c                RegionApplyCFList
 .text.RegionChanMaskSet
                0x0000000008012b66       0x2c ./Drivers/Middlewares/LoRaWAN/Mac/region/Region.o
                0x0000000008012b66                RegionChanMaskSet
 .text.RegionComputeRxWindowParameters
                0x0000000008012b92       0x48 ./Drivers/Middlewares/LoRaWAN/Mac/region/Region.o
                0x0000000008012b92                RegionComputeRxWindowParameters
 .text.RegionRxConfig
                0x0000000008012bda       0x34 ./Drivers/Middlewares/LoRaWAN/Mac/region/Region.o
                0x0000000008012bda                RegionRxConfig
 .text.RegionTxConfig
                0x0000000008012c0e       0x36 ./Drivers/Middlewares/LoRaWAN/Mac/region/Region.o
                0x0000000008012c0e                RegionTxConfig
 .text.RegionLinkAdrReq
                0x0000000008012c44       0x3c ./Drivers/Middlewares/LoRaWAN/Mac/region/Region.o
                0x0000000008012c44                RegionLinkAdrReq
 .text.RegionRxParamSetupReq
                0x0000000008012c80       0x2c ./Drivers/Middlewares/LoRaWAN/Mac/region/Region.o
                0x0000000008012c80                RegionRxParamSetupReq
 .text.RegionNewChannelReq
                0x0000000008012cac       0x2c ./Drivers/Middlewares/LoRaWAN/Mac/region/Region.o
                0x0000000008012cac                RegionNewChannelReq
 .text.RegionTxParamSetupReq
                0x0000000008012cd8       0x2c ./Drivers/Middlewares/LoRaWAN/Mac/region/Region.o
                0x0000000008012cd8                RegionTxParamSetupReq
 .text.RegionDlChannelReq
                0x0000000008012d04       0x2c ./Drivers/Middlewares/LoRaWAN/Mac/region/Region.o
                0x0000000008012d04                RegionDlChannelReq
 .text.RegionAlternateDr
                0x0000000008012d30       0x46 ./Drivers/Middlewares/LoRaWAN/Mac/region/Region.o
                0x0000000008012d30                RegionAlternateDr
 .text.RegionCalcBackOff
                0x0000000008012d76       0x2a ./Drivers/Middlewares/LoRaWAN/Mac/region/Region.o
                0x0000000008012d76                RegionCalcBackOff
 .text.RegionNextChannel
                0x0000000008012da0       0x36 ./Drivers/Middlewares/LoRaWAN/Mac/region/Region.o
                0x0000000008012da0                RegionNextChannel
 .text.RegionSetContinuousWave
                0x0000000008012dd6       0x2a ./Drivers/Middlewares/LoRaWAN/Mac/region/Region.o
                0x0000000008012dd6                RegionSetContinuousWave
 .text.RegionApplyDrOffset
                0x0000000008012e00       0x54 ./Drivers/Middlewares/LoRaWAN/Mac/region/Region.o
                0x0000000008012e00                RegionApplyDrOffset
 .text.CountChannels
                0x0000000008012e54       0x78 ./Drivers/Middlewares/LoRaWAN/Mac/region/RegionCommon.o
 .text.RegionCommonGetJoinDc
                0x0000000008012ecc       0x58 ./Drivers/Middlewares/LoRaWAN/Mac/region/RegionCommon.o
                0x0000000008012ecc                RegionCommonGetJoinDc
 .text.RegionCommonChanVerifyDr
                0x0000000008012f24      0x132 ./Drivers/Middlewares/LoRaWAN/Mac/region/RegionCommon.o
                0x0000000008012f24                RegionCommonChanVerifyDr
 .text.RegionCommonValueInRange
                0x0000000008013056       0x4c ./Drivers/Middlewares/LoRaWAN/Mac/region/RegionCommon.o
                0x0000000008013056                RegionCommonValueInRange
 .text.RegionCommonChanDisable
                0x00000000080130a2       0x84 ./Drivers/Middlewares/LoRaWAN/Mac/region/RegionCommon.o
                0x00000000080130a2                RegionCommonChanDisable
 .text.RegionCommonCountChannels
                0x0000000008013126       0x82 ./Drivers/Middlewares/LoRaWAN/Mac/region/RegionCommon.o
                0x0000000008013126                RegionCommonCountChannels
 .text.RegionCommonChanMaskCopy
                0x00000000080131a8       0x5e ./Drivers/Middlewares/LoRaWAN/Mac/region/RegionCommon.o
                0x00000000080131a8                RegionCommonChanMaskCopy
 .text.RegionCommonSetBandTxDone
                0x0000000008013206       0x36 ./Drivers/Middlewares/LoRaWAN/Mac/region/RegionCommon.o
                0x0000000008013206                RegionCommonSetBandTxDone
 .text.RegionCommonUpdateBandTimeOff
                0x000000000801323c      0x186 ./Drivers/Middlewares/LoRaWAN/Mac/region/RegionCommon.o
                0x000000000801323c                RegionCommonUpdateBandTimeOff
 .text.RegionCommonParseLinkAdrReq
                0x00000000080133c2       0xaa ./Drivers/Middlewares/LoRaWAN/Mac/region/RegionCommon.o
                0x00000000080133c2                RegionCommonParseLinkAdrReq
 .text.RegionCommonLinkAdrReqVerifyParams
                0x000000000801346c      0x13c ./Drivers/Middlewares/LoRaWAN/Mac/region/RegionCommon.o
                0x000000000801346c                RegionCommonLinkAdrReqVerifyParams
 .text.RegionCommonComputeSymbolTimeLoRa
                0x00000000080135a8       0x58 ./Drivers/Middlewares/LoRaWAN/Mac/region/RegionCommon.o
                0x00000000080135a8                RegionCommonComputeSymbolTimeLoRa
 .text.RegionCommonComputeSymbolTimeFsk
                0x0000000008013600       0x34 ./Drivers/Middlewares/LoRaWAN/Mac/region/RegionCommon.o
                0x0000000008013600                RegionCommonComputeSymbolTimeFsk
 .text.RegionCommonComputeRxWindowParameters
                0x0000000008013634      0x108 ./Drivers/Middlewares/LoRaWAN/Mac/region/RegionCommon.o
                0x0000000008013634                RegionCommonComputeRxWindowParameters
 .text.RegionCommonComputeTxPower
                0x000000000801373c       0x72 ./Drivers/Middlewares/LoRaWAN/Mac/region/RegionCommon.o
                0x000000000801373c                RegionCommonComputeTxPower
 .text.RegionCommonCalcBackOff
                0x00000000080137ae      0x118 ./Drivers/Middlewares/LoRaWAN/Mac/region/RegionCommon.o
                0x00000000080137ae                RegionCommonCalcBackOff
 .text.GetNextLowerTxDr
                0x00000000080138c6       0x64 ./Drivers/Middlewares/LoRaWAN/Mac/region/RegionIN865.o
 *fill*         0x000000000801392a        0x2 
 .text.GetBandwidth
                0x000000000801392c       0x3c ./Drivers/Middlewares/LoRaWAN/Mac/region/RegionIN865.o
 .text.LimitTxPower
                0x0000000008013968       0x50 ./Drivers/Middlewares/LoRaWAN/Mac/region/RegionIN865.o
 .text.VerifyRfFreq
                0x00000000080139b8       0x50 ./Drivers/Middlewares/LoRaWAN/Mac/region/RegionIN865.o
 .text.CountNbOfEnabledChannels
                0x0000000008013a08      0x1c2 ./Drivers/Middlewares/LoRaWAN/Mac/region/RegionIN865.o
 *fill*         0x0000000008013bca        0x2 
 .text.RegionIN865GetPhyParam
                0x0000000008013bcc      0x208 ./Drivers/Middlewares/LoRaWAN/Mac/region/RegionIN865.o
                0x0000000008013bcc                RegionIN865GetPhyParam
 .text.RegionIN865SetBandTxDone
                0x0000000008013dd4       0x40 ./Drivers/Middlewares/LoRaWAN/Mac/region/RegionIN865.o
                0x0000000008013dd4                RegionIN865SetBandTxDone
 .text.RegionIN865InitDefaults
                0x0000000008013e14       0xf4 ./Drivers/Middlewares/LoRaWAN/Mac/region/RegionIN865.o
                0x0000000008013e14                RegionIN865InitDefaults
 .text.RegionIN865GetNvmCtx
                0x0000000008013f08       0x1c ./Drivers/Middlewares/LoRaWAN/Mac/region/RegionIN865.o
                0x0000000008013f08                RegionIN865GetNvmCtx
 .text.RegionIN865Verify
                0x0000000008013f24       0xc4 ./Drivers/Middlewares/LoRaWAN/Mac/region/RegionIN865.o
                0x0000000008013f24                RegionIN865Verify
 .text.RegionIN865ApplyCFList
                0x0000000008013fe8      0x120 ./Drivers/Middlewares/LoRaWAN/Mac/region/RegionIN865.o
                0x0000000008013fe8                RegionIN865ApplyCFList
 .text.RegionIN865ChanMaskSet
                0x0000000008014108       0x4c ./Drivers/Middlewares/LoRaWAN/Mac/region/RegionIN865.o
                0x0000000008014108                RegionIN865ChanMaskSet
 .text.RegionIN865ComputeRxWindowParameters
                0x0000000008014154       0xd4 ./Drivers/Middlewares/LoRaWAN/Mac/region/RegionIN865.o
                0x0000000008014154                RegionIN865ComputeRxWindowParameters
 .text.RegionIN865RxConfig
                0x0000000008014228      0x1e8 ./Drivers/Middlewares/LoRaWAN/Mac/region/RegionIN865.o
                0x0000000008014228                RegionIN865RxConfig
 .text.RegionIN865TxConfig
                0x0000000008014410      0x1d8 ./Drivers/Middlewares/LoRaWAN/Mac/region/RegionIN865.o
                0x0000000008014410                RegionIN865TxConfig
 .text.RegionIN865LinkAdrReq
                0x00000000080145e8      0x2b8 ./Drivers/Middlewares/LoRaWAN/Mac/region/RegionIN865.o
                0x00000000080145e8                RegionIN865LinkAdrReq
 .text.RegionIN865RxParamSetupReq
                0x00000000080148a0       0x86 ./Drivers/Middlewares/LoRaWAN/Mac/region/RegionIN865.o
                0x00000000080148a0                RegionIN865RxParamSetupReq
 .text.RegionIN865NewChannelReq
                0x0000000008014926       0xd0 ./Drivers/Middlewares/LoRaWAN/Mac/region/RegionIN865.o
                0x0000000008014926                RegionIN865NewChannelReq
 .text.RegionIN865TxParamSetupReq
                0x00000000080149f6       0x14 ./Drivers/Middlewares/LoRaWAN/Mac/region/RegionIN865.o
                0x00000000080149f6                RegionIN865TxParamSetupReq
 *fill*         0x0000000008014a0a        0x2 
 .text.RegionIN865DlChannelReq
                0x0000000008014a0c       0x90 ./Drivers/Middlewares/LoRaWAN/Mac/region/RegionIN865.o
                0x0000000008014a0c                RegionIN865DlChannelReq
 .text.RegionIN865AlternateDr
                0x0000000008014a9c       0x20 ./Drivers/Middlewares/LoRaWAN/Mac/region/RegionIN865.o
                0x0000000008014a9c                RegionIN865AlternateDr
 .text.RegionIN865CalcBackOff
                0x0000000008014abc       0x60 ./Drivers/Middlewares/LoRaWAN/Mac/region/RegionIN865.o
                0x0000000008014abc                RegionIN865CalcBackOff
 .text.RegionIN865NextChannel
                0x0000000008014b1c      0x14c ./Drivers/Middlewares/LoRaWAN/Mac/region/RegionIN865.o
                0x0000000008014b1c                RegionIN865NextChannel
 .text.RegionIN865ChannelAdd
                0x0000000008014c68      0x170 ./Drivers/Middlewares/LoRaWAN/Mac/region/RegionIN865.o
                0x0000000008014c68                RegionIN865ChannelAdd
 .text.RegionIN865ChannelsRemove
                0x0000000008014dd8       0x5c ./Drivers/Middlewares/LoRaWAN/Mac/region/RegionIN865.o
                0x0000000008014dd8                RegionIN865ChannelsRemove
 .text.RegionIN865SetContinuousWave
                0x0000000008014e34       0xa8 ./Drivers/Middlewares/LoRaWAN/Mac/region/RegionIN865.o
                0x0000000008014e34                RegionIN865SetContinuousWave
 .text.RegionIN865ApplyDrOffset
                0x0000000008014edc       0x5c ./Drivers/Middlewares/LoRaWAN/Mac/region/RegionIN865.o
                0x0000000008014edc                RegionIN865ApplyDrOffset
 .text.certif_running
                0x0000000008014f38       0x14 ./Drivers/Middlewares/LoRaWAN/Patterns/Basic/lora-test.o
                0x0000000008014f38                certif_running
 .text.certif_DownLinkIncrement
                0x0000000008014f4c       0x20 ./Drivers/Middlewares/LoRaWAN/Patterns/Basic/lora-test.o
                0x0000000008014f4c                certif_DownLinkIncrement
 .text.certif_linkCheck
                0x0000000008014f6c       0x30 ./Drivers/Middlewares/LoRaWAN/Patterns/Basic/lora-test.o
                0x0000000008014f6c                certif_linkCheck
 .text.certif_tx
                0x0000000008014f9c      0x134 ./Drivers/Middlewares/LoRaWAN/Patterns/Basic/lora-test.o
 .text.certif_rx
                0x00000000080150d0      0x2e8 ./Drivers/Middlewares/LoRaWAN/Patterns/Basic/lora-test.o
                0x00000000080150d0                certif_rx
 .text.OnCertifTxNextPacketTimerEvent
                0x00000000080153b8       0x14 ./Drivers/Middlewares/LoRaWAN/Patterns/Basic/lora-test.o
 .text.McpsConfirm
                0x00000000080153cc       0x88 ./Drivers/Middlewares/LoRaWAN/Patterns/Basic/lora.o
 .text.McpsIndication
                0x0000000008015454       0xfc ./Drivers/Middlewares/LoRaWAN/Patterns/Basic/lora.o
 .text.MlmeConfirm
                0x0000000008015550       0x98 ./Drivers/Middlewares/LoRaWAN/Patterns/Basic/lora.o
 .text.MlmeIndication
                0x00000000080155e8       0x6c ./Drivers/Middlewares/LoRaWAN/Patterns/Basic/lora.o
 .text.LORA_Init
                0x0000000008015654      0x340 ./Drivers/Middlewares/LoRaWAN/Patterns/Basic/lora.o
                0x0000000008015654                LORA_Init
 .text.LORA_Join
                0x0000000008015994      0x114 ./Drivers/Middlewares/LoRaWAN/Patterns/Basic/lora.o
                0x0000000008015994                LORA_Join
 .text.LORA_JoinStatus
                0x0000000008015aa8       0x2a ./Drivers/Middlewares/LoRaWAN/Patterns/Basic/lora.o
                0x0000000008015aa8                LORA_JoinStatus
 *fill*         0x0000000008015ad2        0x2 
 .text.LORA_send
                0x0000000008015ad4       0xdc ./Drivers/Middlewares/LoRaWAN/Patterns/Basic/lora.o
                0x0000000008015ad4                LORA_send
 .text.LORA_RequestClass
                0x0000000008015bb0       0xdc ./Drivers/Middlewares/LoRaWAN/Patterns/Basic/lora.o
                0x0000000008015bb0                LORA_RequestClass
 .text.TraceUpLinkFrame
                0x0000000008015c8c       0xf8 ./Drivers/Middlewares/LoRaWAN/Patterns/Basic/lora.o
 .text.TraceDownLinkFrame
                0x0000000008015d84       0x90 ./Drivers/Middlewares/LoRaWAN/Patterns/Basic/lora.o
 .text.LPM_SetOffMode
                0x0000000008015e14       0x68 ./Drivers/Middlewares/LoRaWAN/Utilities/low_power_manager.o
                0x0000000008015e14                LPM_SetOffMode
 .text.LPM_SetStopMode
                0x0000000008015e7c       0x68 ./Drivers/Middlewares/LoRaWAN/Utilities/low_power_manager.o
                0x0000000008015e7c                LPM_SetStopMode
 .text.LPM_GetMode
                0x0000000008015ee4       0x64 ./Drivers/Middlewares/LoRaWAN/Utilities/low_power_manager.o
                0x0000000008015ee4                LPM_GetMode
 .text.circular_queue_init
                0x0000000008015f48       0x3c ./Drivers/Middlewares/LoRaWAN/Utilities/queue.o
                0x0000000008015f48                circular_queue_init
 .text.circular_queue_add
                0x0000000008015f84      0x18a ./Drivers/Middlewares/LoRaWAN/Utilities/queue.o
                0x0000000008015f84                circular_queue_add
 .text.circular_queue_get
                0x000000000801610e       0xb0 ./Drivers/Middlewares/LoRaWAN/Utilities/queue.o
                0x000000000801610e                circular_queue_get
 .text.circular_queue_remove
                0x00000000080161be       0xc0 ./Drivers/Middlewares/LoRaWAN/Utilities/queue.o
                0x00000000080161be                circular_queue_remove
 .text.circular_queue_sense
                0x000000000801627e       0x26 ./Drivers/Middlewares/LoRaWAN/Utilities/queue.o
                0x000000000801627e                circular_queue_sense
 .text.circular_queue_get_free_size
                0x00000000080162a4       0x62 ./Drivers/Middlewares/LoRaWAN/Utilities/queue.o
 .text.queue_copy
                0x0000000008016306       0x38 ./Drivers/Middlewares/LoRaWAN/Utilities/queue.o
 .text.add_elementSize_and_inc_writeIdx
                0x000000000801633e       0x72 ./Drivers/Middlewares/LoRaWAN/Utilities/queue.o
 .text.SysTimeAdd
                0x00000000080163b0       0xa4 ./Drivers/Middlewares/LoRaWAN/Utilities/systime.o
                0x00000000080163b0                SysTimeAdd
 .text.SysTimeSub
                0x0000000008016454       0x9c ./Drivers/Middlewares/LoRaWAN/Utilities/systime.o
                0x0000000008016454                SysTimeSub
 .text.SysTimeSet
                0x00000000080164f0       0x60 ./Drivers/Middlewares/LoRaWAN/Utilities/systime.o
                0x00000000080164f0                SysTimeSet
 .text.SysTimeGet
                0x0000000008016550       0x70 ./Drivers/Middlewares/LoRaWAN/Utilities/systime.o
                0x0000000008016550                SysTimeGet
 .text.SysTimeGetMcuTime
                0x00000000080165c0       0x36 ./Drivers/Middlewares/LoRaWAN/Utilities/systime.o
                0x00000000080165c0                SysTimeGetMcuTime
 .text.TimerInit
                0x00000000080165f6       0x3c ./Drivers/Middlewares/LoRaWAN/Utilities/timeServer.o
                0x00000000080165f6                TimerInit
 *fill*         0x0000000008016632        0x2 
 .text.TimerStart
                0x0000000008016634       0xb0 ./Drivers/Middlewares/LoRaWAN/Utilities/timeServer.o
                0x0000000008016634                TimerStart
 .text.TimerIrqHandler
                0x00000000080166e4      0x108 ./Drivers/Middlewares/LoRaWAN/Utilities/timeServer.o
                0x00000000080166e4                TimerIrqHandler
 .text.TimerStop
                0x00000000080167ec       0xfc ./Drivers/Middlewares/LoRaWAN/Utilities/timeServer.o
                0x00000000080167ec                TimerStop
 .text.TimerSetValue
                0x00000000080168e8       0x4a ./Drivers/Middlewares/LoRaWAN/Utilities/timeServer.o
                0x00000000080168e8                TimerSetValue
 .text.TimerGetCurrentTime
                0x0000000008016932       0x20 ./Drivers/Middlewares/LoRaWAN/Utilities/timeServer.o
                0x0000000008016932                TimerGetCurrentTime
 .text.TimerGetElapsedTime
                0x0000000008016952       0x3c ./Drivers/Middlewares/LoRaWAN/Utilities/timeServer.o
                0x0000000008016952                TimerGetElapsedTime
 *fill*         0x000000000801698e        0x2 
 .text.TimerExists
                0x0000000008016990       0x38 ./Drivers/Middlewares/LoRaWAN/Utilities/timeServer.o
 .text.TimerSetTimeout
                0x00000000080169c8       0x48 ./Drivers/Middlewares/LoRaWAN/Utilities/timeServer.o
 .text.TimerInsertTimer
                0x0000000008016a10       0x5c ./Drivers/Middlewares/LoRaWAN/Utilities/timeServer.o
 .text.TimerInsertNewHeadTimer
                0x0000000008016a6c       0x3c ./Drivers/Middlewares/LoRaWAN/Utilities/timeServer.o
 .text.TraceInit
                0x0000000008016aa8       0x2c ./Drivers/Middlewares/LoRaWAN/Utilities/trace.o
                0x0000000008016aa8                TraceInit
 .text.TraceSend
                0x0000000008016ad4      0x110 ./Drivers/Middlewares/LoRaWAN/Utilities/trace.o
                0x0000000008016ad4                TraceSend
 .text.Trace_TxCpltCallback
                0x0000000008016be4       0x84 ./Drivers/Middlewares/LoRaWAN/Utilities/trace.o
 .text.rand1    0x0000000008016c68       0x38 ./Drivers/Middlewares/LoRaWAN/Utilities/utilities.o
                0x0000000008016c68                rand1
 .text.srand1   0x0000000008016ca0       0x1c ./Drivers/Middlewares/LoRaWAN/Utilities/utilities.o
                0x0000000008016ca0                srand1
 .text.randr    0x0000000008016cbc       0x2c ./Drivers/Middlewares/LoRaWAN/Utilities/utilities.o
                0x0000000008016cbc                randr
 .text.memcpy1  0x0000000008016ce8       0x38 ./Drivers/Middlewares/LoRaWAN/Utilities/utilities.o
                0x0000000008016ce8                memcpy1
 .text.memcpyr  0x0000000008016d20       0x44 ./Drivers/Middlewares/LoRaWAN/Utilities/utilities.o
                0x0000000008016d20                memcpyr
 .text.memset1  0x0000000008016d64       0x3e ./Drivers/Middlewares/LoRaWAN/Utilities/utilities.o
                0x0000000008016d64                memset1
 *fill*         0x0000000008016da2        0x2 
 .text.HAL_Init
                0x0000000008016da4       0x40 ./Drivers/STM32L0xx_HAL_Driver/Src/stm32l0xx_hal.o
                0x0000000008016da4                HAL_Init
 .text.HAL_IncTick
                0x0000000008016de4       0x18 ./Drivers/STM32L0xx_HAL_Driver/Src/stm32l0xx_hal.o
                0x0000000008016de4                HAL_IncTick
 .text.HAL_GetTick
                0x0000000008016dfc       0x14 ./Drivers/STM32L0xx_HAL_Driver/Src/stm32l0xx_hal.o
                0x0000000008016dfc                HAL_GetTick
 .text.HAL_DBGMCU_EnableDBGSleepMode
                0x0000000008016e10       0x1c ./Drivers/STM32L0xx_HAL_Driver/Src/stm32l0xx_hal.o
                0x0000000008016e10                HAL_DBGMCU_EnableDBGSleepMode
 .text.HAL_DBGMCU_EnableDBGStopMode
                0x0000000008016e2c       0x1c ./Drivers/STM32L0xx_HAL_Driver/Src/stm32l0xx_hal.o
                0x0000000008016e2c                HAL_DBGMCU_EnableDBGStopMode
 .text.HAL_DBGMCU_EnableDBGStandbyMode
                0x0000000008016e48       0x1c ./Drivers/STM32L0xx_HAL_Driver/Src/stm32l0xx_hal.o
                0x0000000008016e48                HAL_DBGMCU_EnableDBGStandbyMode
 .text.HAL_ADC_Init
                0x0000000008016e64      0x2e8 ./Drivers/STM32L0xx_HAL_Driver/Src/stm32l0xx_hal_adc.o
                0x0000000008016e64                HAL_ADC_Init
 .text.HAL_ADC_MspInit
                0x000000000801714c       0x10 ./Drivers/STM32L0xx_HAL_Driver/Src/stm32l0xx_hal_adc.o
                0x000000000801714c                HAL_ADC_MspInit
 .text.HAL_ADC_Start
                0x000000000801715c       0xa8 ./Drivers/STM32L0xx_HAL_Driver/Src/stm32l0xx_hal_adc.o
                0x000000000801715c                HAL_ADC_Start
 .text.HAL_ADC_PollForConversion
                0x0000000008017204      0x12c ./Drivers/STM32L0xx_HAL_Driver/Src/stm32l0xx_hal_adc.o
                0x0000000008017204                HAL_ADC_PollForConversion
 .text.HAL_ADC_GetValue
                0x0000000008017330       0x16 ./Drivers/STM32L0xx_HAL_Driver/Src/stm32l0xx_hal_adc.o
                0x0000000008017330                HAL_ADC_GetValue
 *fill*         0x0000000008017346        0x2 
 .text.HAL_ADC_ConfigChannel
                0x0000000008017348      0x10c ./Drivers/STM32L0xx_HAL_Driver/Src/stm32l0xx_hal_adc.o
                0x0000000008017348                HAL_ADC_ConfigChannel
 .text.ADC_Enable
                0x0000000008017454       0xc0 ./Drivers/STM32L0xx_HAL_Driver/Src/stm32l0xx_hal_adc.o
 .text.ADC_DelayMicroSecond
                0x0000000008017514       0x40 ./Drivers/STM32L0xx_HAL_Driver/Src/stm32l0xx_hal_adc.o
 .text.HAL_ADCEx_Calibration_Start
                0x0000000008017554      0x12c ./Drivers/STM32L0xx_HAL_Driver/Src/stm32l0xx_hal_adc_ex.o
                0x0000000008017554                HAL_ADCEx_Calibration_Start
 .text.__NVIC_EnableIRQ
                0x0000000008017680       0x34 ./Drivers/STM32L0xx_HAL_Driver/Src/stm32l0xx_hal_cortex.o
 .text.__NVIC_SetPriority
                0x00000000080176b4       0xdc ./Drivers/STM32L0xx_HAL_Driver/Src/stm32l0xx_hal_cortex.o
 .text.__NVIC_SystemReset
                0x0000000008017790       0x24 ./Drivers/STM32L0xx_HAL_Driver/Src/stm32l0xx_hal_cortex.o
 .text.HAL_NVIC_SetPriority
                0x00000000080177b4       0x2a ./Drivers/STM32L0xx_HAL_Driver/Src/stm32l0xx_hal_cortex.o
                0x00000000080177b4                HAL_NVIC_SetPriority
 .text.HAL_NVIC_EnableIRQ
                0x00000000080177de       0x20 ./Drivers/STM32L0xx_HAL_Driver/Src/stm32l0xx_hal_cortex.o
                0x00000000080177de                HAL_NVIC_EnableIRQ
 .text.HAL_NVIC_SystemReset
                0x00000000080177fe        0x8 ./Drivers/STM32L0xx_HAL_Driver/Src/stm32l0xx_hal_cortex.o
                0x00000000080177fe                HAL_NVIC_SystemReset
 *fill*         0x0000000008017806        0x2 
 .text.HAL_DMA_Init
                0x0000000008017808       0xf0 ./Drivers/STM32L0xx_HAL_Driver/Src/stm32l0xx_hal_dma.o
                0x0000000008017808                HAL_DMA_Init
 .text.HAL_DMA_Start_IT
                0x00000000080178f8       0xcc ./Drivers/STM32L0xx_HAL_Driver/Src/stm32l0xx_hal_dma.o
                0x00000000080178f8                HAL_DMA_Start_IT
 .text.HAL_DMA_Abort_IT
                0x00000000080179c4       0x8e ./Drivers/STM32L0xx_HAL_Driver/Src/stm32l0xx_hal_dma.o
                0x00000000080179c4                HAL_DMA_Abort_IT
 .text.HAL_DMA_IRQHandler
                0x0000000008017a52      0x15c ./Drivers/STM32L0xx_HAL_Driver/Src/stm32l0xx_hal_dma.o
                0x0000000008017a52                HAL_DMA_IRQHandler
 .text.DMA_SetConfig
                0x0000000008017bae       0x5c ./Drivers/STM32L0xx_HAL_Driver/Src/stm32l0xx_hal_dma.o
 *fill*         0x0000000008017c0a        0x2 
 .text.HAL_GPIO_Init
                0x0000000008017c0c      0x2fc ./Drivers/STM32L0xx_HAL_Driver/Src/stm32l0xx_hal_gpio.o
                0x0000000008017c0c                HAL_GPIO_Init
 .text.HAL_GPIO_ReadPin
                0x0000000008017f08       0x3a ./Drivers/STM32L0xx_HAL_Driver/Src/stm32l0xx_hal_gpio.o
                0x0000000008017f08                HAL_GPIO_ReadPin
 .text.HAL_GPIO_WritePin
                0x0000000008017f42       0x3a ./Drivers/STM32L0xx_HAL_Driver/Src/stm32l0xx_hal_gpio.o
                0x0000000008017f42                HAL_GPIO_WritePin
 .text.HAL_GPIO_EXTI_IRQHandler
                0x0000000008017f7c       0x38 ./Drivers/STM32L0xx_HAL_Driver/Src/stm32l0xx_hal_gpio.o
                0x0000000008017f7c                HAL_GPIO_EXTI_IRQHandler
 .text.HAL_I2C_Init
                0x0000000008017fb4      0x12c ./Drivers/STM32L0xx_HAL_Driver/Src/stm32l0xx_hal_i2c.o
                0x0000000008017fb4                HAL_I2C_Init
 .text.HAL_I2C_Mem_Read
                0x00000000080180e0      0x268 ./Drivers/STM32L0xx_HAL_Driver/Src/stm32l0xx_hal_i2c.o
                0x00000000080180e0                HAL_I2C_Mem_Read
 .text.I2C_RequestMemoryRead
                0x0000000008018348       0xc4 ./Drivers/STM32L0xx_HAL_Driver/Src/stm32l0xx_hal_i2c.o
 .text.I2C_Flush_TXDR
                0x000000000801840c       0x44 ./Drivers/STM32L0xx_HAL_Driver/Src/stm32l0xx_hal_i2c.o
 .text.I2C_WaitOnFlagUntilTimeout
                0x0000000008018450       0x7e ./Drivers/STM32L0xx_HAL_Driver/Src/stm32l0xx_hal_i2c.o
 .text.I2C_WaitOnTXISFlagUntilTimeout
                0x00000000080184ce       0x7e ./Drivers/STM32L0xx_HAL_Driver/Src/stm32l0xx_hal_i2c.o
 .text.I2C_WaitOnSTOPFlagUntilTimeout
                0x000000000801854c       0x78 ./Drivers/STM32L0xx_HAL_Driver/Src/stm32l0xx_hal_i2c.o
 .text.I2C_IsAcknowledgeFailed
                0x00000000080185c4       0xcc ./Drivers/STM32L0xx_HAL_Driver/Src/stm32l0xx_hal_i2c.o
 .text.I2C_TransferConfig
                0x0000000008018690       0x6c ./Drivers/STM32L0xx_HAL_Driver/Src/stm32l0xx_hal_i2c.o
 .text.HAL_I2CEx_ConfigAnalogFilter
                0x00000000080186fc       0x98 ./Drivers/STM32L0xx_HAL_Driver/Src/stm32l0xx_hal_i2c_ex.o
                0x00000000080186fc                HAL_I2CEx_ConfigAnalogFilter
 .text.HAL_I2CEx_ConfigDigitalFilter
                0x0000000008018794       0x98 ./Drivers/STM32L0xx_HAL_Driver/Src/stm32l0xx_hal_i2c_ex.o
                0x0000000008018794                HAL_I2CEx_ConfigDigitalFilter
 .text.HAL_PWR_DisablePVD
                0x000000000801882c       0x1c ./Drivers/STM32L0xx_HAL_Driver/Src/stm32l0xx_hal_pwr.o
                0x000000000801882c                HAL_PWR_DisablePVD
 .text.HAL_PWREx_EnableFastWakeUp
                0x0000000008018848       0x1c ./Drivers/STM32L0xx_HAL_Driver/Src/stm32l0xx_hal_pwr_ex.o
                0x0000000008018848                HAL_PWREx_EnableFastWakeUp
 .text.HAL_PWREx_EnableUltraLowPower
                0x0000000008018864       0x1c ./Drivers/STM32L0xx_HAL_Driver/Src/stm32l0xx_hal_pwr_ex.o
                0x0000000008018864                HAL_PWREx_EnableUltraLowPower
 .text.HAL_RCC_OscConfig
                0x0000000008018880      0x7a0 ./Drivers/STM32L0xx_HAL_Driver/Src/stm32l0xx_hal_rcc.o
                0x0000000008018880                HAL_RCC_OscConfig
 .text.HAL_RCC_ClockConfig
                0x0000000008019020      0x254 ./Drivers/STM32L0xx_HAL_Driver/Src/stm32l0xx_hal_rcc.o
                0x0000000008019020                HAL_RCC_ClockConfig
 .text.HAL_RCC_GetSysClockFreq
                0x0000000008019274      0x10c ./Drivers/STM32L0xx_HAL_Driver/Src/stm32l0xx_hal_rcc.o
                0x0000000008019274                HAL_RCC_GetSysClockFreq
 .text.HAL_RCC_GetHCLKFreq
                0x0000000008019380       0x14 ./Drivers/STM32L0xx_HAL_Driver/Src/stm32l0xx_hal_rcc.o
                0x0000000008019380                HAL_RCC_GetHCLKFreq
 .text.HAL_RCC_GetPCLK1Freq
                0x0000000008019394       0x2c ./Drivers/STM32L0xx_HAL_Driver/Src/stm32l0xx_hal_rcc.o
                0x0000000008019394                HAL_RCC_GetPCLK1Freq
 .text.HAL_RCC_GetPCLK2Freq
                0x00000000080193c0       0x2c ./Drivers/STM32L0xx_HAL_Driver/Src/stm32l0xx_hal_rcc.o
                0x00000000080193c0                HAL_RCC_GetPCLK2Freq
 .text.HAL_RCCEx_PeriphCLKConfig
                0x00000000080193ec      0x2ac ./Drivers/STM32L0xx_HAL_Driver/Src/stm32l0xx_hal_rcc_ex.o
                0x00000000080193ec                HAL_RCCEx_PeriphCLKConfig
 .text.HAL_RTC_Init
                0x0000000008019698      0x13c ./Drivers/STM32L0xx_HAL_Driver/Src/stm32l0xx_hal_rtc.o
                0x0000000008019698                HAL_RTC_Init
 .text.HAL_RTC_SetTime
                0x00000000080197d4      0x188 ./Drivers/STM32L0xx_HAL_Driver/Src/stm32l0xx_hal_rtc.o
                0x00000000080197d4                HAL_RTC_SetTime
 .text.HAL_RTC_GetTime
                0x000000000801995c       0xb8 ./Drivers/STM32L0xx_HAL_Driver/Src/stm32l0xx_hal_rtc.o
                0x000000000801995c                HAL_RTC_GetTime
 .text.HAL_RTC_SetDate
                0x0000000008019a14      0x15c ./Drivers/STM32L0xx_HAL_Driver/Src/stm32l0xx_hal_rtc.o
                0x0000000008019a14                HAL_RTC_SetDate
 .text.HAL_RTC_GetDate
                0x0000000008019b70       0x9c ./Drivers/STM32L0xx_HAL_Driver/Src/stm32l0xx_hal_rtc.o
                0x0000000008019b70                HAL_RTC_GetDate
 .text.HAL_RTC_SetAlarm_IT
                0x0000000008019c0c      0x298 ./Drivers/STM32L0xx_HAL_Driver/Src/stm32l0xx_hal_rtc.o
                0x0000000008019c0c                HAL_RTC_SetAlarm_IT
 .text.HAL_RTC_DeactivateAlarm
                0x0000000008019ea4      0x140 ./Drivers/STM32L0xx_HAL_Driver/Src/stm32l0xx_hal_rtc.o
                0x0000000008019ea4                HAL_RTC_DeactivateAlarm
 .text.HAL_RTC_WaitForSynchro
                0x0000000008019fe4       0x4e ./Drivers/STM32L0xx_HAL_Driver/Src/stm32l0xx_hal_rtc.o
                0x0000000008019fe4                HAL_RTC_WaitForSynchro
 .text.RTC_EnterInitMode
                0x000000000801a032       0x54 ./Drivers/STM32L0xx_HAL_Driver/Src/stm32l0xx_hal_rtc.o
                0x000000000801a032                RTC_EnterInitMode
 .text.RTC_ByteToBcd2
                0x000000000801a086       0x50 ./Drivers/STM32L0xx_HAL_Driver/Src/stm32l0xx_hal_rtc.o
                0x000000000801a086                RTC_ByteToBcd2
 .text.RTC_Bcd2ToByte
                0x000000000801a0d6       0x3a ./Drivers/STM32L0xx_HAL_Driver/Src/stm32l0xx_hal_rtc.o
                0x000000000801a0d6                RTC_Bcd2ToByte
 .text.HAL_RTCEx_BKUPWrite
                0x000000000801a110       0x2c ./Drivers/STM32L0xx_HAL_Driver/Src/stm32l0xx_hal_rtc_ex.o
                0x000000000801a110                HAL_RTCEx_BKUPWrite
 .text.HAL_RTCEx_BKUPRead
                0x000000000801a13c       0x28 ./Drivers/STM32L0xx_HAL_Driver/Src/stm32l0xx_hal_rtc_ex.o
                0x000000000801a13c                HAL_RTCEx_BKUPRead
 .text.HAL_RTCEx_EnableBypassShadow
                0x000000000801a164       0x68 ./Drivers/STM32L0xx_HAL_Driver/Src/stm32l0xx_hal_rtc_ex.o
                0x000000000801a164                HAL_RTCEx_EnableBypassShadow
 .text.HAL_SPI_Init
                0x000000000801a1cc       0xd4 ./Drivers/STM32L0xx_HAL_Driver/Src/stm32l0xx_hal_spi.o
                0x000000000801a1cc                HAL_SPI_Init
 .text.HAL_SPI_MspInit
                0x000000000801a2a0       0x10 ./Drivers/STM32L0xx_HAL_Driver/Src/stm32l0xx_hal_spi.o
                0x000000000801a2a0                HAL_SPI_MspInit
 .text.HAL_SPI_TransmitReceive
                0x000000000801a2b0      0x376 ./Drivers/STM32L0xx_HAL_Driver/Src/stm32l0xx_hal_spi.o
                0x000000000801a2b0                HAL_SPI_TransmitReceive
 *fill*         0x000000000801a626        0x2 
 .text.SPI_WaitFlagStateUntilTimeout
                0x000000000801a628       0xe0 ./Drivers/STM32L0xx_HAL_Driver/Src/stm32l0xx_hal_spi.o
 .text.SPI_EndRxTxTransaction
                0x000000000801a708       0x7a ./Drivers/STM32L0xx_HAL_Driver/Src/stm32l0xx_hal_spi.o
 .text.HAL_TIM_Base_Init
                0x000000000801a782       0x58 ./Drivers/STM32L0xx_HAL_Driver/Src/stm32l0xx_hal_tim.o
                0x000000000801a782                HAL_TIM_Base_Init
 .text.HAL_TIM_Base_Start
                0x000000000801a7da       0x44 ./Drivers/STM32L0xx_HAL_Driver/Src/stm32l0xx_hal_tim.o
                0x000000000801a7da                HAL_TIM_Base_Start
 *fill*         0x000000000801a81e        0x2 
 .text.TIM_Base_SetConfig
                0x000000000801a820       0xbc ./Drivers/STM32L0xx_HAL_Driver/Src/stm32l0xx_hal_tim.o
 .text.HAL_TIMEx_MasterConfigSynchronization
                0x000000000801a8dc       0x86 ./Drivers/STM32L0xx_HAL_Driver/Src/stm32l0xx_hal_tim_ex.o
                0x000000000801a8dc                HAL_TIMEx_MasterConfigSynchronization
 *fill*         0x000000000801a962        0x2 
 .text.HAL_UART_Init
                0x000000000801a964       0xa8 ./Drivers/STM32L0xx_HAL_Driver/Src/stm32l0xx_hal_uart.o
                0x000000000801a964                HAL_UART_Init
 .text.HAL_UART_Transmit_DMA
                0x000000000801aa0c      0x120 ./Drivers/STM32L0xx_HAL_Driver/Src/stm32l0xx_hal_uart.o
                0x000000000801aa0c                HAL_UART_Transmit_DMA
 .text.HAL_UART_IRQHandler
                0x000000000801ab2c      0x248 ./Drivers/STM32L0xx_HAL_Driver/Src/stm32l0xx_hal_uart.o
                0x000000000801ab2c                HAL_UART_IRQHandler
 .text.HAL_UART_TxHalfCpltCallback
                0x000000000801ad74       0x10 ./Drivers/STM32L0xx_HAL_Driver/Src/stm32l0xx_hal_uart.o
                0x000000000801ad74                HAL_UART_TxHalfCpltCallback
 .text.HAL_UART_ErrorCallback
                0x000000000801ad84       0x10 ./Drivers/STM32L0xx_HAL_Driver/Src/stm32l0xx_hal_uart.o
                0x000000000801ad84                HAL_UART_ErrorCallback
 .text.UART_SetConfig
                0x000000000801ad94      0x62c ./Drivers/STM32L0xx_HAL_Driver/Src/stm32l0xx_hal_uart.o
                0x000000000801ad94                UART_SetConfig
 .text.UART_AdvFeatureConfig
                0x000000000801b3c0      0x168 ./Drivers/STM32L0xx_HAL_Driver/Src/stm32l0xx_hal_uart.o
                0x000000000801b3c0                UART_AdvFeatureConfig
 .text.UART_CheckIdleState
                0x000000000801b528       0x88 ./Drivers/STM32L0xx_HAL_Driver/Src/stm32l0xx_hal_uart.o
                0x000000000801b528                UART_CheckIdleState
 .text.UART_WaitOnFlagUntilTimeout
                0x000000000801b5b0       0x94 ./Drivers/STM32L0xx_HAL_Driver/Src/stm32l0xx_hal_uart.o
                0x000000000801b5b0                UART_WaitOnFlagUntilTimeout
 .text.UART_EndTxTransfer
                0x000000000801b644       0x26 ./Drivers/STM32L0xx_HAL_Driver/Src/stm32l0xx_hal_uart.o
 *fill*         0x000000000801b66a        0x2 
 .text.UART_EndRxTransfer
                0x000000000801b66c       0x40 ./Drivers/STM32L0xx_HAL_Driver/Src/stm32l0xx_hal_uart.o
 .text.UART_DMATransmitCplt
                0x000000000801b6ac       0x54 ./Drivers/STM32L0xx_HAL_Driver/Src/stm32l0xx_hal_uart.o
 .text.UART_DMATxHalfCplt
                0x000000000801b700       0x1e ./Drivers/STM32L0xx_HAL_Driver/Src/stm32l0xx_hal_uart.o
 .text.UART_DMAError
                0x000000000801b71e       0x7e ./Drivers/STM32L0xx_HAL_Driver/Src/stm32l0xx_hal_uart.o
 .text.UART_DMAAbortOnError
                0x000000000801b79c       0x2e ./Drivers/STM32L0xx_HAL_Driver/Src/stm32l0xx_hal_uart.o
 .text.UART_EndTransmit_IT
                0x000000000801b7ca       0x34 ./Drivers/STM32L0xx_HAL_Driver/Src/stm32l0xx_hal_uart.o
 .text.HAL_UARTEx_WakeupCallback
                0x000000000801b7fe       0x10 ./Drivers/STM32L0xx_HAL_Driver/Src/stm32l0xx_hal_uart_ex.o
                0x000000000801b7fe                HAL_UARTEx_WakeupCallback
 .text.atoi     0x000000000801b80e        0xc /opt/st/stm32cubeide_1.9.0/plugins/com.st.stm32cube.ide.mcu.externaltools.gnu-tools-for-stm32.10.3-2021.10.linux64_1.0.0.202111181127/tools/bin/../lib/gcc/arm-none-eabi/10.3.1/../../../../arm-none-eabi/lib/thumb/v6-m/nofp/libc_nano.a(lib_a-atoi.o)
                0x000000000801b80e                atoi
 *fill*         0x000000000801b81a        0x2 
 .text.__libc_init_array
                0x000000000801b81c       0x48 /opt/st/stm32cubeide_1.9.0/plugins/com.st.stm32cube.ide.mcu.externaltools.gnu-tools-for-stm32.10.3-2021.10.linux64_1.0.0.202111181127/tools/bin/../lib/gcc/arm-none-eabi/10.3.1/../../../../arm-none-eabi/lib/thumb/v6-m/nofp/libc_nano.a(lib_a-init.o)
                0x000000000801b81c                __libc_init_array
 .text.memset   0x000000000801b864       0x10 /opt/st/stm32cubeide_1.9.0/plugins/com.st.stm32cube.ide.mcu.externaltools.gnu-tools-for-stm32.10.3-2021.10.linux64_1.0.0.202111181127/tools/bin/../lib/gcc/arm-none-eabi/10.3.1/../../../../arm-none-eabi/lib/thumb/v6-m/nofp/libc_nano.a(lib_a-memset.o)
                0x000000000801b864                memset
 .text.validate_structure
                0x000000000801b874      0x194 /opt/st/stm32cubeide_1.9.0/plugins/com.st.stm32cube.ide.mcu.externaltools.gnu-tools-for-stm32.10.3-2021.10.linux64_1.0.0.202111181127/tools/bin/../lib/gcc/arm-none-eabi/10.3.1/../../../../arm-none-eabi/lib/thumb/v6-m/nofp/libc_nano.a(lib_a-mktime.o)
 .text.mktime   0x000000000801ba08      0x39c /opt/st/stm32cubeide_1.9.0/plugins/com.st.stm32cube.ide.mcu.externaltools.gnu-tools-for-stm32.10.3-2021.10.linux64_1.0.0.202111181127/tools/bin/../lib/gcc/arm-none-eabi/10.3.1/../../../../arm-none-eabi/lib/thumb/v6-m/nofp/libc_nano.a(lib_a-mktime.o)
                0x000000000801ba08                mktime
 .text.__cvt    0x000000000801bda4       0xc6 /opt/st/stm32cubeide_1.9.0/plugins/com.st.stm32cube.ide.mcu.externaltools.gnu-tools-for-stm32.10.3-2021.10.linux64_1.0.0.202111181127/tools/bin/../lib/gcc/arm-none-eabi/10.3.1/../../../../arm-none-eabi/lib/thumb/v6-m/nofp/libc_nano.a(lib_a-nano-vfprintf_float.o)
                0x000000000801bda4                __cvt
 .text.__exponent
                0x000000000801be6a       0x8e /opt/st/stm32cubeide_1.9.0/plugins/com.st.stm32cube.ide.mcu.externaltools.gnu-tools-for-stm32.10.3-2021.10.linux64_1.0.0.202111181127/tools/bin/../lib/gcc/arm-none-eabi/10.3.1/../../../../arm-none-eabi/lib/thumb/v6-m/nofp/libc_nano.a(lib_a-nano-vfprintf_float.o)
                0x000000000801be6a                __exponent
 .text._printf_float
                0x000000000801bef8      0x484 /opt/st/stm32cubeide_1.9.0/plugins/com.st.stm32cube.ide.mcu.externaltools.gnu-tools-for-stm32.10.3-2021.10.linux64_1.0.0.202111181127/tools/bin/../lib/gcc/arm-none-eabi/10.3.1/../../../../arm-none-eabi/lib/thumb/v6-m/nofp/libc_nano.a(lib_a-nano-vfprintf_float.o)
                0x000000000801bef8                _printf_float
 .text._printf_common
                0x000000000801c37c       0xde /opt/st/stm32cubeide_1.9.0/plugins/com.st.stm32cube.ide.mcu.externaltools.gnu-tools-for-stm32.10.3-2021.10.linux64_1.0.0.202111181127/tools/bin/../lib/gcc/arm-none-eabi/10.3.1/../../../../arm-none-eabi/lib/thumb/v6-m/nofp/libc_nano.a(lib_a-nano-vfprintf_i.o)
                0x000000000801c37c                _printf_common
 *fill*         0x000000000801c45a        0x2 
 .text._printf_i
                0x000000000801c45c      0x224 /opt/st/stm32cubeide_1.9.0/plugins/com.st.stm32cube.ide.mcu.externaltools.gnu-tools-for-stm32.10.3-2021.10.linux64_1.0.0.202111181127/tools/bin/../lib/gcc/arm-none-eabi/10.3.1/../../../../arm-none-eabi/lib/thumb/v6-m/nofp/libc_nano.a(lib_a-nano-vfprintf_i.o)
                0x000000000801c45c                _printf_i
 .text._scanf_float
                0x000000000801c680      0x410 /opt/st/stm32cubeide_1.9.0/plugins/com.st.stm32cube.ide.mcu.externaltools.gnu-tools-for-stm32.10.3-2021.10.linux64_1.0.0.202111181127/tools/bin/../lib/gcc/arm-none-eabi/10.3.1/../../../../arm-none-eabi/lib/thumb/v6-m/nofp/libc_nano.a(lib_a-nano-vfscanf_float.o)
                0x000000000801c680                _scanf_float
 .text.nanf     0x000000000801ca90        0x8 /opt/st/stm32cubeide_1.9.0/plugins/com.st.stm32cube.ide.mcu.externaltools.gnu-tools-for-stm32.10.3-2021.10.linux64_1.0.0.202111181127/tools/bin/../lib/gcc/arm-none-eabi/10.3.1/../../../../arm-none-eabi/lib/thumb/v6-m/nofp/libc_nano.a(lib_a-sf_nan.o)
                0x000000000801ca90                nanf
 .text.sprintf  0x000000000801ca98       0x40 /opt/st/stm32cubeide_1.9.0/plugins/com.st.stm32cube.ide.mcu.externaltools.gnu-tools-for-stm32.10.3-2021.10.linux64_1.0.0.202111181127/tools/bin/../lib/gcc/arm-none-eabi/10.3.1/../../../../arm-none-eabi/lib/thumb/v6-m/nofp/libc_nano.a(lib_a-sprintf.o)
                0x000000000801ca98                sprintf
                0x000000000801ca98                siprintf
 .text.sulp     0x000000000801cad8       0x30 /opt/st/stm32cubeide_1.9.0/plugins/com.st.stm32cube.ide.mcu.externaltools.gnu-tools-for-stm32.10.3-2021.10.linux64_1.0.0.202111181127/tools/bin/../lib/gcc/arm-none-eabi/10.3.1/../../../../arm-none-eabi/lib/thumb/v6-m/nofp/libc_nano.a(lib_a-strtod.o)
 .text._strtod_l
                0x000000000801cb08      0xc28 /opt/st/stm32cubeide_1.9.0/plugins/com.st.stm32cube.ide.mcu.externaltools.gnu-tools-for-stm32.10.3-2021.10.linux64_1.0.0.202111181127/tools/bin/../lib/gcc/arm-none-eabi/10.3.1/../../../../arm-none-eabi/lib/thumb/v6-m/nofp/libc_nano.a(lib_a-strtod.o)
                0x000000000801cb08                _strtod_l
 .text._strtod_r
                0x000000000801d730       0x10 /opt/st/stm32cubeide_1.9.0/plugins/com.st.stm32cube.ide.mcu.externaltools.gnu-tools-for-stm32.10.3-2021.10.linux64_1.0.0.202111181127/tools/bin/../lib/gcc/arm-none-eabi/10.3.1/../../../../arm-none-eabi/lib/thumb/v6-m/nofp/libc_nano.a(lib_a-strtod.o)
